:1000000000000120D5020100FD020100FF020100F5
:1000100001030100030301000503010000000000CB
:1000200000000000000000000000000007030100C5
:1000300009030100000000000B0301000D03010093
:100040000F0301000F0301008D0801000F030100E1
:1000500071AC00000F0301000F0301000F0301004A
:100060000F0301000F0301000F0301000F03010044
:100070000F0301000F0301000F0301000F03010034
:100080000F030100510C01000F0301000F030100D9
:100090000F0301000F0301000F0301000F03010014
:1000A0000F0301000F0301000F0301000F03010004
:1000B0000F0301000F03010000000000000000001A
:1000C0000F0301000F0301000F0301000F030100E4
:1000D0000F0301000F0301000F03010000000000E7
:1000E0000000000000000000000000000000000010
:1000F0000000000000000000000000000000000000
:1001000000000000000000000000000000000000EF
:1001100000000000000000000000000000000000DF
:1001200000000000000000000000000000000000CF
:1001300000000000000000000000000000000000BF
:1001400000000000000000000000000000000000AF
:10015000000000000000000000000000000000009F
:10016000000000000000000000000000000000008F
:10017000000000000000000000000000000000007F
:10018000000000000000000000000000000000006F
:10019000000000000000000000000000000000005F
:1001A000000000000000000000000000000000004F
:1001B000000000000000000000000000000000003F
:1001C000000000000000000000000000000000002F
:1001D000000000000000000000000000000000001F
:1001E000000000000000000000000000000000000F
:1001F00000000000000000000000000000000000FF
:1002000010B5054C237833B9044B13B10448AFF350
:1002100000800123237010BDA00200200000000018
:1002200010A1010008B5034B1BB103490348AFF30C
:10023000008008BD00000000A402002010A1010001
:10024000154B002B08BF134B9D46A3F5803A0021A8
:100250008B460F461348144A121A13F02AF80F4B14
:10026000002B00D098470E4B002B00D09847002061
:10027000002104000D000D48002802D00C48AFF307
:10028000008012F05FFF2000290010F021FD12F025
:10029000A7FD00BF000008000000012000000000D2
:1002A00000000000A00200208809002000000000DB
:1002B000000000000020704700207047F0B50446A1
:1002C00085B00E46684611461F460AF051F823686D
:1002D0006A465D6A31463B462046A84705B0F0BDF8
:1002E000F0B5044685B00E46684611461F4609F033
:1002F0004EFF23686A465D6A31463B462046A84762
:1003000005B0F0BD70B590B00C4615461E4605F020
:10031000F5FD48B364B321464022684613F09DFFC3
:100320002F21684613F030FF28B9234603224021CD
:10033000684609F09FFF3F223146684613F067FF89
:100340000C480EF08FFE78B10B4B93F90030062B62
:100350000CD10A4B93F9003043B901232A46694670
:1003600004480FF0DCF8012010B070BD0020FBE75E
:100370002046F9E7E8030020E0030020B80300204E
:1003800007B5002300931A46194603480FF0DAFD1B
:1003900003B05DF804FB00BFBC02002007B50023DA
:1003A00000931A46194603480FF0CCFD03B05DF8E0
:1003B00004FB00BFC402002082B002AB012003E9AD
:1003C000060002B0704700207047406818B14068CE
:1003D00008B1007C0009704743682BB15B681BB112
:1003E0001A7C61F307121A747047406808B508B1A7
:1003F00001F08CFF012008BD13B500220446114610
:10040000684604F01BF9606801F080FF052807D8F2
:10041000DFE800F0110311060611012002B010BD43
:1004200061684FF40072684604F0FAFC00216846E7
:1004300004F0C6FBF2E70020F0E713B50022044603
:100440001146684604F0FAF82046FF22694604F097
:1004500032FC204602B010BD07B5002300931A46B7
:10046000194603480FF06EFD03B05DF804FB00BFB2
:10047000CC020020704700002DE9FF4102AC84E867
:10048000060006463B493C489DF828809DF82C50C4
:100490001F460FF09FFD204604F0B0FE204604F0FA
:1004A0004BFA50BB204604F0ADFC052804D8DFE829
:1004B00000F0152417030317054630492E480FF0A6
:1004C00089FD0A2229462C480FF0EDFD2A480FF03D
:1004D00091FD204604F092FE00200BE04FF0010851
:1004E000CDE90085336894E80600DD6B30463B4675
:1004F000A847012004B0BDE8F081204604F0CCFB01
:10050000012812D0022831D01D491B480FF062FD8E
:10051000204604F0C1FB0A22014617480FF0DCFD1B
:1005200015480FF067FD0125C7E70021204604F0BC
:1005300099FA13280ED81E21204604F003FB716897
:100540004FF40072204604F0C0FC4FF490517068E4
:1005500002F050FD0195336801250095D3F83C80E9
:1005600094E806003B463046C047C2E700230393A9
:10057000F0E700BFF47C0100700300200A7D010059
:10058000FD7C010008B511B9B0F9080008BDB0F94B
:100590000A208A4203DC0089084400B2F6E740687A
:1005A00001F04CFFF9E7000007B5002300931A465D
:1005B000194603480FF0C6FC03B05DF804FB00BF0A
:1005C000D40200200A460068022100F0A1BD00000C
:1005D00070B503680546F3B17221FFF7F3FF286891
:1005E0000E4E03680021DB69984700242868042C1C
:1005F00003680CD0DB689847A35D984205D0286853
:1006000003685B6A9847002070BD0134EEE75B6ABF
:1006100098470120F8E71846F6E700BF647D01001F
:100620002DE9F041036804461BB900263046BDE8B9
:10063000F081FFF7CDFF07460028F6D0254672214E
:100640002046FFF7BFFF55F8100B03680421DB6954
:10065000984704F11608002620680368DB6898476D
:10066000C0B205F8010B0138C0B2FD2898BF3E4664
:10067000A845F1D1206803685B6A9847D6E7F8B5CA
:10068000036804460F4613B900252846F8BDFFF756
:100690009FFF05460028F7D072212046FFF792FF02
:1006A000206803682646DB690421984756F8100B3A
:1006B000036806225B68394698473B682361BB881C
:1006C000B380206803685B6A9847DEE770B503680B
:1006D00004460D46164613B90025284670BDFFF79F
:1006E00077FF0028F8D072212046FFF76BFF2068C3
:1006F00003684021DB699847731E2A460021206861
:100700000FF04CFF06B2206803685B6A9847002E22
:10071000E2D00023AB55E0E738B5036804460D4648
:100720000BB9002038BDFFF753FF0028F9D0284649
:1007300013F065FD0F28F4D872212046FFF742FF21
:10074000206803684021DB699847294620680FF03C
:100750004AFC2068036800211B689847054620680A
:1007600003685B6A9847281C18BF0120DAE738B590
:10077000036804460D460BB9002038BDFFF728FF7B
:100780000028F9D0284613F03AFD0F28F4D872213A
:100790002046FFF717FF206803685021DB69984760
:1007A000294620680FF01FFC2068036800211B68A1
:1007B00098470546206803685B6A9847281C18BF5D
:1007C0000120DAE770B5036804460D46164613B9F2
:1007D0000025284670BDFFF7FBFE0028F8D07221E7
:1007E0002046FFF7EFFE206803682021DB69984769
:1007F000731E2A46002120680FF0D0FE06B2206842
:1008000003685B6A9847002EE2D00023AB55E0E70F
:1008100038B5036804460D460BB9002038BDFFF714
:10082000D7FE0028F9D0284613F0E9FC1F28F4D899
:1008300072212046FFF7C6FE206803682021DB698D
:100840009847294620680FF0CEFB206803680021F6
:100850001B6898470546206803685B6A9847281C10
:1008600018BF0120DAE773B5036805460E461BB9C9
:100870000024204602B070BDFFF7AAFE04460028FF
:10088000F6D072212846FFF79DFE286803681021E4
:10089000DB69984704220DEB020128680FF069FE1E
:1008A000019930460FF06BFB286803685B6A984734
:1008B0003379002BDCD0FF2BDBD17379FF2BD8D120
:1008C000B379FF2BD5D1F479FF3C18BF0124D0E7D1
:1008D00073B5036805460E461BB90024204602B0D6
:1008E00070BDFFF775FE04460028F6D07221284639
:1008F000FFF768FE286803681C21DB69984704221B
:100900000DEB020128680FF034FE019930460FF01C
:1009100036FB286803685B6A98473379002BDCD084
:10092000FF2BDBD17379FF2BD8D1B379FF2BD5D136
:10093000F479FF3C18BF0124D0E773B5036805467E
:100940000E461BB90024204602B070BDFFF740FEE2
:1009500004460028F6D072212846FFF733FE2868A7
:1009600003681421DB69984704220DEB0201286813
:100970000FF0FFFD019930460FF001FB2868036876
:100980005B6A98473379002BDCD0FF2BDBD173797E
:10099000FF2BD8D1B379FF2BD5D1F479FF3C18BF09
:1009A0000124D0E773B5036805460E461BB9002441
:1009B000204602B070BDFFF70BFE04460028F6D0BB
:1009C00072212846FFF7FEFD286803681821DB69BD
:1009D000984704220DEB020128680FF0CAFD019927
:1009E00030460FF0CCFA286803685B6A9847337981
:1009F000002BDCD0FF2BDBD17379FF2BD8D1B3795F
:100A0000FF2BD5D1F479FF3C18BF0124D0E737B5CF
:100A10004B6801930368044613B9002003B030BD4E
:100A2000FFF7D6FD0028F8D072212046FFF7CAFD57
:100A3000206803681021DB69984720680368042256
:100A40005B680DEB020198470546206803685B6A06
:100A50009847281C18BF0120E0E737B54B68019381
:100A60000368044613B9002003B030BDFFF7B0FDA2
:100A70000028F8D072212046FFF7A4FD2068036803
:100A80001C21DB6998472068036804225B680DEB32
:100A9000020198470546206803685B6A9847281C4E
:100AA00018BF0120E0E737B54B680193036804469F
:100AB00013B9002003B030BDFFF78AFD0028F8D03D
:100AC00072212046FFF77EFD206803681421DB6950
:100AD00098472068036804225B680DEB0201984781
:100AE0000546206803685B6A9847281C18BF0120E8
:100AF000E0E737B54B6801930368044613B900205B
:100B000003B030BDFFF764FD0028F8D07221204605
:100B1000FFF758FD206803681821DB6998472068B3
:100B2000036804225B680DEB0201984705462068C4
:100B300003685B6A9847281C18BF0120E0E713B5DB
:100B4000E723009303680446A3B1FFF741FD88B192
:100B500072212046FFF736FD206803680C21DB690F
:100B600098470422694620680FF003FD2068036857
:100B70005B6A9847009B0020DAB262F30700C3F378
:100B8000072262F30F20C3F3074262F317401B0EE4
:100B900063F31F6002B010BD37B5019103680446CE
:100BA00013B9002003B030BDFFF712FD0028F8D0C4
:100BB00072212046FFF706FD206803680C21DB69DF
:100BC00098472068036804225B680DEB0201984790
:100BD0000546206803685B6A9847281C18BF0120F7
:100BE000E0E707B5FFF7ABFF80F48070C0F30020AB
:100BF00003B05DF804FB37B505460C46FFF79FFFD1
:100C000084F001040190C0F3072064F300008DF824
:100C100005000199284603B0BDE83040FFF7BCBF8E
:100C200007B5FFF78CFFC0F3402003B05DF804FB6D
:100C300037B50D460446FFF782FF0190C0F3072049
:100C400065F341008DF805000199204603B0BDE829
:100C50003040FFF7A1BF07B5FFF771FF80F010002C
:100C6000C0F3001003B05DF804FB37B505460C4631
:100C7000FFF765FF84F00104019064F304108DF820
:100C800004000199284603B0BDE83040FFF784BF57
:100C900037B50D460446FFF752FF019065F3030098
:100CA0008DF804000199204603B0BDE83040FFF7FD
:100CB00073BF37B50D460446FFF741FF019065F35A
:100CC00047108DF804000199204603B0BDE830407C
:100CD000FFF762BF07B5FFF732FF00F00F0003B068
:100CE0005DF804FB07B5FFF72AFFC0F3421003B01D
:100CF0005DF804FB70B51E4D0C468AB00646043400
:100D00001C4928460FF066F9214607A80FF083FE1C
:100D100007A928460FF062F92846174D0FF06AF927
:100D200007A80FF0E8FD294601A80FF029FE01A948
:100D300004A80FF070FE214604A80FF0ACFE29466F
:100D4000044607A80FF01CFE07A920460FF0A3FEDB
:100D5000014630460FF05FFE07A80FF0CCFD04A857
:100D60000FF0C9FD01A80FF0C6FD30460AB070BDF6
:100D700070030020697D0100747D01007FB50D4680
:100D80000446222128460FF0DBFE22210646284693
:100D90000FF0F0FE002E034604F1040422DB0028CD
:100DA00020DD721C294601A80FF0E8FE01A92046AB
:100DB0000FF03BFE01A80FF09EFD0D490D480FF00E
:100DC00009F9214601A80FF026FE01A909480FF0F4
:100DD00005F908480FF00EF901A80FF08CFD01206D
:100DE00004B070BD294620460FF006FEE5E700BFBF
:100DF000767D0100700300207FB503680446002B58
:100E000039D07721FFF7DEFB206803680021DB691A
:100E100098470025206802690368954204D21B6840
:100E2000002198470135F5E7DB69144E002198470A
:100E300000252068715D036801351B689847042D03
:100E4000F7D1206803685B6A98470D4901A80FF045
:100E500097FD01A92046FFF791FF01A80FF04BFD78
:100E600007212046FFF714FF07212046FFF721FF47
:100E7000012004B070BD1846FBE700BF647D01008F
:100E8000CA9B01007FB50368044613B9002004B073
:100E900070BDFFF79DFB0028F8D0E3681F2BF5D845
:100EA000264672212046FFF78DFB56F8040B036897
:100EB0006021DB699847314620680FF08FF8206881
:100EC000036800211B6898470546206803685B6A31
:100ED00098478DB10A490B480FF07CF8314601A8BC
:100EE0000FF099FD01A907480FF078F805480FF0B9
:100EF00081F801A80FF0FFFC281C18BF0120C6E7ED
:100F00008E7D01007003002030B5036885B0044673
:100F100013B9002005B030BDFFF75AFB0028F8D008
:100F2000254672212046FFF74DFB55F8040B036858
:100F30006021DB6998470022216801A80FF048FB77
:100F400001A928460FF071FD01A80FF0D4FC20681C
:100F500003685B6A98470B490B480FF03BF829463A
:100F600001A80FF058FD01A907480FF037F806480F
:100F70000FF040F801A80FF0BEFCE068003018BF89
:100F80000120C7E7817D01007003002007B5002321
:100F900000931A46194603480EF0D4FF03B05DF8DB
:100FA00004FB00BFDC02002007B5002300931A46B3
:100FB000194603480EF0C6FF03B05DF804FB00BFFE
:100FC000E402002001207047C08A704703699942FB
:100FD00028BF1946816108467047037D10B5044655
:100FE00033B9A069236998422CBF0020012010BDAD
:100FF00003681B699847FF28F3D10020F7E70368CF
:1010000010B504461B699847A3690133A36110BD5D
:101010007047000008B502698369934205D2C1692F
:10102000034819440EF0DDFD08BD4FF0FF30FBE72B
:10103000EC02002010B5D0E906345A1C82610A4641
:101040000248E1180EF0CFFD012010BDEC02002097
:10105000037D10B504462BB10368FF211B68984738
:101060000023237510BD000008B590F82020772AD2
:101070000BD10368DB6A9847044905480EF0AAFFC4
:101080000348BDE808400EF0B5BF08BDB37D0100C0
:1010900070030020F0B50D4685B004463F21284678
:1010A00017460FF04DFD031E0BDB0022294601A859
:1010B0000FF064FD01A928460FF0B7FC01A80FF05E
:1010C0001AFC114928460FF0F2FC064660B10023D5
:1010D000A3614FF4FA43236101208423E361207567
:1010E00084F8207005B0F0BD084928460FF0DFFCF9
:1010F0000028F7D08423C4E906662361267584F8A6
:1011000020700120EEE700BF9A7D0100A77D01005D
:1011100001294FF0000303D002290CD01846704774
:1011200083614FF4FA4303618423C361017580F83E
:101130002020012070478421C0E906330161037536
:10114000F5E7000007B5002300931A461946044846
:101150000EF0F8FE034803B05DF804EB0EF03EBD60
:10116000ED020020EC02002038B50023836083806C
:101170008371036804460D46002B4CD0344A126834
:10118000002A48D0002908BF1D462B7C03F00F031E
:10119000062B15D12F4A304829460DF012FC08B114
:1011A000436923712D4A2C4829460DF00AFC00287A
:1011B00049D0037C03F00F03022B2DD0052B2ED03A
:1011C000274A216824480DF0FCFB054608BB254949
:1011D00025480EF0FFFE0A22617923480EF07CFFBD
:1011E000224921480EF0F6FE0A2221791E480EF00F
:1011F00073FF1D480EF0FEFE2B46194A2168164863
:101200000DF027FC164A216813480DF0DAFB05465D
:1012100008B11435A56038BD43696371D0E7C36870
:10122000002BCDD01A7C02F00F02022AC8D15A69D5
:101230006271DB68002BC3D01A7C02F00F02022A15
:10124000BED15B69E9E7286811F0ADFD6071B7E7D1
:1012500038040020089B010078070020FC7D010075
:10126000627E0100657E0100700300201B8B01007F
:1012700010B5044601601146FFF776FF204610BD09
:1012800070B5044686B028B3037C03F00F03062B29
:1012900020D106A8002140F8184DFFF765FF029BFA
:1012A0000D4A0E4800261E6021460DF08AFB88B1CB
:1012B000037C03F00F03052B0CD1C56855B1214603
:1012C00003A80395FFF750FF059B1E600FF0D4FCA9
:1012D0006D68F3E706B070BDF07D0100780700206F
:1012E00038B583680446BBB1124B1B68A3B10068D4
:1012F000FFF7C6FFA36800251D602379032B0CD8D8
:10130000012B94BF0221294660790FF04DFEA3689E
:101310005A7865F303025A7038BD402B03D0422B34
:10132000FAD1294600E002216079BDE838400FF08B
:101330003BBE00BF3804002041790C4A002352F81C
:101340002300884203D10A4A52F82300704752F81A
:10135000230028B942F82310054A42F823007047B9
:101360000133052BEBD10020704700BF04030020A0
:101370001803002010B50A4A4079002352F8234090
:10138000844203D1074A42F8231010BD52F823408B
:1013900014B952F82320F5E70133052BEED1F4E719
:1013A0000403002018030020F0B52DED028B9DB042
:1013B0000446FFF7C1FF05460FF008FC0023014675
:1013C00043F69822284608F0E9FF002800F0E9805B
:1013D00006231622617907A80EF0FAF9372107A82B
:1013E0000EF006FA0022114607A80EF01DFB0021A0
:1013F00008EE900A07A80EF0AFFB6C4908EE100A41
:101400006B480EF0E7FD0A22617969480EF064FE30
:10141000684967480EF0DEFD18EE900A11F002F9F7
:10142000022502460B46009561480EF011FF624905
:101430005F480EF0CFFD18EE100A11F0F3F800959A
:101440000B4602465A480EF003FF5C4958480EF01E
:10145000C1FD57480EF0CEFD594A216859480DF09C
:10146000B0FA594A2168074656480DF0AAFAF4EE38
:10147000688AF1EE10FA064610D60CAD18EE901AF6
:10148000284603F0E8F80023CDE90133009395E8FE
:101490000C004FF0FF31384608F09AFFB4EE488A4E
:1014A000F1EE10FA10D60CAD18EE101A284603F023
:1014B000D2F80023CDE90133009395E80C004FF0FA
:1014C000FF31304608F084FF404A21683D480DF066
:1014D00078FA054600285ED0037C03F00F03042B46
:1014E00059D1F5EE408AF1EE10FA54D0B5EE408AAB
:1014F000F1EE10FA4FD0F4EE688AF1EE10FA4AD10C
:10150000B4EE488AF1EE10FA45D100213C220DA834
:101510000C9111F0CEFE696940220CA812F09DFEDC
:101520002F210CA812F030FE28B96B69032240214C
:101530000CA808F09FFE26490CA812F016FE04A87D
:1015400018EE901A08F023FE22480DF08BFD40B1F2
:10155000214B93F9003023B904AA0CA91D480DF0C2
:10156000C9FF0CA812F04BFE1CAB1844482300F82E
:10157000413C18EE101A04A808F009FE15480DF0B9
:1015800071FD40B1144B93F9003023B904AA0CA9A2
:1015900010480DF0AFFF0FF019FB01462046FFF792
:1015A000E9FE1DB0BDEC028BF0BD00BF5E7E010008
:1015B000700300206A7E01007A7E0100817E0100B6
:1015C000837E010078070020887E01008C7E010068
:1015D000089B0100E8030020B80300202DE9F04F2C
:1015E000054600688BB00F46924640B1A86830B1FE
:1015F0000378FF2903F0100335D11BB901200BB08C
:10160000BDE8F08F032AF9D04778A149A1480EF030
:10161000E1FC0A2269799F480EF05EFD9E499D48D3
:101620000EF0D8FCAB689B4859780A2201F00F01F4
:101630000EF052FD3F09994996480EF0CBFC0A2264
:10164000394694480EF048FD92480EF0D3FCAB6842
:101650005A7802F00F02BA4207D11A786FF30412D7
:101660001A700020CBE7002BFBD100220DF11808E7
:101670001146404602F0E2FFAB685B7803F00F03CF
:10168000BB4223D0BAF1030F20D0854981480EF028
:10169000A1FC0A2269797F480EF01EFD7E497D4833
:1016A0000EF098FCAB687B4859780A2201F00F01D4
:1016B0000EF012FD794977480EF08CFC0A2239466B
:1016C00074480EF009FD73480EF094FC29680C2F45
:1016D00000F2B780DFE807F0073A9CA9AB9C7B9C3F
:1016E000ADAF8CB1B300AB685B7803F00F03023B86
:1016F000082B24D8DFE803F0052323A5230F232399
:101700001900684A68480DF05CF9AB681C78064619
:1017100004F001042DE0654A63480DF052F9AB680E
:101720001C780646C4F3400423E0614A5E480DF08D
:1017300048F9AB681C780646C4F3800419E05D4A9A
:1017400059480DF03EF90646002412E05A4A564820
:101750000DF037F9AA681378D94303F0010461F357
:1017600000031370064620B90122414608A803F081
:1017700042FB524A29684C480DF023F9504A296827
:10178000814649480DF01DF94E4A2968834646486E
:101790000DF017F90590BBF1000F07D1B9F1000F5B
:1017A00004D14A46414608A803F025FB002E4BD140
:1017B000404603F0C1F8002846D1AB685A7867F379
:1017C00003025A701A7866F304121A7016E73E4A3A
:1017D00035480DF0F6F8A9680B7883F00202C2F3E1
:1017E0004002C3F34004064662F341030B70C0E7B6
:1017F000364A2D480DF0E5F8A9680B7883F004020D
:10180000C2F38002C3F38004064662F38203EDE76D
:10181000284A25480DF0D5F80646002894D1022222
:10182000414608A803F0E7FA8EE7294A6AE7294A01
:1018300068E7294A70E7294A6EE7294A76E7294A84
:1018400074E70024264694E7AB68BAF1030F5A7890
:1018500012D067F303025A701A786FF304121A70E9
:10186000059BCDF80090CDE901B3214698E80C0026
:10187000304608F0ADFDC1E602F00F01B9423FF479
:10188000BDAE67F307125A701A7842F010029CE757
:10189000F47D010070030020A07E0100FE7D0100A8
:1018A000FC7D0100027E010078070020017E01001E
:1018B000087E01000F7E0100147E01004A7E0100B7
:1018C0008C7E01004F7E0100197E01001F7E010009
:1018D000257E01002A7E0100307E0100367E010057
:1018E0003D7E0100437E01002DE9F043614A95B041
:1018F00006468846016860480DF063F85F4A316823
:1019000081465D480DF05DF85D4A316807465A48EA
:101910000DF057F8B9F1000F02D10FB900287CD0B3
:10192000584A316854480DF04CF8574A316805461A
:1019300051480DF046F85549044655480EF04AFB0B
:101940000A22717952480EF0C7FB524950480EF0F6
:1019500041FB0A2241464E480EF0A5FB4C480EF0D2
:1019600049FB5FB33B7C03F00F03042B26D14022DD
:10197000796904A812F071FC47480DF073FBE8B1D7
:10198000464B93F90030CBB92F2104A812F0FCFB91
:1019900028B97B690322402104A808F06BFCB8F148
:1019A000000F43D025B12B7C03F00F03042B37D05D
:1019B0003B4A012304A938480DF0B1FDB9F1000FED
:1019C0002BD099F8103003F00F03042B25D1354BA1
:1019D000D9F814101A6804A800F00CFF04A800F04D
:1019E00047FEB8B1B8F1000F34D025B12B7C03F01D
:1019F0000F03042B25D002AC01220021204602F067
:101A00001DFE01220023CDE9002304A894E806006E
:101A100001F052FB04A800F06FFC15B0BDE8F083A4
:101A20006A691378002BC9D00123C3E724B1237C52
:101A300003F00F03042B02D001231B4ABAE76269AB
:101A4000EFE769690B78002BE4D0002204A802F0CC
:101A5000F3F9DFE724B1237C03F00F03042B02D05A
:101A600002AC0222C9E761690B78002BD2D0424652
:101A7000ECE700BF4A7E0100780700208C7E010061
:101A80004F7E0100147E01000F7E0100577E010091
:101A9000700300207F7E0100E8030020B8030020CF
:101AA000A0940100DC030020B194010070B59AB04D
:101AB000054604AC84E806003A483B490EF08AFA31
:101AC0000A22697937480EF007FB384935480EF08D
:101AD00081FA204603F092FB2968354A35480CF01C
:101AE00070FF0023CDE90133009394E80C004FF020
:101AF000FF3108F06DFC29682F4A2E480CF061FF79
:101B000029682E4A06462B480CF05BFF054658B361
:101B1000037C03F00F03042B26D1416940220AA85D
:101B200012F09BFB2F210AA812F02EFB28B96B693B
:101B3000032240210AA808F09DFB002300931022F5
:101B40004FF4007306A9204603F044FA1C480DF038
:101B500089FA48B11B4B93F900302BB9012306AA2F
:101B60000AA917480DF0DBFCD6B1337C03F00F0354
:101B7000042B15D1144B71691A680AA800F03AFEBB
:101B80000AA800F075FD40B101220023CDE9002331
:101B90000AA894E8060001F08FFA0AA800F0ACFB4E
:101BA0001AB070BD700300205E7E01007F7E0100D0
:101BB000F07D0100780700204A7E01008C7E010044
:101BC000E8030020B8030020DC03002010B50378F0
:101BD0008B42044604D14378402B01D1408810BD8C
:101BE00040232170637008460FF0E8F880B26080EF
:101BF000F5E7000083682DE9F04104460D46002B0F
:101C000000F07B810379072B02D1042940F0758114
:101C1000A44F3B780133DBB22A46FF2120463B70BC
:101C2000FFF7DCFC637922790E3B072BC2F34008F7
:101C300001D9072A32D19C4A21689C480CF0C1FE88
:101C4000064658B3037C03F00F03052B26D12379F6
:101C5000A27961799648FFF7B9FF002280463146A4
:101C600092480CF0A4FE436998451FDA0026032D24
:101C700060D0A3685A7802F00F02013A0B2A59D8B3
:101C8000DFE812F01F00ED0042006A00ED00720074
:101C9000ED009100A200AA00D300E50060790FF0EA
:101CA000BDF9A8EB00035E425E41E0E73146012248
:101CB0007E480CF07CFE4669B045CCBF002601266C
:101CC000D5E7B3F802800EF081FF4FF6FF7381B2C3
:101CD0004FF47A72404608F061FB58B3754A2168A8
:101CE00072480CF06EFE28B12A4603212046FFF709
:101CF00075FC1FE0704A21686C480CF062FE0028F9
:101D0000F2D12A460D21F1E7B3F802800EF05EFF12
:101D10004FF6FF734FF4967281B2404608F03EFBD7
:101D200040B12A4604212046FFF758FC0EF04EFF32
:101D3000A3685880A2681378C3F3C001B14200F0D1
:101D4000438113F0E00F00F09C80C3F3421101398E
:101D500061F347131370CCE0B3F802800EF036FF46
:101D60004FF6FF739622D7E7B3F802800EF02EFFEE
:101D70004FF6FF7381B24FF47A72404608F00EFBC3
:101D80000028D7D04D4A216848480CF01AFE10B1FF
:101D90002A460821AAE74A4A216844480CF011FE65
:101DA0000028F5D1ADE7B3F802800EF00FFF4FF633
:101DB000FF734FF4967281B2404608F0EFFA0028A4
:101DC000B8D02A460921AEE7B3F802800EF0FEFE35
:101DD0004FF6FF739622EEE7B3F802800EF0F6FEA0
:101DE0004FF6FF7381B24FF47A72404608F0D6FA8C
:101DF00000289FD0334A21682C480CF0E2FD10B136
:101E00002A460B2172E7304A216828480CF0D9FD98
:101E10000028F5D12D4A216824480CF0D2FD002875
:101E20007FF46FAF2A46062160E7B3F802800EF018
:101E3000CDFE4FF6FF734FF4967281B2404608F024
:101E4000ADFA00283FF476AF2A460C216BE7B3F8D1
:101E500002800EF0BBFE4FF6FF739622EDE7B3F85B
:101E600002800EF0B3FE4FF6FF7381B24FF416728C
:101E7000404608F093FA00283FF45CAF2A46002160
:101E800034E70EF0A3FEA36858805B7803F00F03DD
:101E9000002E4FD0072B27D8DFE803F046261A265E
:101EA000261A264900030020537E010078070020EF
:101EB0002C030020257E01002A7E0100307E0100D7
:101EC000367E01003D7E0100437E01001F7E010041
:101ED0003E4A21683E480CF074FD80B12A46062136
:101EE0002046FFF77BFB20B1A3681A7866F3C30294
:101EF0001A703B78013BDBB23B70BDE8F081354A9C
:101F0000216833480CF05DFD0028E7D1324A216892
:101F10002F480CF056FD0028E0D1304A21682C48AB
:101F20000CF04FFD0028D9D12A460121D8E72A46D6
:101F30000A21D5E7013B0C2BD6D801A252F823F099
:101F4000751F0000E91E00007B1F00007B1F0000C2
:101F5000E91E0000811F0000E91E0000C31F0000F1
:101F6000C31F0000C31F0000C31F0000C31F0000E9
:101F70007B1F00002A460221B2E72A460521AFE76F
:101F8000124A216812480CF01CFD10B12A460721A4
:101F9000A6E7104A21680E480CF013FD0028F5D181
:101FA0000D4A21680A480CF00CFD0028EED121688A
:101FB0000A4A07480CF005FD01460028E6D12A46EA
:101FC0008EE72A4600218BE70221C1E6197E010037
:101FD00078070020307E0100367E0100017E01007E
:101FE0002DE9F047032986B007466DD00168624AA3
:101FF00062480CF0E6FC3B79BA797979064660488C
:10200000FFF7E4FD05B2002E6CD0337C03F00F0324
:10201000052B67D1314659480CF0BFFC032856D92F
:102020000022314655480CF0C2FC01224469534855
:1020300031460CF0BCFC0222D0F814A04F483146C7
:102040000CF0B5FC43694D484FF00A0803223146B5
:1020500008FB03F90CF0ABFC436908FB03F82146CD
:10206000CDF800804B46524628460EF03AFC044616
:10207000314642480CF091FC052830D1042231460B
:102080003E480CF094FCB0F914A03C484445C4BF51
:10209000444640F2FF3531464C45BCBF4C46002516
:1020A0000CF07BFC022826D10022314633480CF08C
:1020B0007EFC4369AB424FDC012231462F480CF0D5
:1020C00076FC4369AB4254DB06B0BDE8F08705EB14
:1020D000850464004FF000094FF42058C8E74FF022
:1020E000010AD2E705EB850464004FF000094FF4C4
:1020F00020584FF0010ABB68B3F902002A1A002ADF
:10210000B8BF5242524507DC1A785109052907D851
:10211000013161F3471202E01A786FF347121A7027
:102120001B789F2B03D94C4501D04445CCD1A84204
:10213000CAD00022114604AE02A802F07FFA22465D
:1021400002A9304602F0E3FD96E806003846FFF7A4
:10215000ADFCBB685D80B7E70024BB68B3F9023013
:10216000A342B1D021463846FFF7BEFBBB685C8076
:10217000AAE70124F1E700BF537E010078070020A1
:102180002C030020836810B5044643B34B1E032B79
:1021900015D8DFE803F01E0202160379402B0BD09E
:1021A00005D8032B0BD82046FFF724FD07E0422B70
:1021B00002D004D3803BF4E72046FFF711FF002054
:1021C0000FE00379072BFAD10421FFF709FF04215F
:1021D000E9E70379042BF2D1FFF7E6F8EFE74FF0D8
:1021E000FF3010BD002303807047000013B50024AA
:1021F000234600942246214603480DF0A3FE034BDC
:102200001C805C8002B010BDF80200202C0300206E
:1022100010B5044670B3204911F0C3FF58B31F49ED
:10222000204611F0BEFF40B31D49204611F0B9FF12
:1022300028B31C49204611F0B4FF10B31A492046B8
:1022400011F0AFFFF8B11949204611F0AAFFE0B133
:102250001749204611F0A5FFC8B11649204611F0D4
:10226000A0FFB0B11449204611F09BFF002814BF15
:102270000020152010BD0120FCE70220FAE7052010
:10228000F8E70620F6E71320F4E71420F2E70E2023
:10229000F0E70F20EEE700BFB07E0100B97E01003D
:1022A000D47E0100DD7E0100527F01005B7F0100D2
:1022B000257F01002E7F0100647F010070B5054677
:1022C00080B1047864B1084E012404EB84013144E8
:1022D000284611F066FF18B101340E2CF5D1002408
:1022E000204670BD0446FBE7887F0100806910B17D
:1022F00003681B691847704710B50446806910B120
:1023000003685B689847204610BD000008B50322AB
:10231000416804480CF04BFB08B1007D08BDFF206C
:10232000FCE700BF7807002010B503220C46416887
:1023300009480CF03CFB70B1037C13F00D0F0AD17F
:10234000416921F07F41022221F0FF0162F3030382
:1023500021430374416110BD7807002010B50322AA
:102360000C46416808480CF022FB60B1037C03F086
:102370000F03022B01BF24F07F41406921F0FF01D0
:10238000084018BF002010BD7807002010B50322B8
:102390000C46416809480CF00AFB70B1037C13F04D
:1023A0000D0F0AD1022262F30303037424F07F416C
:1023B000436921F0FF011943416110BD78070020F6
:1023C00010B50446806968B103685B69984718B125
:1023D000A06903681B699847A0690368DB68984790
:1023E00008B9012010BD2046FFF790FF20B14FF43F
:1023F00080712046FFF7CAFFE368002BF1D04FF44D
:1024000000712046FFF7C2FFEBE7000010B5032282
:102410000C46416808480CF0CAFA58B1037C13F026
:102420000D0F07D1E143436941F07F4141F0FF01C6
:102430001940416110BD00BF7807002038B50C4637
:102440008168054609B9002038BD0B7C03F00F03F5
:10245000022B03D1002CF6D14869F5E7052BF2D108
:1024600005480CF09AFA8442EDDAE2B2A968024813
:102470000CF09DFA4069E7E77807002038B50D4673
:102480008168044621B9DFED1A7A17EE900A38BD4B
:102490000B7C03F00F03052B15D116480CF07DFAC9
:1024A000854210DAEAB2A16812480CF080FA0028DE
:1024B000E9D0037C03F00F03022B0FD1D0ED057A96
:1024C000F8EEE77AE1E7002DDDD1A268137C03F096
:1024D0000F03022B07D1D2ED057AF1E7032BD2D1FE
:1024E000D0ED057AD1E7032BCDD1D2ED057ACCE73B
:1024F000000000007807002008B5816869B10B7CF6
:1025000003F00F03022B06D0052B06D104480CF074
:1025100044FA00B208BD0120FCE70020FAE700BF42
:102520007807002008B5C16809B9002008BD087CFB
:1025300000F00F039A1E012A00D90BB90009F5E734
:10254000052BF2D1002203480CF031FA0028ECD020
:10255000007CF3E778070020C26810B5BAB1137C9D
:1025600003F00F039C1E012C00D983B95161C3688D
:102570001A7C022161F303021A74C268137C03F00F
:10258000F001602902BF0A2161F30713137410BD23
:10259000C26810B5BAB1137C03F00F039C1E012C66
:1025A00000D983B95161C3681A7C032161F3030226
:1025B0001A74C268137C03F0F001602902BF07217E
:1025C00061F30713137410BDC36853B11A7C02F092
:1025D0000F02901E012800D91AB91A7C61F3071264
:1025E0001A74704708B5016909B9002008BD0B7C51
:1025F00003F00F03022B01D14869F7E7052BF4D153
:10260000002203480CF0D3F90028EED04069EDE732
:10261000780700202DE9F041036904460F46A3B96D
:1026200041681248114E0CF0B8F90546042D0CDC37
:102630003046D4F804800CF0F6F941460246206199
:1026400030460CF0CDF90135F0E7226962B1137C18
:1026500013F00F0106D1022161F303031374236900
:102660005F6101E00229FAD0BDE8F081780700201F
:10267000406828B1007C00F00F00431F58425841C9
:1026800070470000F8B50446FFF7F2FF002832D08B
:1026900061683748364F0CF080F90546032D6668AF
:1026A00009DC38460CF0BFF93146024638460CF0DA
:1026B00097F90135F2E7002231462D480CF077F901
:1026C00002F054FC01222075616829480CF06FF972
:1026D0000222A060616826480CF069F90422E060DB
:1026E000616823480CF063F92061207D0C282CD010
:1026F00002D803280ED0F8BD102830D01228FAD105
:102700000C200EF0F9FA1B4B44600360054606F0FE
:10271000E5FC18E010200EF0EFFA174B03600546B9
:10272000446000212046FFF789FE03B2002BB6BFAC
:1027300040422B8128816868FFF7DEFE0F4B2B603B
:1027400000236881AB81A561D5E714200EF0D4FA8F
:102750000B4B44600360054606F014F9F3E70EF0F6
:10276000CBFA084B44600360054606F0F9FEEAE741
:102770007807002034950100247D01009095010028
:10278000509401003096010010B500230446C0E9C2
:10279000002183610377C362FFF774FF204610BDF9
:1027A00070B5056806462F21284611F077FD0446CE
:1027B00098B1002300F8013BFFF780FD0B49054667
:1027C0000B480DF007FC0A22294609480DF06BFC66
:1027D00007480DF00FFC284670BD2846FFF76EFD38
:1027E00005460028F7D03460F5E700BF917E010070
:1027F000700300202DE9F043054689B0002400F164
:102800001C082A601646CDF8048084610477C462EF
:102810000F462346002939D0002A37D02F213846C9
:1028200011F0B2FC814650B3234602AAF85C19B2FB
:1028300038B12F2805D0142B02D0D0540133F5E73E
:10284000194608AB1944002301F8183C10483146DA
:102850000CF0B7F80F22686009F10101404611F051
:10286000FCFC01A8FFF79CFF019BE86203B92B77F2
:102870002846FFF707FF284609B0BDE8F0833A462F
:10288000314603480CF09DF86860F1E76B60EFE7B4
:102890007807002008B583693BB9007D052809D079
:1028A00014280CBF0020FF2008BD1A681846926B40
:1028B0009047F3E75020F7E708B50522416805483F
:1028C0000CF075F820B1037C13F0F00018BF180964
:1028D00008BD00BF780700202DE9F7436D4685E865
:1028E0000600416881461F4619B9002003B0BDE8C3
:1028F000F0833448DFF8CC800CF04FF80446052C08
:10290000D9F8046009DC40460CF08DF831460246E7
:1029100040460CF065F80134F1E7052231462948BC
:102920000CF045F804460028DFD0284602F0B4F940
:102930000F28DAD8284602F04BF8002807DD237C60
:1029400013F00D0F10D003F00F03072B0CD0237CD6
:102950001D491E486FF3071323740DF03BFB1B4802
:102960000DF048FB0120C1E70EF030F9064628467D
:1029700002F02EF8002F237C0CBF0222072262F304
:102980000303304460612374284602F085F9237CF8
:102990000F4960F3071323740C480DF01BFB284606
:1029A00002F016F80A22014608480DF05AFB0949C0
:1029B00006480DF00FFB0A22616904480DF051FB37
:1029C000CDE700BF78070020ED7F010070030020F5
:1029D000F77F010002800100F0B587B06F4687E8FD
:1029E0000600054697E8030002AC84E80500384677
:1029F0001E4602F051F901380C2838D8DFE800F003
:102A0000424B959E8C0739373754627E70004EBB1F
:102A10000722214604A802F0EEF9494949480DF081
:102A2000D9FA204602F038F90A22014645480DF04D
:102A300053FB454943480DF0CDFA204601F0C8FF4D
:102A40000A2201463F480DF00CFB3E480DF0D2FA39
:102A50009DF8303094E806002846FFF73DFF01203E
:102A600007B0F0BD2846FFF727FF0028D0D100208F
:102A7000F6E70EB10622CCE72846FFF71DFF002837
:102A8000F8D1F4E70EB90222C3E72846FFF714FF96
:102A90000028F8D1EBE70EB10122BAE72846FFF78C
:102AA0000BFF0028F8D1E2E74FF480312846FFF70A
:102AB00055FC08B10B22ACE72846FFF7FDFE0028C5
:102AC000F8D1D4E74FF480312846FFF747FC08B926
:102AD0000A229EE72846FFF7EFFE0028F8D1C6E756
:102AE0004FF400312846FFF739FC08B90C2290E773
:102AF0002846FFF7E1FE0028F8D1B8E74FF400318F
:102B00002846FFF72BFC08B10D2282E72846FFF785
:102B1000D3FE0028F8D1AAE70EB1032279E72846B0
:102B2000FFF7CAFE0028F8D1A1E70EB9052270E729
:102B30002846FFF7C1FE0028F8D198E7042268E78D
:102B40001C800100700300203080010018B103498F
:102B500003480DF03FBA0349FAE700BF9D7E01002C
:102B600070030020A27E01002DE9F0439FB04FF0DA
:102B7000000802AC84E806000646102241460AA876
:102B80001D46269FCDF8248010F093FB2046CDE90A
:102B900006888DF8208002F031FBEA051AD5204620
:102BA00002F07AF8172800F2CE80012303FA00F031
:102BB000974B18420AD1974B0340002B40F0C78037
:102BC00010F0240F00F0BF80934900E0934906A85D
:102BD00011F0F1FA92480CF045FA002800F0AB80B1
:102BE000904B93F900209846002A40F0A480002FD3
:102BF00044D13B46032240210EA807F03BFB7368FB
:102C00003F2219680EA811F002FBAB0540F1AE801F
:102C1000204602F041F8022800F0A880204602F089
:102C20003BF8052800F0A280204602F037F8012882
:102C300040F090804FF001094FF40073142209A96D
:102C4000CDF80090204602F0C5F94B4609AA0EA91E
:102C500073480CF064FC744974480DF0BBF90EA97C
:102C600072480DF0C0F9724970480DF0B3F909A926
:102C70006E480DF0B8F96D480DF0BCF9204601F032
:102C80006CFE05F4005908B1A90503D4B9F1000F91
:102C900000F09D800023032240210EA807F0EAFAED
:102CA00073683F2219680EA811F0B1FA47B1614963
:102CB0000EA811F05AFA3F2239460EA811F0A7FAD1
:102CC0005C490EA811F051FA3F22B9F1000F67D00C
:102CD00059490EA811F09BFA204601F0DFFF043895
:102CE00001285FD81722214604A802F084F80023A7
:102CF00000934FF44073142209A9204602F06AF9A8
:102D000049494A480DF066F90EA948480DF06BF99B
:102D1000474946480DF05EF909A944480DF063F9AA
:102D200042480DF067F93E480CF09CF918B198F94B
:102D30000030002B40D030462946FFF727FB00200B
:102D40001FB0BDE8F0833D4938480DF043F925F444
:102D500080753FE7204601F0A1FF02283FF46AAFEB
:102D6000204601F09BFF08283FF464AFE80585D5B5
:102D70009DF81830002B81D0012306AA0EA92848FF
:102D80000CF0CDFB284929480DF024F90EA927485D
:102D90000DF029F9264925480DF01CF906A967E729
:102DA000274996E70023B9F1000F00930CBF4FF4B9
:102DB00000734FF440739EE70EA9012309AA184837
:102DC0000CF0ADFB4FF400713046FFF71FFBEA0536
:102DD00040F18480204601F05FFF0138142835D887
:102DE000DFE810F0D9003400340034003400D9009A
:102DF0003400340034003400340034003400DD008A
:102E0000D7003400340034003000D300D50000BFB8
:102E100042C0380001008000B97E0100B07E010090
:102E2000E8030020B8030020168001007003002092
:102E3000FE7D01001B8B01009C7F010008800100CA
:102E4000927F01005C4906A811F0B5F90023032226
:102E500040210EA807F00EFA73683F2219680EA8E9
:102E600011F0D5F947B155490EA811F07EF93F226E
:102E700039460EA811F0CBF950490EA811F075F99A
:102E80003F224F490EA811F0C2F94E494E480DF0AD
:102E9000A1F80EA94C480DF0A6F84C494A480DF08F
:102EA00099F806A948480DF09EF847480DF0A2F899
:102EB00047480CF0D7F800283FF43DAF98F90030B0
:102EC000002B7FF438AF0EA9012306AA40480CF06E
:102ED00026FB4FF480713046FFF798FA6B0552D508
:102EE0004FF480313046FFF739FA002859D039497C
:102EF00006A811F060F90023032240210EA807F074
:102F0000B9F973683F2219680EA811F080F947B12A
:102F10002A490EA811F029F93F2239460EA811F0CE
:102F200076F926490EA811F020F93F222A490EA869
:102F300011F06DF9234924480DF04CF80EA92248F0
:102F40000DF051F8214920480DF044F806A91E481B
:102F50000DF049F81C480DF04DF81D480CF082F8B2
:102F600000283FF4E8AE98F90030002B7FF4E3AE80
:102F70000EA9012306AA16480CF0D1FA4FF480617D
:102F80003046FFF743FA0120DAE614495BE71449BB
:102F900059E7144957E7337D052B7FF457AF1249A2
:102FA00051E74FF400313046FFF7D8F908B10F4927
:102FB0009EE70F499CE700BF527F01001B8B010079
:102FC0008D7F01001680010070030020FE7D01004E
:102FD000E80300200A7F0100B57F01005B7F01004C
:102FE000647F01002E7F0100257F01001C7F01000E
:102FF000017F0100F0B5CB070C4644BF21F480549B
:1030000024F0010414F4805785B005460CD004F474
:10301000E0612846FFF7BAF9144915480CF0DAFFC9
:103020004FF0FF3005B0F0BD07F0AAF89528EED9B3
:1030300002F064FF0028EAD002AE3A463946304634
:1030400001F0FCFA4FF440722946304601F0E8FEE8
:103050004FF4E0612846FFF781F9009744EA000346
:1030600096E806002846FFF77FFDDBE7CE7F0100EC
:103070007003002010B54FF440710446FFF76EF95D
:10308000014670B1074B93F90030062B09D1204659
:10309000FFF7B0FF20464FF44071BDE81040FFF746
:1030A000B5B910BDE003002083691BB11A6818464A
:1030B000926B1047007D70472DE9F04F93B00AAE38
:1030C00009939DF8703003939DF87430049305467E
:1030D00086E8060007F054F8B0F5966F04460EDA5D
:1030E000AF49B0480CF076FF0A222146AD480CF0FB
:1030F000DAFFAC480CF07EFF4FF0FF39A9E30DF08A
:1031000065FD0790304601F07DFE0290074602F013
:10311000F5FE099B06901BB11A78002A40F01B8629
:103120002B7F13B105F11C030993002F40F02B8670
:10313000099B002B40F01186EB6A0293002B00F0F4
:103140002286304601F05EFE002840F01C869DF885
:103150000820314610A801F059FE00F014BE6B683B
:10316000002BC9D0029B042B07D1049B96E80600D4
:103170002846FFF7B1FB81466BE396E803000CABF2
:1031800083E80300304601F087FD092800F222821F
:10319000DFE810F00A002002200220026D01200268
:1031A00020022002AF01AF0100220DF138091146C3
:1031B000484601F043FA304601F0CFFB07460028AD
:1031C00000F04F81029B0C2B1AD8DFE813F00D00A2
:1031D00019006900190019001900190019001900D7
:1031E0001900170103013301DDF82480B8F1000F45
:1031F0000AD06D496D480CF0EDFE6C480CF0FAFEFB
:103200000024A2462746F6E0284601F00FF80028E1
:10321000D4BF002101210A22044664480CF043FF78
:10322000634962480CF0DFFE304601F0D1FB0A2210
:1032300001465E480CF015FF5C480CF0DBFE002CEC
:10324000304640F37F8501F0C3FB70BB022231465C
:1032500010A801F0D0FD40F201144FF0010806E083
:103260000122314610A801F0C6FD40F201144FF4CE
:1032700000722946484602F017FB484601F00EFD51
:10328000042814D1304601F009FD022814D130463B
:1032900001F004FD0EA9024610A801F002FD0BE0AA
:1032A000002427464FF0FF38E1E74446D5E748467B
:1032B00001F0F4FC0528E5D02B7D072B08D1304622
:1032C00001F052FB20B102220EA910A801F0E9FC86
:1032D0002846FFF7E9FE00B200900DF1380A0DF123
:1032E000280910A899E80C00514602F001F8504650
:1032F00001F084FF3FB1484601F0D0FC022859D1CB
:10330000504602F0FDFA9AE8030089E8030044F40D
:1033100090544FF0000A4FF0FF392B7D072B40F0FF
:103320005082039B73B3AB681B7C03F00F03052B28
:1033300040F05981069B002B00F05281284600F096
:1033400075FF049B00930028099BA9680AAA2846D8
:10335000D4BF4FF000094FF0010900F0E7FE029BD7
:10336000012B4FFA89F840F03E810AA801F0F5FAE6
:10337000039038B1049B00930CAA4B4606CA28461A
:10338000FFF72AFB0AA801F087FC0338042800F2A3
:103390005081DFE810F02A014E01ED017201510168
:1033A0003B8001008C0300207B8001007003002023
:1033B000A07E0100484601F071FC0128A0D04846DB
:1033C00001F06CFC0A289BD0484601F067FC0B28F2
:1033D00099D195E729464FF40072484602F064FA05
:1033E000304601F013FAC1B2484601F0B7F998B976
:1033F000BA4600273C464FF0FF388CE729464FF489
:103400000072484602F050FA304601F0F8F90146E1
:10341000484601F089F9EAE799E80300022286E8C4
:1034200003000027314610A801F0F0FC4FF490543F
:10343000BA46E0E74FF400722946484602F034FAF3
:10344000304601F0C2F90146484601F098F999E882
:1034500003004FF0000A86E803004FF490545746EB
:10346000C9E7824604464FF0FF39C84655E7029B3C
:10347000092B20D0284600F0D9FE00280DDD0222BD
:10348000314610A8012701F0B6FC40F201144FF0BC
:10349000FF394FF0000AB8463FE70122314610A835
:1034A0004FF0000A01F0A7FC40F201144FF0FF3981
:1034B0000127D04631E74FF480312846FEF74EFF12
:1034C00007464FF4803128465FB1FEF79FFF40F278
:1034D00001444FF001094FF0000A57464FF0FF3802
:1034E0001BE7FEF753FF40F201444FF00109BA46D3
:1034F000F3E796E803000DF1380888E8030030464A
:1035000001F02BFAE0B90524304601F0C5FB4FF479
:10351000007209282946304608BF644202F0C4F907
:103520000022314610A801F066FC029B0B2B49D803
:10353000DFE803F021480D484848484848482343FD
:10354000304601F01DFA04460028DCD0DCE70027F5
:103550002846FFF79FF921460246304601F058F908
:10356000044690BB98E8030086E803004FF0010A88
:103570004FF0FF39B2E70127EAE72146304601F074
:10358000A3F950B10222314610A84FF0000A01F011
:103590003DFC4FF490545746EAE798E8030086E86C
:1035A0000300AE49AE480CF015FDAD480CF022FD0D
:1035B00000244FF0010A2746DAE72146304601F0A1
:1035C000A8F9DEE70024A246F5E74FF490544FF047
:1035D000000ACDE700244FF0FF39A246274644E712
:1035E000069B0393CEE60023FBE72846FEF78EFEFC
:1035F0000528804602D04FF003092AE199499A48EC
:103600000CF0E8FC0A22414697480CF04CFD964825
:103610000CF0F0FC4FF4007229460AA802F044F9BD
:1036200001220AA910A801F0E6FB44F4807444F0DA
:1036300001044FF0000B47E02846FEF767FE06281E
:1036400080460DD1894988480CF0C4FC0A224146C5
:1036500085480CF028FD84480CF0CCFC0222E0E701
:10366000834981480CF0B6FC0A2241467E480CF0A2
:103670001AFD7D480CF0BEFCBDE74FF480312846B2
:10368000FEF76CFE002871D1B8F1FF3F08D1284643
:1036900000F0CCFD0028D4BF4FF000084FF0010827
:1036A000B8F1000F5DD14FF4007229460AA802F06C
:1036B000FBF801220AA910A801F09DFB44F48074D4
:1036C00044F001044FF0060B0AA801F03AF9002873
:1036D0006BD10AA844F0010401F03FF9002867D03B
:1036E00044F40074039B13B124F40074A4B2224682
:1036F00029460AA801F0E9FB4FF00109BAF1000FD1
:1037000040F07183A869002840F0E4814FF4003153
:103710002846FEF723FE002800F0E5815549504871
:103720000CF058FC4E480CF065FC630500F1FD827E
:1037300051494D480CF04EFC0A2249464A480CF0CB
:10374000B2FC4E4948480CF045FC0DF03FFA079B8F
:103750000A22C11A44480CF0B2FC43480CF04AFC5F
:1037600077E0474940480CF035FC44E74549F9E724
:10377000B8F1FF3F08D1284600F058FD0028D4BF1B
:103780004FF000084FF00108B8F1000F0BD00222F3
:103790000AA910A844F4807401F02DFB44F0010440
:1037A0004FF0050B90E73849DCE744F4807490E76C
:1037B0004FF4007229460AA801F032FB00288FD18D
:1037C00090E7B8F1FF3F08D1284600F02FFD002810
:1037D000D4BF4FF000084FF00108B8F1000F2B499B
:1037E000214818BF01270CF0F5FB0A2241461E486C
:1037F0000CF059FC26491C480CF0ECFB0A22394617
:1038000019480CF050FC18480CF0F4FB09980028FB
:1038100044D0FEF7FDFC08902846FEF777FD0FFA2E
:1038200080FB089BBBF1000F01D10FFA88FB002B36
:103830005BD09B4530D017490B480CF0CBFB0A22DC
:10384000594609480CF02FFC07480CF0D3FB6FF0E9
:103850000209484613B0BDE8F08F00BF9080010018
:103860008C0300209C80010070030020B1800100C7
:10387000C88001007C810100EF810100FA81010014
:10388000E680010000810100158101003281010004
:10389000408101004781010000230993029B012B15
:1038A00030D1039B1BB10AA801F057F803900AA876
:1038B00001F0F2F9152800F2F880DFE810F0B70007
:1038C000CA00A7002600B700970074005000B70098
:1038D000B700F300F30004010401E100E100F60089
:1038E000F600F600E100E100E100A8690028D5D06B
:1038F000049A0368CDE900720AAA9C6A099B06CA69
:10390000A04738E400230393D1E72846FEF7FEFCE6
:10391000052807467FF46FAE8D498E480CF05AFBA0
:103920000A2239468B480CF0BEFB8A480CF062FB39
:103930004FF4007229460AA801F0B6FF2B7D052B33
:103940000CBF0E2201220AA910A801F054FA44F477
:10395000807444F001044FF0000B012768E0284612
:10396000FEF7D4FC0628074616D17B4979480CF0AF
:1039700031FB39460A2277480CF095FB75480CF06C
:1039800039FB0AA910A8022201F035FA4FF40021F0
:103990002846FEF73BFDDAE770496E480CF01AFB4B
:1039A0000A22394662E64FF480312846FEF7D6FCFB
:1039B00000287FF4DBAEB8F1000F7FF4D2AE4FF4F5
:1039C000007229460AA801F06FFF01220AA910A877
:1039D00001F011FA44F480744FF400212846FEF7F8
:1039E000D5FC44F001044FF0060BB6E7B8F1000F28
:1039F0003FF4D9AE02220AA910A844F4807401F061
:103A0000FAF944F001044FF0050BA6E70AA800F00C
:103A100098FF074600285BD02846FEF777FC05286C
:103A20003FF4E9AD44F4807444F001044FF0000B1E
:103A3000039B002B3FF462AE049B00930CAA08F09A
:103A4000010306CA284624F40074FEF7C5FFA4B299
:103A500054E60AA800F075FF00283FF47CAFB8F1E7
:103A6000000F0DD03E493B480CF0B4FA2846012126
:103A7000FEF75AFC4FF488512846FFF7BBFABAE527
:103A80000AA800F05EFF074610B30AA800F065FF21
:103A900028B94FF4007229460AA801F005FF44F442
:103AA0004074C1E744F4806455E70AA800F044FF7D
:103AB00008B144F480740AA800F04FFF074638B1FB
:103AC00044F40074B2E74FF0000B4FF4806444E715
:103AD000BB4642E703680AAA1B6B06CA9847002840
:103AE0007FF414AE1AE6D5F81880B8F1000F39D07B
:103AF0000AAE24B122462946304601F0E6F9049A7E
:103B0000A8690368CDE900729F6A099B96E80600E0
:103B1000B8478146A86903689B6B9847052808BF8A
:103B200044F0010414F4806F18BF4FF00109BBF199
:103B3000000F03D059462846FEF7F6FB069B002BE4
:103B40003FF4F6AD21462846FFF754FAF0E500BFF2
:103B50009C80010070030020B1800100C88001003A
:103B6000638101002B7D052B75D0062BDFD10AA8C0
:103B700000F0E2FE00286ED041462846FEF75EFCCB
:103B8000074606B20AA801F087F8049B8046002B7E
:103B900047D024B1224629460AA801F096F9002E02
:103BA000C5D0BCBF7E4236B206F1FF339BB2B4BF74
:103BB00001270027192BBAD8012130460DF0F4F95E
:103BC000B8F1150F09D8012303FA08F8874B18EA52
:103BD000030F35D118F0A40F3AD1854985480CF070
:103BE000F9F90A22314683480CF05DFA824981488E
:103BF0000CF0F0F90A2205997E480CF054FA7D4841
:103C00000CF0F8F9304606F0EDFD28B12846FEF735
:103C100053FE08B902F044FF44F4807444F00104F8
:103C20007DE0304606F0DEFD0028B2D073497448CE
:103C30000CF0D0F972480CF0DDF96FF0040908E6D9
:103C400087F001030593194630460DF0D5F9C4E716
:103C500005973946F8E724B1224629460AA801F01B
:103C600034F9029B022B5DD0032B09D0012B7FF48A
:103C70005EAF44F4807444F00104DDF8089056E728
:103C80002846FEF7AFFC030C074611D15D495E489C
:103C90000CF0A0F96B685C4819680CF0A4F95A485C
:103CA0000CF0A8F96B6859491A6859480BF022FCC6
:103CB000304600F0ADFE0EF0B5FC0022554B0EF084
:103CC00009FD0EF0B7FF0FFA80F8082006F06EFD30
:103CD00068F30F07064660F31F474F4945480CF04D
:103CE00079F96B68434819680CF07DF94B494148F4
:103CF0000CF070F90A2241463E480CF0D4F94849CC
:103D00003C480CF067F9B1B20A223A480CF0CBF902
:103D100038480CF06FF939462846FEF77BFC4FF027
:103D2000010904E744F4007478E7069B002B3FF494
:103D3000FFAC29464FF480620AA801F0C6F84FF4A0
:103D4000806100E700F044FE00287FF489AA044661
:103D50008046FFF78CBA029AAAB91B78002B3FF471
:103D6000EBA909A8FEF71CFD0290304601F04AF8C5
:103D700028B99DF80820314610A801F047F8029BA9
:103D8000002B3FF4D9A927491A480CF023F90A223D
:103D9000214618480CF087F9234916480CF01AF907
:103DA0006B68144819680CF01EF9204911480CF092
:103DB00011F909990F480CF016F91D490D480CF03E
:103DC00009F9304601F01AFA099B002B3FF4C7A904
:103DD0001B78242B7FF4C3A9164906480CF0FAF887
:103DE00004480CF007F96FF0030932E542C03000D7
:103DF000BB810100700300207F7E0100AE810100C5
:103E00008C030020C0810100BC030020D081010090
:103E1000E803002000005940DF810100E681010035
:103E2000EA8101004F8001005A8001006180010099
:103E3000A07E0100678001002DE9F04F8FB0804621
:103E4000CDE90221002900F0688106F099F9B0F56A
:103E5000966F044610DAB249B2480CF0BBF80A2259
:103E60002146B0480CF01FF9AE480CF0C3F84FF0F3
:103E7000FF300FB0BDE8F08F029B0BB11B782BB960
:103E800098F81C3013B108F11C030293029BE3B9AC
:103E9000D8F82C6016BB4021039810F075F9002863
:103EA00039D00446002304F8013B0398214606F06C
:103EB00097FC039481460024039D2F5D6FB3384621
:103EC00011F0BFF928550134F6E71B78002BDFD03D
:103ED00002A8FEF765FC06460028D9D00D2EDAD1DF
:103EE00008AC00221146204600F0A8FB039A2146A8
:103EF0000AA800F074FF324621460AA800F086FFA7
:103F00000023019301230093029B94E8060040469E
:103F1000FFF7D2F8ADE78146CDE7284600F040FB39
:103F200004ACC2B205463946204600F087FB052E98
:103F300024D0062E08BF17255FFA86FA0AAF52462C
:103F40002146384600F062FF092D19DC082D80F269
:103F5000D480AA1C03DB6B1C40F3DF80D5B103A81F
:103F600006F065F8024618B12146384600F0B7FE63
:103F700001230093CDF804900023C6E71825DBE762
:103F8000172D00F08980182DE9D1002221463846EE
:103F900000F031FF06AD03A9284606F069F8524645
:103FA0002946384600F032FF284600F077FE10F12F
:103FB000000A18BF4FF0010A4FF0000B039A0FFAE6
:103FC0008BF35AB1BBF1030F07D003A806F02FF80B
:103FD00047F82B000BF1010BF0E75B460B2E0DD0E1
:103FE0000C2E13D00A2E19D1284600F0F1FC81B214
:103FF000204600F099FBCDF8049083E7284600F0B6
:10400000E7FCC1B2204600F0A9FBF4E7284600F027
:10401000DFFC0146204600F0B2FBECE753449BB2C4
:10402000013B032B30D8DFE803F00207122095E8AC
:10403000030084E80300DEE7284600F0C9FC9DF891
:10404000283082B2214608A800F092FED3E7284625
:1040500000F0BEFC9DF82C2000929DF8283082B222
:10406000214608A800F06DFEC5E7284600F0B0FC28
:104070009DF82C200092214682B29DF8283008A895
:1040800000F05FFE0C99C5E7274926480BF0A2FF18
:1040900024480BF0AFFFAEE700222146384600F07F
:1040A000AAFE0025039A2BB242B1042D0AD003A820
:1040B00005F0BDFF47F825000135F3E7032B10D0CD
:1040C000042B98D19DF8341001919DF83010009187
:1040D0009DF82C309DF82820214608A800F06CFEA1
:1040E00089E79DF8301000919DF82C309DF828202C
:1040F000214608A800F050FE7DE708AC03A9204641
:1041000005F0B6FFEAB22146384600F074FE52468A
:104110002146384600F07AFE6DE70020A9E600BF90
:10412000018201008C030020198201002DE9F04F6B
:104130008FB0814616469A469DF860B000296DD032
:104140000B7C03F00F03052B68D1354DCC682B7821
:10415000DFF8D48001332B70002C5CD0237C03F07B
:104160000F03042B55D16269D9F8001040460AF0BC
:1041700028FC074600284CD0037C03F00F03052BD6
:1041800047D1284B01461A6802A8FEF7FDFA6EB126
:1041900002A8FEF76DFA48B100230093CDF804B0F1
:1041A00053463168726802A8FEF786FF002239463E
:1041B00040460AF0FCFB00B3037C03F00F03022B24
:1041C0001BD14369072B18D10122394640460AF01A
:1041D000EEFBCDF800B00146534632464846FFF7A5
:1041E000A5FF9EB990B12B7802A8013B2B70FEF77A
:1041F00083F801200FB0BDE8F08F3EB902A8FEF7AA
:1042000037FA18B102A800F011F8EBE702A8FEF7A0
:1042100073F86468A0E72B78013B2B700020E9E776
:104220006D030020DC030020780700207FB500220A
:104230000546114602A800F001FA6B684748196864
:104240000BF0D1FE464945480BF0C4FE2846FEF768
:104250000FFA58B9434941480BF0BCFE3F480BF0F8
:10426000C9FE4FF0FF34204604B070BD2846FEF76B
:104270004DF80646A86958B10368DB6A984704B24E
:10428000002C05DB14BF01200020FEF75FFCEAE7ED
:104290002B7D072B13D0701C152810D80126324C0B
:1042A00006FA00F0044004D110F0490F07D0204670
:1042B000EBE72E4929480BF08DFE3446D3E74FF447
:1042C0000072294602A800F0ABFD2B7D033B062BB4
:1042D0003DD8DFE803F038233C3C04382300AB68CA
:1042E0001B7C03F00F03052B4FF000041BD120496A
:1042F0001A480BF06FFE234622460094A968284610
:10430000FFF714FF1B49044614480BF063FE2046D8
:10431000FEF71CFC11480BF06DFEA4E7002102A87B
:1043200000F04EFC044614490C480BF053FE2146A5
:104330000A220A480BF0B7FE08480BF05BFE003477
:1043400018BF01248FE702A800F042FBEAE70B49FF
:1043500002480BF03FFE002485E700BF70030020F9
:10436000A07E01004E820100848030009D7E01000D
:104370005A86010057820100648201005A820100BE
:10438000F0B54FF4006185B00546FDF7E7FF002862
:1043900047D0002202AC1146204600F04FF94FF4FE
:1043A00040722946204600F03BFDAB69002B38D017
:1043B0004FF400612846FEF729F81B491B480BF013
:1043C00009FEA869002301260268CDE90063976A07
:1043D00094E80600B847431C044622D06B68134893
:1043E00019687CB90BF0FFFD114910480BF0F2FD84
:1043F00010490E480BF0EEFD0C480BF0FBFD20467B
:1044000005B0F0BD0BF0EFFD094908480BF0E2FDE7
:10441000094906480BF0DEFD04480BF0EBFD34467D
:10442000EDE70224EBE700BFDF7F0100700300200F
:1044300006800100728C0100558501002DE9F04FC6
:10444000044689B08946FFF79BFF0522616847480B
:104450000AF0ADFA0646002872D0037C03934FEAB7
:10446000131A45690CF0B2FBBAF1000F68D0A5EB46
:10447000000804AD52460B21284606AF00F0DEF8D6
:1044800042462946384600F02AFCB9F1040F17D1FC
:104490000023009395E806004FF400532046FEF7F2
:1044A00063FB0A224FF47A71314898FBF1F10BF06B
:1044B000D8FD30492E480BF08DFD2D480BF09AFDAC
:1044C000B8F1000F3CDA2C4B984539DB05F058FE6B
:1044D0004FF00008CDF8008083464FF4005395E874
:1044E00006002046FEF740FBBBF5966F10DA234925
:1044F00023480BF06FFD0A22594621480BF0D3FDEB
:104500001F480BF077FD4FF0FF3009B0BDE8F08F8A
:10451000337C68F30713337452464146384600F043
:104520008DF8039B03F00F03DA1F534253410193AD
:104530000123009397E8060043462046FEF7BCFDA2
:10454000B9F1010F02D12046FEF794FDA06908B928
:104550000020DAE703685B6998470028F8D0A06973
:1045600003680FFA89F19B689847CEE77807002027
:1045700070030020268201000200008035820100C5
:104580008C03002007B5002300931A461946034800
:104590000BF0D8FC03B05DF804FB00BF3003002033
:1045A000F8B50646F0B10378E3B12D2B1ED0A3F188
:1045B0003002092A1AD9252B1AD07B2B1AD0232B8B
:1045C0001BD00F4F012404EBC4053D4428460FF0D7
:1045D00016FE2946024630460FF02DFE20B101346A
:1045E000192CF0D14FF0FF342046F8BD0024FBE732
:1045F0000824F9E76FF00104F6E71724F4E700BF99
:1046000086820100F8B5064690B1037883B10A4F5F
:10461000002404EBC4053D4428460FF0F0FD294674
:10462000024630460FF007FE20B10134172CF0D1BE
:104630004FF0FF342046F8BD6783010010B500231A
:104640008370C370037143718371C37161F3071386
:104650004370027010BD10B50023072403708370EF
:10466000C37064F307134370416010BD93B2112B04
:1046700070B516469CBF134AD25C4B7888BF0022A7
:1046800062F307134B7005460C460F480F490BF0B9
:10469000A1FC0A2231460C480BF005FD0C490A48E2
:1046A0000BF098FC617808480A2209090BF014FD08
:1046B00005480BF09FFC23682B6063686B602846FD
:1046C00070BD00BF6F82010070030020AC84010048
:1046D000B78401004B781B09013B082B1AD8DFE88F
:1046E00003F0160E0E19191919050C000C4B4B602E
:1046F0000B6803604B68436070470A4BF7E764231D
:104700008B71CB7923F00103CB7100234B71FF2315
:104710000B71EDE700230B714B718B71CB71E7E7E8
:104720000000A0410000964243781A0903D0022AF3
:1047300005D000207047022262F30713437040F255
:104740006D139942A8BF1946C379817123F0010303
:10475000C1F300211943C1710120704743781A0940
:1047600003D0022A05D000207047022262F307130B
:1047700043706429A8BF642141710120704713B5BB
:104780000446084631B9E37960F34703E371012039
:1047900002B010BD642300934FF4FA7200239921F4
:1047A0000CF09FF863781A0908D0032A0BD820EA86
:1047B000E0706428A8BF64200130E4E7022262F3BD
:1047C00007136370F3E70020E2E707B5C27912F040
:1047D000FE0F11D043781B09013B022B0CD8500867
:1047E0004FF4FA73009364229923002101380CF0EE
:1047F00078F803B05DF804FB4FF0FF30F9E7C379B8
:10480000827903F0010342EA032070474079704740
:1048100043781B09013B10B50A2B53D8DFE803F09E
:104820000606525252482F2F2F101000027964238F
:1048300091FBF3F1114481F308010171012010BDD6
:10484000632944684FF064030FDC03FB04112AB1B1
:1048500053439942A8BF194621EAE1714378416068
:10486000062262F307134370E8E791FBF3F121445A
:10487000E2B19142A8BF114621EAE17116E0436816
:1048800007EE903AFDEEE77A642417EE903A91FB3A
:10489000F4F1194422B19142A8BF114621EAE17115
:1048A00007EE901AF8EEE77A17EE901A4160C5E726
:1048B00043681944002AF9D0642353439942A8BF9E
:1048C0001946D9E70020BAE743781B09022B1ED10D
:1048D000C279837902F0010243EA0223642291FB48
:1048E000F2F11944B1F5B77F0FDA40F26D1331EAF6
:1048F000210128BF1946C379817123F00103C1F357
:1049000000211943C171012070470021F3E7002005
:10491000704743781B09022B0CD14379642291FB29
:10492000F2F1194421EAE1719142A8BF11464171A7
:1049300001207047002070470078003018BF012028
:104940007047437803F00F03012B04D80078003040
:1049500018BF0120704700207047437813F0F00F14
:1049600014BF012000207047407800F0E0002028AC
:1049700004D0A0F1400358425841704701207047CD
:1049800043781B09013B0A2B1ED8DFE803F00A0A13
:104990001D06061B0F0F0F060600436864205843D0
:1049A00070470079642310FB03F0704743689FED64
:1049B000077A07EE903A67EE877AFDEEE77A17EE10
:1049C000900A704740687047002070470000C84256
:1049D00043781B09013B0A2B18D8DFE803F00808CD
:1049E000170606120A0A0A06060040687047007990
:1049F0007047406807EE900AFDEEE77A17EE900ADE
:104A000070474068642390FBF3F0704700207047C4
:104A100043781B09013B0A2B1ED8DFE803F0131370
:104A20001D06060E191919060600436807EE903A8E
:104A3000F8EEE77A17EE900A70474368642293FB1A
:104A4000F2F3F3E7037907EE903AF8EE677AF1E7CD
:104A5000436807EE903AEDE7DFED017AEAE700BF41
:104A60000000000043781B0907B50B2B60D8DFE876
:104A700003F06216165F5F5F44245F5F06064068BE
:104A800049B1D0F1640056D46428A8BF642000B2B4
:104A900003B05DF804FB0028F6DA0846F8E7007971
:104AA00031B1002100916423FF220BF01AFFEEE7E1
:104AB00064230093FF220B46F7E7436807EE903A22
:104AC00099B19FED1F7A77EE677AF5EEC07AF1EE35
:104AD00010FA30D4F4EEC77AF1EE10FA2DDCFDEEC8
:104AE000E77A17EE903A18B2D2E7F5EEC07AF1EE17
:104AF00010FAD2D49FED127AECE7436861B142F22A
:104B00007372934217DC13F1630F16DB6FF06300CF
:104B100093FBF0F06430BAE713F1630FBDDB42F2B0
:104B2000737293424FF06400B2DC93FBF0F0AEE797
:104B30004FF0FF30ACE70020AAE76420A8E700BFF1
:104B40000000C84213B50446084663781B09013BC0
:104B50000A2B32D8DFE803F00F0F313131281A3138
:104B600031060600FF2300930023642219460BF050
:104B7000B8FE606007E0FF2300930023642219461B
:104B80000BF0AFFE2071012002B010BDFF23009397
:104B90000023642219460BF0A4FE07EE900AF8EEFB
:104BA000E77A17EE900AE4E746F29C33009300237D
:104BB000642219460BF095FE60600020E4E70000D7
:104BC00043781B090B2B5FD8DFE803F06117175EF2
:104BD0005E5E461E5E5E0606406841B1002839DB17
:104BE000FF28A8BFFF20C0F1FF0001B20AE00028A3
:104BF00008DBFF28A8BFFF20F7E700790029F4D0E1
:104C0000C0F1FF01084670474368A9B107EE103AAA
:104C1000B5EEC07AF1EE10FA1CD4DFED1E7AB4EED8
:104C2000E77AF1EE10FA32DC77EEC77AFDEEE77A3A
:104C300017EE903A19B2E5E707EE903AF5EEC07A32
:104C4000F1EE10FADED49FED137AF4EEC77AF1EEAE
:104C500010FAEBDDFF21D5E7406859B110F1630F81
:104C6000F8DBB0F5C84F12DA6FF0630190FBF1F09A
:104C7000FF30BAE710F1630FC4DBB0F5C84FE9DAD3
:104C8000642190FBF1F0B0E74FF0FF31BAE700216B
:104C9000B8E700BF00007F43007870474078000904
:104CA00070474B7810B562F307134B700B680360C5
:104CB0004B68436010BD4B7810B51C09013C012CBA
:104CC00084BF012464F3071382F30802D2B288BFC1
:104CD0004B700B680A7103604B68436010BD4B78E2
:104CE0004A6030B50A2565F307134B700B68036003
:104CF0004B68436030BD4B784A6030B5072565F39B
:104D000007134B700B6803604B68436030BD4B78F2
:104D100030B5062565F307134B700A235A434A60E2
:104D20000B6803604B68436030BD4B784A6030B518
:104D3000062565F307134B700B6803604B684360EF
:104D400030BD70B54C788A71022666F307144C703A
:104D5000C2F30024CA794B7122F001029DF8103091
:104D60000B7122430B68CA7103604B68436070BDCE
:104D700070B54C788A71032666F307144C70C2F341
:104D80000024CA794B7122F0010222430B68CA71D8
:104D900003604B68436070BD70B54D784B7104265D
:104DA00066F307159DF810304D700B718A710B6812
:104DB00003604B68436070BD70B54D784B7105263C
:104DC0009DF810300B7166F307159DF814304D7087
:104DD000CB718A710B6803604B68436070BD4B7880
:104DE0004A6030B50C2565F307134B700B68036000
:104DF0004B68436030BD10B50A700B6803604B68A8
:104E0000436010BD407800F00F0070474B7810B53C
:104E100062F303034B700B6803604B68436010BD83
:104E20002DE9F041044616460D4619B900273846CB
:104E3000BDE8F0810846FDF71BFC07460028F5D0C9
:104E40002846FDF76FFBF305804603D52846FDF79E
:104E50005DFA207006F40076B8F1000F09D063788F
:104E600068F307136370002EE1D0EB685B69636041
:104E7000DDE7002EDAD0EA68137C03F00F03022B83
:104E800003D0032B09D04746D1E7637852696260AB
:104E90000A2161F307136370C9E753696278072138
:104EA00061F307126270E2E710B500230446037055
:104EB00043708370C370037143718371C3714FF486
:104EC0000072FFF7ADFF204610BDF8B50546174646
:104ED0000C4611B900263046F8BD0846FDF7C8FB60
:104EE00006460028F6D079050CD52B780A3B032B13
:104EF00008D8DFE803F01F02242A4FF4803120464F
:104F0000FDF744FAFA0507D52978A1F10A03032B26
:104F100002D92046FDF708FABB05DCD56B78696835
:104F20001B09073B2046042B18D8DFE803F01111BA
:104F3000171414004FF480312046FDF767FA4FF440
:104F400000312046FDF762FADCE74FF40031D6E786
:104F5000FDF71EFBBFE7FDF7FFFABCE7FDF7FCFA24
:104F6000697820460909FDF72FFBB4E770B5174EA5
:104F7000174D044634B3237C03F00F03023B042B8C
:104F800020D8DFE803F0031F0F06080065692846F4
:104F900070BDE468EEE721463246284609F011FD6F
:104FA0000446E7E766693046FFF72CFB051E09DB80
:104FB000304609F0FBFD237C6561022262F30303A6
:104FC0002374E4E74FF0FF35E1E700BF8182010081
:104FD000780700202DE9F0432DED028B85B00446C3
:104FE000154699469DF838800F46002948D0002A7A
:104FF00000F0E78000230B70017871B319F4807F13
:105000002BD0714B01EBC101194438460FF025F943
:10501000637813F0F00F07D019F4007F04D02A460C
:105020006A4938460FF0F3F838460FF0E8F82D1AC1
:105030003E18013D637813F0F00F21D019F4007F82
:105040001ED01B09013B0B2B1AD8DFE803F00840E8
:1050500071A6AC257B7B7B221FB43E46EAE7207914
:10506000B8F1000F06D0642300930023FF221946F5
:105070000BF037FC564A0346294630460EF0B4FF83
:10508000384605B0BDEC028BBDE8F0836368514A39
:10509000F2E76368504AEFE7616800294FF0640265
:1050A0000EDA91FBF2F04B4202FB1011494293FBE6
:1050B000F2F34A4A0091294630460EF095FFDFE7A9
:1050C00091FBF2F302FB13120092454AF3E72046EC
:1050D000FFF77BFBE279A37994F8059001B20029F0
:1050E000207902F0010202DBB8F1000F14D043EA8C
:1050F0000224B8F1000F06D0642300930023FF229E
:1051000019460BF0EEFBCDE900902346354A2946BF
:1051100030460EF069FFB3E7CDE90101CDF800900C
:1051200043EA0223304A294630460EF05DFFA7E7E6
:10513000E379A2796179009103F0010342EA032344
:105140002A4AB8E7636808EE103AB5EEC08AF1EE75
:1051500010FA4CBFF1EE487AF0EE487AFDEEE78A9D
:10516000B8EEE87A77EEC77A9FED217A67EE877A14
:1051700017EE900A0CF006F807EE900AB5EEC08A1A
:10518000FDEEE77AF1EE10FACDED007A18EE903AE6
:1051900001D5184A8FE7184A8DE72279A379019241
:1051A00062790092B2E7E279A379029222790192C0
:1051B00062790092B6E72A46616830460FF04DF8F2
:1051C0005EE717465CE700BF86820100A07E010013
:1051D000C6840100C9840100CD840100D18401008E
:1051E000D2840100DE840100DB840100E18401003F
:1051F00000007A44E7840100E884010030B58BB0F8
:10520000134C00232022009302A94FF4407305465B
:10521000FFF7E0FE02A920460AF0E5FE0D49204610
:105220000AF0D8FE69780A22090920460AF054FFDC
:10523000094920460AF0CEFE69780A2201F00F01E2
:1052400020460AF049FF20460AF0D4FE0BB030BDDC
:1052500070030020BA840100BF84010070B54B7850
:10526000B2EB131F86B005460C46164606D12368DE
:105270002B6063686B60284606B070BD18491948FA
:105280000AF0A8FE617817480A2209090AF024FFEB
:10529000154914480AF09EFE0A22314611480AF0C8
:1052A0001BFF12490F480AF095FE0023CDE9043395
:1052B00066F3071322788DF811304FF0FF338DF825
:1052C0001020009302A86368226804A900F010F877
:1052D000029B2360039B63602046FFF78FFFC6E7B6
:1052E000F084010070030020FE7D0100A07E01001B
:1052F0002DE9F04F8DB004AD85E80C00BDF85830B5
:10530000112B98BFB64A804628460C4694BF12F827
:1053100003904FF00009FFF758FA011E02DB204608
:10532000FFF72DFA9DF811306278C3F3030161F3A2
:10533000030262709DF810102170C2F303120B2A51
:1053400038D8DFE812F0A0000C000C00C9002F01D3
:105350000D01A800CF00CF00CF00A800A8001B09B6
:105360000C2B77D8DFE803F0265244180A0739558A
:10537000767630306E009DF81720E2719DF8162089
:10538000A2719DF8152062719DF814202271627837
:1053900063F3071262700DE0BDF81630C3F3080224
:1053A000E379A27123F0010343EA1223E3719DF82C
:1053B00015306371B9F1000F00F0FC804A462146B8
:1053C00006A8FFF74BFFF5E0059B002B36DBFF2B14
:1053D000A8BFFF23DBB22371ECE7059B13F1630F3A
:1053E0002CDBB3F5C84F2BDA642293FBF2F3F1E721
:1053F000BDF81630C3F30802E379A27123F001036C
:1054000043EA1223E3719DF8153063719DF814305F
:10541000E1E7DDED057AF5EEC07AF1EE10FA0DD494
:105420009FED707AF4EEC77AF1EE10FA08DCFCEE2C
:10543000E77ACDED037A9DF80C30CCE70023CAE77C
:10544000FF23C8E763780C2262F307136370059BA0
:105450006360AFE7644965480AF0BCFD9DF8111030
:1054600062480A2209090AF037FE61495F480AF0DA
:10547000B1FD61785D480A2209090AF02DFE5B48FA
:105480000AF0B8FD96E762781B0963F307120598E6
:10549000627060608EE71B09032B04D00C2BD1D007
:1054A000059A626073E700212046FFF789FBBDF88B
:1054B00016302071C3F30802E379A27123F00103CF
:1054C00043EA1223E3719DF8153063716378022279
:1054D00062F3071363706DE700212846FFF770FB46
:1054E0002071F3E71B090C2BB4D801A252F823F06A
:1054F000B55300002F5500005D550000A754000073
:105500005D5500005D550000255500005155000017
:1055100051550000515500003D5500004B5500000D
:1055200045540000059B636006226378D0E79DF830
:10553000143007EE903AF8EE677A03E0DDED057A75
:10554000F8EEE77A17EE903A82E7DDED057AF2E7BA
:10555000627863F307126270059B79E7627894E7DB
:1055600001271B090C2B3FF675AF01A252F823F05F
:10557000B5530000C95500001D560000C955000074
:10558000A9550000A9550000C9550000C9550000E3
:105590005554000055540000C9550000C95500007D
:1055A000455400000027DCE7059A6260627863F3E7
:1055B000071262702368C8F800306368C8F80430C6
:1055C00040460DB0BDE8F08F013B0A2B00F2CD80C4
:1055D000DFE803F0BACB10CBCBBFC4CBCBBDBD0053
:1055E0006F82010000007F433684010070030020B9
:1055F000FE7D0100FF23BDF816208DF814306421D4
:1056000061F30802ADF8162000228DF815209DF8F0
:105610001120022161F307128DF811200023FF25CC
:105620009DF815000095642219460BF05AF90028E0
:10563000C0F29D8000239DF8150000956422194654
:105640000BF04FF9A84208DC002300959DF81500E7
:10565000642219460BF045F905469DF81400FAF747
:1056600009FF0646002F47D09DF817707F08013FBD
:105670003FB27B1C40F088807F2D4FF0FF0778DC25
:105680000023C5F17F00194647F6816270430097F9
:105690000BF027F94FF4FF73009300231946E071D4
:1056A0007F2228460BF01DF90023194600903A4648
:1056B00030460BF016F900970646642328467F22F1
:1056C00000210BF00EF9BE420546A8BF3E466C49CC
:1056D0006C480AF07FFC0A2229466A480AF0E3FC7B
:1056E000694968480AF076FC0A22314665480AF0A2
:1056F000DAFC64480AF07EFC00231A46194606A824
:105700000AF0E0FABDF816004FF6FF73009300238D
:10571000194640F26D12C0F308000BF0E2F8F2B245
:10572000E9B280B20AF0E4FA030CA371030A6371D0
:105730002071564953480AF04DFC2046FFF75EFDA4
:1057400006A80AF054FA35E69DF8143053E7059B95
:1057500051E7059B642293FBF2F34CE7DDED057AFC
:10576000FDEEE77A17EE903A45E7002343E7002580
:1057700073E76423284600973A4680210BF0B1F87E
:1057800000230546E371A2E74FF01E0B64231A467F
:10579000CDF800B0002138460BF0A3F84FF0640AB2
:1057A00003905B463846CDF800A0524600210BF02E
:1057B00098F87F2D83464FF0FF0754DCC5F17F003A
:1057C000002370431946324A00970BFB00F00BF0A0
:1057D00088F84FF4FF73E071039800930023194693
:1057E000E32228180BF07DF80023194600903A4672
:1057F000824630460BF075F800230646009728468F
:105800007F2219460BF06DF8BE420546A8BF3E4602
:1058100020491C480AF0DEFB0A22039919480AF0C5
:1058200020FC1D4917480AF0D5FB0A2259461548A5
:105830000AF017FC194913480AF0CCFB0A22294642
:1058400010480AF030FC16490E480AF0C3FB0A2241
:1058500031460C480AF027FC12490A480AF0BAFB04
:105860000A22514642E75346284600973A4680218D
:105870000BF037F84FF0000A054684F807A0C7E799
:1058800048840100700300205584010088840100D1
:10589000646A310063840100698401006F8401003F
:1058A000778401007F84010073B504460D46FFF73D
:1058B000B7FA0646E8B9104910480AF08BFB2846AB
:1058C000FDF7F2FB214602B26846FEF7CFFE214605
:1058D0006846FEF7FFFE29464FF400722046FFF7A8
:1058E000F4FA2046FFF78AFC4FF490512846FDF762
:1058F00081FB304602B070BD8F8401007003002030
:1059000043781B09013B012B37B5054620D80023FE
:10591000FF2400790094642219460AF0E2FF00286F
:1059200014DB002328790094642219460AF0D9FF79
:10593000A04207DC002300942879642219460AF06B
:10594000D0FFC4B22C71012003B030BD0024F9E7B0
:105950000020F9E707B5002300931A4619460348CB
:105960000AF0F0FA03B05DF804FB00BF3803002032
:1059700002F008BE02F0C8BD07B5002300931A4626
:10598000194603480AF0DEFA03B05DF804FB00BFD5
:1059900040030020024B0F221A70C820704700BF3E
:1059A000E003002008B5044904480AF013FB04F0A2
:1059B000E5FC4FF4FA7008BD7B8A0100BC030020AF
:1059C00038B5094D01244FF47A700BF033F92146B4
:1059D00001340A222846E4B20AF07EFB142CF2D1EC
:1059E0004FF4FA7038BD00BFBC03002008B504F0C6
:1059F00087F8C82008BD10B5044604300AF07BFFC4
:105A0000204610BD0128F8B507460C46174E184D24
:105A100013DD48680DF0C7F9C1B216483170FBF7C5
:105A200037F9022F07D0A0680DF0BDF9C1B21148B7
:105A30002970FBF73EF9C82401E04FF4C8740E4901
:105A40000E480AF0C7FA0A2231780C480AF044FBE3
:105A50000B490A480AF0BEFA0A22297807480AF0D8
:105A60003BFB06480AF0C6FA2046F8BD05000020B8
:105A700006000020440400201C8C0100BC03002010
:105A8000308C010030B587B00023044600931A46DD
:105A90000D4602A819460AF055FA04A80AF04AFA77
:105AA000042C12DD04A9286904F072FB68B104A972
:105AB0002548FAF7D2FF04A9E86804F069FB50B161
:105AC00004A92148FBF715F80BE002A91E48FAF7D4
:105AD000C4FF032CEFDC02A91B48FBF70AF8022CD9
:105AE0001CDD04A9A86804F053FBB8B104A916484A
:105AF000FAF7D9FF04A9686804F04AFBA0B104A929
:105B00001148FAF784FF114911480AF063FA00219D
:105B10000D48FBF78DF8C82007B030BD02A90A4830
:105B2000FAF7C1FF012CE5DC02A90748FAF76FFF7D
:105B3000012CE8D102A90448FAF769FF0549044895
:105B40000AF048FADFE700BF44040020C6860100DF
:105B5000BC030020B686010008B548B14968054875
:105B6000FAF705FE044905480AF034FAC82008BDD2
:105B70000146F4E744040020658A0100BC030020CC
:105B8000012838B50C4630DD4D68214928460EF015
:105B9000CEFA28B901211F48FBF767F8C82038BDA5
:105BA0001D4928460EF0C3FA01460028F3D01B49D0
:105BB0001B480AF00FFA1748FBF74DF80A22014676
:105BC00017480AF070FA16480AF014FA616811488A
:105BD000FAF71EFE616812480AF005FA11491048EA
:105BE0000AF0F8F90E480AF005FA0F4B93F9002075
:105BF000012A02DDF0221A70D0E70C490C480AF0A5
:105C0000E9F90B480AF0F6F94FF4FA70C7E700BF5C
:105C100024920100440400202D920100F48601002A
:105C2000BC03002014870100E00300201B87010053
:105C30008C03002008B548B149680548FAF76CFDA7
:105C4000044905480AF0C6F9C82008BD0146F4E732
:105C50004404002028870100BC03002030B5144D07
:105C6000144C85B0772201212846FBF751FA002316
:105C70000193114B0093114902954FF0FF332046D9
:105C800003930AF0A7F90E4B0E4819686A4608F00C
:105C90005DFE2846FBF7E8F90B4920460AF09AF921
:105CA00020460AF0A7F90948FBF7ECF805B030BD2B
:105CB0005C040020BC030020A89B0100C4890100F3
:105CC0003804002078070020DE8901004404002009
:105CD000012810B50C4622DD124960680EF027FA43
:105CE00018B901211048FAF786FF104960680EF0D4
:105CF0001EFA014610B90C48FAF77DFF0C490D4811
:105D00000AF068F90848FAF76CFF0A2201460948C8
:105D10000AF0C9F907480AF06DF9C82010BDFFF76D
:105D20009DFFFAE724920100440400202D92010017
:105D3000EE890100BC03002008B50A48FBF75CF8B7
:105D400018B1094909480AF045F9722201210848A9
:105D5000FBF7DEF90648FBF77BF90548FBF784F90A
:105D6000C82008BD44040020868D0100BC0300202B
:105D70005C0400202DE9F041484F3B688CB0002BBB
:105D800000F08980464B1B7853B1464946480AF0DB
:105D900021F945480AF02EF900200CB0BDE8F08149
:105DA0004249434D4348444E0AF014F941480AF031
:105DB00021F92B7801335BB22B70336803B3DC68B5
:105DC000DFF810811CB3237C03F00F03052B15D1E2
:105DD0002146404608F0E1FD80B1326821686846FE
:105DE000FCF708FD6846FCF743FC10B16846FCF779
:105DF0007DFA0AF041FF6846FCF77EFA6468E1E745
:105E00002E492C480AF0E6F82A480AF0F3F82C4B01
:105E10002C49284800241C600AF0DCF825480AF0C8
:105E2000E9F864200AF006FF274B28491C70284B2C
:105E300020481C700AF0CEF804F0A2F90A220146AC
:105E40001C480AF03CF93968224808F0A6F9224BB0
:105E500022491C60224B17481C60224B3C601C608E
:105E6000214B34601C60214B1C60214B1C70214B6A
:105E70001C600AF0AFF804F083F90A2201460D48CD
:105E80000AF01DF90B480AF0B5F81B4B1C702B7873
:105E9000013B5BB22B7001207FE700BF380400207C
:105EA0006D030020909101008C030020A791010058
:105EB0008804002070030020DC030020BD91010055
:105EC00034040020CD91010080040020D591010010
:105ED0006C03002078070020D80300206A820100AC
:105EE000A004002068030020E403002088030020B1
:105EF000640300202C0400206E030020034B93F960
:105F00000000053818BF0120704700BFE0030020E3
:105F100030B593B000230A460546402101A804F09D
:105F2000A9F901A80EF06BF901A90446024628461A
:105F30000EF081F900280CBF2046002013B030BDC0
:105F4000F0B504469DB00E4601B18AB969496A4868
:105F50000AF040F8694968480AF03CF8214666486A
:105F60000AF041F8664964480AF034F862481DE0D6
:105F700000258D5404F004F90A22014607465E48C4
:105F80000AF091F85F495C480AF024F821465A4823
:105F90000AF029F85C4958480AF01CF8B7F59D7FCB
:105FA00008DA5A495A480AF015F859480AF022F80E
:105FB0001DB0F0BD04215748574F03F0DFFE57498D
:105FC0004D480AF007F831464B480AF00CF853499F
:105FD000494809F0FFFF48480AF00CF83C222946DE
:105FE0000DA80C950DF065F997F90020052A27D129
:105FF00003212046FFF78CFF05B26DBB484DEB68CF
:106000001B78DB07D4D501212046FFF781FF00B2C2
:106010000028CDD0242120460EF040F90028C7D119
:106020004049354809F0D6FF2146334809F0DBFFE7
:10603000314809F0DFFF2146284609F0FCF9B7E7AF
:1060400001212046FFF764FF05B2C5B902212046B1
:10605000FFF75EFF05B2C5B12544334928460EF06F
:10606000A0F8A0B930460EF0CAF801280FD9214691
:106070002B4809F0E0F9304608F0C0FD98E73F22D0
:1060800021460CA80EF0E9F8E6E728496BE7204620
:1060900024210EF003F90446002889D1244B294617
:1060A0001A686846FCF7A6FB6846FCF7E1FAE0B11F
:1060B000224631466846FDF7BFFE002815DD9DF8F3
:1060C000303093B197F90030052B0ED019490A48AA
:1060D00009F080FF0CA9084809F085FF064809F07F
:1060E00089FF0CA90E4809F0A6F96846FCF704F9E7
:1060F0005EE700BFC99B01007003002053860100CA
:1061000008A101005C8601005F8601006286010033
:106110008C0300203C040020E0030020747D01007B
:10612000E80300206F860100129201008D860100B5
:10613000DC030020988601002DE9F041164917483C
:10614000174E184F154D09F045FF0024A6F10F0812
:1061500016F8013F0F2B03D83946284609F043FFB4
:10616000052C4FF010020DD03178284609F079FF48
:106170000D49284609F02EFF0134E4B2062CE7D180
:10618000BDE8F08198F81510284609F06AFF284606
:1061900009F030FFF0E700BFFF890100BC030020D9
:1061A000530400208C9B01000680010010B58AB0CA
:1061B0000DF11F0304930DF12503039309AB0C4666
:1061C00002930DF1230301930DF12203009308AA1A
:1061D0000DF121030E4960680DF03AFF05280BDC34
:1061E0000C490D4809F0F6FE61680B4809F0FBFE0A
:1061F0004FF4C8700AB010BD08A90848FAF73FFA72
:10620000FFF79AFF0649074809F0E4FEC820F1E7C6
:106210008D8A0100A18A01008C0300204404002023
:10622000B38A0100BC03002008B508B9002008BDEE
:10623000037C03F00F03052BF8D1CAB201460648D0
:1062400008F0B5FB0028F1D0037C03F00F03042B0A
:10625000ECD14069EBE700BF78070020F7B53C4C74
:106260002678002E6CD13B4B93F90030012B67DD73
:10627000394B1968002963D0384A394808F0A1FB26
:10628000054600285CD00146354808F086FB07B279
:10629000002F55D031462846FFF7C6FF012F06468E
:1062A00050D0294601222E4808F081FB45696846F6
:1062B00005F082FA10222B49684603F08FFF2A4925
:1062C0002A4809F087FE3146284809F08CFE284903
:1062D000264809F088FE0A222946244809F0E3FEF0
:1062E0002349224809F07FFE1E49204809F07BFE21
:1062F0001E4809F07FFE40F202211E4805F0F4FC22
:10630000AAB231461C481D4D09F062FD15491A48D4
:1063100009F062FD1A4B186818B10021FFF784FFDD
:106320002860296889B1144809F05EFD00211248EF
:1063300009F062FD012313490C48237009F04AFE5D
:1063400003B0F0BD40F20225B1E70F49EBE700BF13
:1063500080040020E0030020380400200E860100A5
:10636000780700205403002015860100BC0300209C
:1063700006800100C8040020A40400208803002037
:10638000E403002024860100B293010008B5094B04
:106390001B7873B1084B1B6813B1DA68074B1A609E
:1063A0000749084809F016FE0648BDE8084009F00C
:1063B00021BE08BD6403002068030020E403002020
:1063C0003F870100BC03002008B50B4B1B788BB145
:1063D0000A4A13685B6813601BB9BDE80840FFF701
:1063E000D5BF0749074809F0F5FD0648BDE8084054
:1063F00009F000BE08BD00BF64030020E4030020D4
:10640000D9860100BC0300202DE9F04FA7B000237E
:1064100097488DF81330CDE90533CDE9073308F0FF
:1064200021FE944F054610B105233B70F8E0924CD5
:10643000216841B99149924809F0CCFD904809F092
:10644000D9FD0F23F1E78F4808F0A7FA0FFA80F87B
:10645000B8F1010FEEDD294620688B4EFFF7E4FE10
:10646000002800F0E08030608849894809F0B2FDDA
:106470003168874809F0B7FD854809F0BBFD012167
:106480002068FFF7D1FEB8F1020F824600F0CE80FF
:10649000022221687B4808F08AFAB8F1030FD0F88D
:1064A000149000F0C58003212068FFF7BDFE05466B
:1064B000102205A97748FAF709F9002840F0BB80B7
:1064C000B8F1040F40F3B78004212068FFF7ACFE59
:1064D000714904466E4809F07DFD6D4809F08AFD5A
:1064E0001FFA89F25146624809F028F90DF1240893
:1064F0006A495F4809F025F90DF1340B102268490B
:1065000040460DF0AAFE002301222021584603F048
:10651000B1FE644958460DF028FE63495C4809F015
:1065200059FD51465A4809F05EFD6049584809F046
:1065300051FD0A224946564809F0B5FD5C495448C8
:1065400009F048FD2946524809F04DFD5949504887
:1065500009F040FD2B780BB91C461D46CDF80C8088
:106560004FF002094FF001082A46CDE90198CDF815
:1065700000B0234631683E484F4D08F089FE0028A0
:106580005BD04E4B4E49424800241C7009F022FD5E
:1065900031683F4809F027FD3D4809F02BFD494B84
:1065A000032283F800804121234615A803F062FEF0
:1065B000454915A80DF0D9FD15A92D4809F08CF80D
:1065C00023464A46412115A803F054FE3F4915A829
:1065D0000DF0CBFD15A93E4809F01CFD15A9244876
:1065E00009F07AF842462346412115A803F042FEFD
:1065F000364915A80DF0B9FD15A9354809F00AFD71
:1066000015A91B4809F068F805233B700AF0DEFA6B
:10661000304928601E4809F0DDFC1D4809F0EAFCFD
:1066200027B0BDE8F08F2C4B33601DE740F25B795B
:106630000DF113053CE705AC52E72849104809F075
:10664000C9FC0B4809F07FF80A2201460C4809F002
:106650002AFD23490A4809F0BDFC094809F0CAFC93
:10666000FFF7B2FE0AF0B2FA0C232860DDE600BFA5
:10667000E8030020E0030020E4030020678F01000E
:106680008C0300207807002088030020A38F0100DE
:10669000BC03002044040020B08F0100415F0000D3
:1066A000589301009C930100D08F010006800100E7
:1066B000F18F0100B891010090040020280400200F
:1066C000F88F01006E03002006900100FC7D0100A0
:1066D000700300200C900100B29301002F90010084
:1066E0004190010007B51049104809F073FC684655
:1066F00005F062F8684603F097FD0D4B00930D4BD3
:1067000068465B68019303F08FFD684605F098F8D2
:10671000684603F089FD684605F070F8684603F0A6
:1067200083FD03B05DF804FB9E8C0100BC030020D8
:10673000749C01006406002010B5114C11492046DC
:1067400009F048FC1049204609F04DFC4FF4FA705E
:106750000AF070FA012115200AF026FC002115200C
:106760000AF04AFC4FF4FA700AF064FA152001218D
:106770000AF042FC4FF4FA70BDE810400AF05ABA31
:10678000BC030020EF9101000F92010070B592B0A0
:1067900002A809F0CFFB04A809F0CCFB06A809F079
:1067A000C9FB08A809F0C6FB71497248724E09F08E
:1067B00011FC704809F01EFC02A97048FAF753F862
:1067C000F8B96F496B486F4C09F004FC4FF47A62DA
:1067D00042F6E0616C4804F08FFE002840F09180A2
:1067E0006A496B4809F0F6FB6A49694809F0F2FB0F
:1067F000237801332370F6233370FFF79DFF12B027
:1068000070BD5E48FAF70CFA18B15E4B1B78022B8C
:10681000D7D961495748614C10AD09F0DBFB039BA8
:1068200010942846119303F0FFFC04A95348FAF78B
:1068300084F800285DD05A494E4809F0CBFB059BEF
:1068400010942846119303F0EFFC06A94B48FAF781
:10685000A9F8002841D05349464809F0BBFB079BE3
:1068600010942846119303F0DFFC08A94348FAF777
:106870002FF810B34C493F4809F0ACFB099B11932A
:106880002846109403F0D0FC039B0095CDE90B340F
:10689000059B3D480A94CDE90D34079BCDE90F34A3
:1068A000099B11930CAA0EAB0AA904F0AFFE314864
:1068B00009F0A0FB02233370A1E7039B32480C943C
:1068C000CDE90D34059BCDE90F34079B11930EAA3A
:1068D0002B460CA904F0CAFEE9E7039B2A480E9454
:1068E000CDE90F342A46059B11930EA904F0E6FE6C
:1068F000DDE7039B244810942946119304F0F8FE29
:10690000D5E72A491B4809F065FB10A804F054FF9D
:10691000119B039310A8214B109303F085FC15489D
:1069200009F068FB02A91548FAF771F8204B1348E3
:106930005B68119304A90593FAF7B5F810A804F061
:106940007FFF119B0D48079306A9FAF7D2F810A80C
:1069500004F054FF119B0948099308A9FAF77DF840
:1069600001210648FAF764F900232370A2E700BF6B
:10697000C48C0100BC030020E0030020440400207C
:10698000D18C01004803002054040020058D010033
:106990008C030020478D0100DD8C0100749C0100F8
:1069A000F38C0100F98C0100FE8C0100768D010052
:1069B0006406002018B10349034809F00BBB0349E2
:1069C000FAE700BFED910100BC0300200BA101001C
:1069D00010B5264C2649204609F0FCFA25492046E8
:1069E00009F0F8FA244B1868003018BF0120FFF7AF
:1069F000E1FF2249204609F0EDFA214B18680030EA
:106A000018BF0120FFF7D6FF1E49204609F0E2FA21
:106A10001D4B1868003018BF0120FFF7CBFF1B4942
:106A2000204609F0D7FA1A4B1868003018BF012029
:106A3000FFF7C0FF1749204609F0CCFA164B18782B
:106A4000FFF7B8FF204609F0D5FA1449204609F0AF
:106A5000C1FA03F095FB0A220146204609F02FFBFC
:106A60002046BDE8104009F0C5BA00BFBC030020B5
:106A7000E58B0100F28B0100DC030020FA8B0100A2
:106A8000D8030020038C0100E40300200A8C0100DD
:106A90002C040020138C010080040020558001008C
:106AA0000020704710B5484C4849204609F092FA3A
:106AB0004749204609F08EFA4649204609F08AFAED
:106AC0004549204609F086FA204609F093FA4349E1
:106AD000204609F07FFA4249204609F07BFA4149F5
:106AE000204609F077FA4049204609F073FA3F49F9
:106AF000204609F06FFA3E49204609F06BFA3D49FD
:106B0000204609F067FA3C49204609F063FA3B4900
:106B1000204609F05FFA3A49204609F05BFA394904
:106B2000204609F057FA3849204609F053FA374908
:106B3000204609F04FFA3649204609F054FA354903
:106B4000204609F047FA3449204609F043FA334910
:106B5000204609F03FFA3249204609F03BFA314914
:106B6000204609F037FA3049204609F033FA2F4918
:106B7000204609F02FFA2E49204609F02BFA2D491C
:106B8000204609F027FA2C49204609F023FA2B4920
:106B9000204609F01FFA2A49204609F01BFA294924
:106BA000204609F017FA2849204609F013FA274928
:106BB000204609F00FFA2046254909F00BFA204635
:106BC000BDE8104009F016BABC030020968D010004
:106BD000B88D0100CB8D0100D98D0100E18D010040
:106BE000F18D0100FD8D01000A8E01001F8E010054
:106BF0002E8E0100368E0100418E01004E8E010066
:106C0000588E0100678E01006F8E01007B8E01009F
:106C10000F920100918E0100B08E0100C58E01001F
:106C2000D28E0100E08E0100EC8E0100F48E010096
:106C3000FF8E01000C8F0100148F01001F8F0100D7
:106C40002E8F0100378F0100458F0100538F010007
:106C50005F8F010008B5FFF725FFFFF743FD0349EC
:106C6000034809F0B7F9C82008BD00BF56870100E6
:106C7000BC03002070B594B003F082FA064609F018
:106C8000A5FF05462D4808F0EDF9002854D02C4BFF
:106C90001C7864B2002C4FD123460122402104A865
:106CA00003F0E8FA274904A80DF05FFA264904A882
:106CB0000DF05BFA254904A80DF057FA31466846F5
:106CC00003F056FB01236A4604A91C4808F027FC80
:106CD00023460122402104A803F0CCFA194904A854
:106CE0000DF043FA184904A80DF03FFA184904A81A
:106CF0000DF03BFA68464FF47A71B5FBF1F103F001
:106D000037FB01236A4604A90C4808F008FC234617
:106D10000122402104A803F0ADFA0E4904A80DF0A9
:106D200024FA0F220C4968460DF097FA01236A46AF
:106D300004A9024808F0F3FB14B070BDE80300207A
:106D4000B8030020A39301001B8B010006930100F0
:106D5000BB9301009C9301009693010010B50C4C6D
:106D60002046F9F75DFC78B90A490B4809F032F979
:106D7000DE232374AD236374BE23A374EF23E37473
:106D8000FE232375FF236375BDE81040FFF7D4B9D8
:106D9000440400203E8A0100BC03002008B5002006
:106DA00007F0E8FF1C491D4809F014F91C491D486B
:106DB00007F06EFF1C491D4807F06AFF1C491D487B
:106DC00007F066FF1C491D4807F062FF1C491D487B
:106DD00007F05EFF1C491D4807F05AFF1C491D487B
:106DE00007F056FF1C491D4807F052FF1C491D487B
:106DF00007F04EFF1C491D4807F04AFF1C491D487B
:106E000007F046FF1C491D4807F042FF1C491D487A
:106E1000BDE8084007F03CBF048A01007003002071
:106E2000556C0000088A0100D15C00000D8A010049
:106E300095590000128A0100815B00001C9401003A
:106E4000AD610000178A0100855A00001B8A01000D
:106E5000595B00001E8A0100C1590000258A01000B
:106E6000355C0000218A0100395D00002A8A01009A
:106E7000A5590000308A0100055A00001186010062
:106E8000ED590000378A01002DE9F04F424E33687A
:106E900087B08046002B7CD0404D2C7864B2002C0B
:106EA00077D12B783E4FDFF8089101335BB22B701E
:106EB0003B7801335BB23B70D9F800A009F086FE45
:106EC000234601460B22504603F068FA002858D0AA
:106ED000B8F1030F0BD0334BD3F800A009F076FEC6
:106EE000234601466422504603F058FA04463368AC
:106EF000DFF8C0B0DE68AEB3337C03F00F03062BBF
:106F00002ED1314600226846FAF7B2F9414668466A
:106F1000FBF738F91CB104216846FBF733F9224A24
:106F20003146584607F04DFDD0B1037C03F00F0306
:106F3000052B15D1D0F80CA0BAF1000F10D0514696
:106F4000324603A8FAF794F9414603A8FBF71AF969
:106F50001CB1042103A8FBF715F9DAF804A0EBE74C
:106F60007668C8E7B8F1030F03D009F02FFEC9F81F
:106F700000001CB109F02AFE0A4B18600B48FBF711
:106F800031F93B78013B5BB23B702B78013B5BB244
:106F90002B7007B0BDE8F08FD8030020D503002088
:106FA0006D030020EC040020F07D01002C03002084
:106FB0008C040020780700200220FFF765BF000046
:106FC00010B5094C237801335BB2237009F054FEED
:106FD0000320FFF759FF09F04FFE07F0B9FE2378B1
:106FE000013B5BB2237010BDB8030020F0B51E4E0C
:106FF000336885B0002B34D01C4B1C7864B284BB42
:107000001B4D2F6809F0E2FD2346014641F288320C
:10701000384603F0C3F920B3164A137801335BB244
:1070200013703368DC681646A4B1237C03F00F03A9
:10703000062B08D12146002201A8FAF719F90121EF
:1070400001A8FBF79FF809F017FE0220FFF71CFFCD
:107050006468E9E709F0BAFD28603378013B5BB268
:10706000337005B0F0BD00BFD8030020D503002069
:10707000980400206D03002030B51449144885B0F1
:1070800008F0A8FF124808F0B5FF124B1968D9B1F3
:10709000114CCD682278013252B2227085B12B7C1E
:1070A00003F00F03062B07D10022294601A8FAF7A7
:1070B000DFF801A8FAF714F909F0DEFD6D68EDE7D5
:1070C0002378013B5BB2237005B030BD1C85010005
:1070D000BC030020D80300206D0300202DE9F04FF1
:1070E000A54C23688FB0002B00F04181A34F3B7863
:1070F000002B40F03C813B78A149A248A24EA34D11
:1071000001335BB23B7008F065FF9E4808F072FFE8
:107110009F4A21689F4807F054FC9F4A30602168CD
:107120009C4807F04EFC9D4B9D4A18602168994889
:1071300007F047FC9B4B9C4A18602168954807F074
:1071400040FCB1462860994E002800F08180C36859
:10715000002B7DD01B7C03F00F03052B78D19449C5
:10716000884808F037FF29688A4807F016FC914BD9
:10717000014618700A22834808F0AEFF814808F0E3
:1071800039FF2B68DB683360FFF768F88A4A2168AB
:10719000804807F016FC894B186070B1884C237842
:1071A0005BB902F0AFFC002814BF01230023237059
:1071B00003D08449734808F00DFF834A002313600D
:1071C000D9F800309246002B00F0B380D3F80C8041
:1071D000DFF820B27D4DD9F80030002B00F0CA80D6
:1071E000B8F1000F00F0A28098F8102002F00F0212
:1071F000052AF2D14146674807F0CFFB0128EAD9BA
:10720000D9F80020414602A8FBF7BEFA02A8FBF716
:107210002FFAA8B102A8FBF7D3F8064680B90146B9
:1072200002A8FBF70BF9041E02A8BCBF64420126AA
:10723000FBF76CF89DF81C20052A0BD0062A46D0D7
:1072400009F01AFD02A8D8F80480FBF755F8C2E748
:10725000306099E718B9022102A8FBF765F84FF4EE
:10726000807102A8FBF792F8059B23B14FF40071DF
:1072700002A8FBF78BF820B203F0B4FA064660B11F
:107280005349544808F0A6FE0A222146514808F006
:107290000AFF504808F0AEFED2E70121204609F06F
:1072A00083FE3146204609F0A7FE5946284608F0DD
:1072B00091FE21460A22284608F0F5FE4649284656
:1072C00008F088FE4549284608F084FEB8E701909A
:1072D0000121204609F068FE20B203F083FA019BE9
:1072E00020B10021204609F087FEA9E7D6B113F1AD
:1072F000FF3618BF01263146204609F07DFE384989
:10730000284608F067FE0A222146284608F0CBFEF0
:107310003449284608F05EFE0A223146284608F025
:10732000C2FECFE7013B5E425E41E4E7DB68CAF89C
:10733000003026482C4C08F05DFEFFF79DFEFFF75D
:1073400047FB2A4B2A4801221A7004F0D9FA20B1CF
:10735000274804F097FB0423237094F90030072B8F
:1073600004BF042323703B78013B5BB23B700FB03A
:10737000BDE8F08FDB68FFDE380400206D030020DD
:10738000AD850100BC030020DC0300206803002061
:10739000BD8501007807002028900100A00400208E
:1073A000B07D0100D8030020C3850100E403002064
:1073B000C885010064030020DC8501002C04002046
:1073C00030040020DF850100340400207003002019
:1073D000EF8501008C030020078601000C86010068
:1073E000BB8101007F7E0100E00300206C030020D0
:1073F000A4030020FF850100F0B5464C267876B244
:1074000089B02746002E40F0818023784249434DC1
:10741000434801335BB2237008F0DCFD404808F0BC
:10742000E9FD722201212846F9F772FE2846F9F794
:10743000F1FD7B2846D13B493B4808F0CBFD3A485B
:1074400008F0D8FD394B049330464FF0FF330793D3
:1074500005960695FEF78EFC04A93548354E07F0D3
:10746000D3F930602846F9F7FFFD3568BDB93249D8
:10747000324808F0AFFD314808F0BCFD304901A8A2
:1074800009F07EFA01A92F48F9F778FC01A809F064
:1074900032FA2378013B5BB22370002010E02A49C6
:1074A0001F4808F097FD1E4808F0A4FD2378013B13
:1074B0005BB22370FFF712FE2248F9F725FD012089
:1074C00009B0F0BD2846F9F788FD80B12846F9F7E4
:1074D000BFFD1B4904A809F053FA04A91948F9F79C
:1074E0004DFC04A809F007FA1648F9F7CBFC0B4845
:1074F000F9F7BAFD15490A4808F06CFD084808F08C
:1075000079FD3B78013B5BB23B70C6E74FF0FF3043
:10751000D6E700BF6D030020458C01005C0400200D
:10752000BC030020608C010070030020A89B0100B8
:1075300078070020380400206E8C01008C030020A6
:10754000CA9B0100440400207A8C01008D8C01004C
:107550002DE9F041C0B000211C2214A813910BF0BA
:10756000A8FE202213A9A248F9F72CF978B9202205
:10757000A04913A80CF071FE9F49A04808F02AFD0D
:1075800013A99E4808F02FFD9C4808F033FD984D44
:107590006A7D2B7C04922A7D0392EA7C0292AA7C6B
:1075A00001926A7C00924021954A1BA80CF01CFDB8
:1075B0009449924808F00EFD13A9904808F013FD75
:1075C0001BA98E4808F00FFD8C4808F013FD4FF4FE
:1075D0007A730022CDE90F238B4A0E922BAC08223E
:1075E0008DF84820ADF84A3013AA50230EA9204642
:1075F00006F05AFA4FF47A63844985483B9308F0C1
:10760000E9FC02F0BDFD0A220146814808F057FD61
:107610007F4808F0EFFC204606F075FA1BA92046CB
:1076200006F098FB7B4906460AA809F0A9F9294605
:1076300007A8F9F75FFB079A0A99204606F068FA4F
:1076400007A809F058F90AA809F055F9204606F0EC
:107650007EFB002E40F0C580204606F089FBDFF857
:10766000FC810646204606F0F5FC074600B321469D
:1076700007A806F0F3FB41460AA809F081F90AA918
:1076800007A809F026FA07460AA809F034F907A85E
:1076900009F031F9002FE5D021460AA806F0F8FBE1
:1076A0000AA92846F9F76AFB0AA809F024F9D9E7DC
:1076B0005949524808F08EFC0A2231464F4808F0DA
:1076C000F2FC4E4808F096FCC82E7ED1534B54492C
:1076D0000A934F480B974FF0FF330D930C9408F02B
:1076E00079FC02F04DFD0A220146494808F0E7FC0A
:1076F000474808F07FFC0120FEF73CFBA0B9494950
:10770000494808F067FC484808F074FC204606F039
:10771000EFF94FF4FA76454B2B933DA809F0EBF8BF
:10772000304640B0BDE8F08141493948414D08F04C
:1077300051FC374808F05EFC3949354808F04AFCEE
:1077400002F01EFD0A220146314808F0B8FC30481C
:1077500008F050FC0AA9384807F056F8286020467F
:1077600006F0C6F92C6884B934492F4808F032FC79
:10777000334907A809F004F907A91D48F9F7FEFAEB
:1077800007A809F0B8F82646C5E72E49204808F0B2
:1077900021FC02F0F5FC0A2201461D4808F08FFC8E
:1077A0001B4808F027FCFFF799FC2749134808F00D
:1077B00011FC264B1B78002BADD00D48F9F711FAC0
:1077C0000028A8D0FEF74AFAA5E7B6F5987F0CBFC7
:1077D0001F492049144808F0FDFB204606F088F9AF
:1077E00099E71D49104808F0F5FB4FF0FF3692E786
:1077F000440400202B930100BC8A0100BC0300203C
:10780000DA8A0100098B0100089A01001D8B010032
:1078100070030020338B0100468B0100A89B010000
:107820009A8B0100598B01008C030020149B0100EE
:10783000658B010038040020780700207B8B010055
:10784000CA9B0100928B0100A08B01006C030020F9
:10785000A78B0100BB8B0100D58B0100418B010080
:107860002DE9F0433C4C23688DB0002B70D03B4D8C
:107870002E6809F0ABF9002301464FF47A723046C6
:1078800002F08CFD074610B109F0A0F92860344DD4
:10789000DFF8D8902B7801335BB22B702368DE6859
:1078A0007BB2002B14BF4FF004084FF0020822688F
:1078B000FAB1F6B1337C03F00F03052BF8D1314652
:1078C000484607F06AF80128F1D92268314668462F
:1078D000FAF75AFF6846FAF7CBFE18B141466846F8
:1078E000FCF7ACFD09F0C8F968467668FAF704FDC4
:1078F000DDE72B78013B5BB22B701A4B93F900301C
:10790000052B25D027B3184F00263D463968F9B11D
:10791000F6B90B7C03F00F03052B0DD122686846E6
:10792000FAF732FF01216846FCF788FD061C68461D
:1079300018BF0126FAF7E0FC2B684BB109F09CF95F
:107940002B685B682B60002BE0D12368DB682B6021
:107950000DB0BDE8F08300BFDC03002094040020DC
:107960006D030020E003002034040020780700208D
:10797000F8B580EAE074A4EBE074054620B20E4648
:1079800002F030FF074668B11549164808F022FB9F
:107990000A222146134808F086FB1248BDE8F84049
:1079A00008F028BB0121204609F0FEFA022E09D179
:1079B0003946204609F020FB0B490C4808F00AFB29
:1079C0000A48EBE736B9E943C90F204609F014FB32
:1079D0000749F2E7E90F204609F00EFB0549ECE7FD
:1079E0003D8601008C0300204B86010070030020BF
:1079F0009F940100B09401002DE9F04F2DED028B12
:107A0000874C95B0256809F0E1F80023014647F25C
:107A10003052284602F0C2FC002800F0FC8009F039
:107A2000D5F82060FFF726F97E497F487F4C804DCE
:107A300008F0D0FA02F0A4FB0A2201467A4808F0C6
:107A40003EFB7C49784808F0C5FA217876480A223E
:107A500049B208F028FB7849734808F0BBFA774B25
:107A6000714819680A2208F02AFB6F4808F0C2FA28
:107A70002A68002A00F0CF802378DFF8F8910133DC
:107A80005BB22370D468002C00F0C080237C03F02C
:107A90000F03052B13D100222146484606F087FF2D
:107AA0004369052B0BD12A68214608A8FAF76CFE1A
:107AB00008A8FAF7DDFD20B908A8FAF71DFC6468EC
:107AC000E1E708A906A8FDF7EFF908A8FAF78AFD8B
:107AD0000021074608A8FAF7B1FC064606A8FCF7FD
:107AE00097FF08EE900A08A8FAF710FC3BB207EEE1
:107AF000903A9FED537AF8EEE77A834687EE878ACD
:107B000008A8FCF793FB4F498246474808F062FA01
:107B10004FF0020818EE900A0AF084FDCDF80080BC
:107B200002460B46CDE904013F4808F091FB464967
:107B30003D4808F04FFA18EE100A0AF073FDCDF830
:107B4000008002460B46CDE90201374808F080FB71
:107B50003E49354808F03EFA59460A22324808F0B4
:107B6000A2FA5FEA174B4CD0082002F01FFE4FF636
:107B7000FF7381B240F62712584602F00FFCA8B1FD
:107B80002168334808F02FFA3249314808F022FAC8
:107B900022683149314807F0ADFCB9B208A8FAF7BC
:107BA00039FD41463046FFF7E3FE85E7DFED2C7AED
:107BB000B4EEE78AF1EE10FA04DD2268294927487D
:107BC00007F098FCBAF1000F01D10121EAE7002289
:107BD000254BDDE904010AF0C5FBDDE902230BF0CA
:107BE00009F808B10021DDE7F4EEC88AF1EE10FAD9
:107BF000EBD91E490C4808F0EDF90B4808F0FAF9EA
:107C00005AE71B49084808F0E5F955E7074A137891
:107C1000013B5BB2137015B0BDEC028BBDE8F08F79
:107C20009C04002055800100700300206D0300209B
:107C3000DC030020598501006185010084040020D7
:107C40000000C842698501006F850100E0800100E5
:107C50008C0300207585010085850100E803002064
:107C600000001842918501000000F03F9E85010050
:107C70007B850100780700202DE9F3470024344D6F
:107C800000942246214623463248334FDFF808A1AC
:107C900008F058F928464FF47A76304B6C60AE60A5
:107CA00040F8143B4FF0080808F044F985F82080AC
:107CB00029462B4D0122384608F072F84FF0010991
:107CC00000943B4629460722264802F0A1F83B468D
:107CD0002946CDF800900322234802F099F8009439
:107CE0003B460622214F22482946224D02F090F8B9
:107CF0004FF48053C5E901462B612C751E4BEC8275
:107D00001E492B60381DC5E9064485F8204008F05F
:107D100037FE3D601A4D1B495246384609F02CFA91
:107D2000C5E90146184C194B19482B60494685F89E
:107D300010806E8202F020F82946204607F01EFDD2
:107D400014495246204602B0BDE8F04709F014BA83
:107D5000C80400204C030020A4040020649A010001
:107D6000E0070020700300208C0300204404002062
:107D7000BC0300205C040020C07D0100CA9B010000
:107D8000A4030020F7590000E8030020089A01002E
:107D90003C040020D1ED0000000000202DE9F04758
:107DA0000024C8B03C22214609A808940BF081FAAF
:107DB0007C22214629A828940BF07BFA2346012235
:107DC000402108A802F056FAAF49B04EB04F08A8BB
:107DD0000CF0CBF97F22AF4928A80CF03EFA012322
:107DE00028AA08A9AC4807F09AFB234601224021A3
:107DF00008A802F03FFAA94908A80CF0B6F97F22BA
:107E0000A74928A80CF029FAA64928A80CF0ADF932
:107E1000012328AA08A9A04807F081FB23460122D4
:107E2000402108A802F026FA9F4908A80CF09DF905
:107E30007F229E4928A80CF010FA012328AA08A93D
:107E4000954807F06CFB23460122402108A802F068
:107E500011FA974908A80CF088F97F22954928A8BB
:107E60000CF0FBF9012328AA08A98B4807F057FB5F
:107E700033783D6801335BB23370002D00F03B81F5
:107E80008D4BDFF86092B3F80080ADF800801E22C1
:107E900021460DF102000BF00CFA3E2221460DF1B5
:107EA0006200ADF86080DFF840A2DFF840820BF09E
:107EB00000FAED683B68002B00F0AE80002D00F06A
:107EC000AB802B7C03F00F03052B40F08E802946FE
:107ED000404606F062FD002800F0878028680CF01C
:107EE0008EF90134044400222946404606F05FFD25
:107EF0004369112B12D8DFE803F07C87877C7C096B
:107F00007C7C7C7C11111111111111871F226B498E
:107F100068460CF0A2F900238DF86030002301229E
:107F2000402108A802F0A6F93F22296808A80CF011
:107F30006EF9494608A80CF018F9514608A80CF04B
:107F400014F901235E4A544808A907F04DFB0023A9
:107F50000122402108A802F08DF93F22296808A8D3
:107F60000CF055F9494608A80CF0FFF8554908A847
:107F70000CF0FBF80123544A474808A907F034FBEA
:107F800000230122402108A802F074F93F22296849
:107F900008A80CF03CF94D4908A80CF0E6F8514649
:107FA00008A80CF0E2F801236A4608A93A4807F04D
:107FB000B6FA9DF86030C3B100230122402108A821
:107FC00002F058F93F22296808A80CF020F93F492F
:107FD00008A80CF0CAF83B4908A80CF0C6F8012321
:107FE00018AA08A92C4807F09AFA08F045FE6D680F
:107FF00060E71F22364968460CF02FF935493F22C9
:1080000018A80CF02AF989E71F22334968460CF0BA
:1080100024F93F223149F3E700230122402108A837
:1080200002F028F92E49DFF8C4901B4D08A80CF087
:108030009CF80123621E08A9174807F0EAFA3B687A
:10804000DC683B68002B53D0002C51D0237C03F01C
:108050000F03052B14D12146484606F09EFC78B14B
:10806000D4F8008040460CF0CAF841460246284643
:1080700006F09FFE63681BB12C21284606F08CFE9B
:1080800008F0FAFD6468DCE79C9301006D030020B2
:10809000DC03002096930100E803002076930100A2
:1080A000D5930100C2930100A39301001593010031
:1080B000889301000F930100FC840100829301006A
:1080C00071930100AA93010037930100D386010048
:1080D00069930100259301007C93010065930100E1
:1080E0008F930100CD860100FC92010078070020EB
:1080F000044806F046FF3378013B5BB2337048B06A
:10810000BDE8F087E803002030B59F4C94F90030BB
:10811000113393B0242B35D8DFE813F0A301940179
:1081200034003400340034000301F3003400340020
:1081300034003400340034003400340034002500AE
:10814000510054006400A100BE00E300340034007C
:10815000340034003400130120016F012F0134007A
:10816000340034006001894B89481B78002B14BF10
:108170000921012101F001FE03F0D0FA022801D00B
:10818000FEF704FB94F90030012B40F38481814B0E
:108190001B78002B40F0748103F0CAFA054603F007
:1081A000BDFA022800F06E81013D042D00F27381BA
:1081B000DFE815F075017701850187016801022369
:1081C0002370DFE7744D2B7853B9FEF747F87349F6
:1081D000734807F0FFFE724807F00CFF01232B7075
:1081E0000323EDE7694D6A482B78002B14BF0B2160
:1081F000032101F0C2FD6B4B1B78002B40F0638123
:108200006948F8F728FDE0B1684B1B78BBB9FFF768
:108210009FF9C82808D02B7843B16549654807F015
:10822000D9FE644807F0E6FE0423C9E701A803F07D
:10823000C3FA029B002B00F0DE800F23C0E75E49EB
:10824000ECE72B784BB104235C495A48237007F0C4
:10825000C1FE584807F0CEFE94E70F23F4E74B4BDE
:108260004B481B78002B14BF0B21032101F085FD27
:10827000534B196841B953494E4807F0ABFE4D487E
:1082800007F0B8FE07239BE74F4806F086FB01285E
:10829000F1D9FEF7B9F875E74C4B1D6808F096FC6C
:1082A000002301464FF4FA52284602F077F80028DE
:1082B0003FF468AF00230322412101A801F0DAFF57
:1082C000434901A80BF051FF01A9424807F007FA02
:1082D000FFF764FD062340493648237007F07AFE15
:1082E00050E72A4B2A481B78002B14BF0A21022191
:1082F00001F043FD374806F0B5FE00287FF442AF99
:1083000092E708F063FC314B1860F52323701F4B94
:108310001F481B78002B14BF0921012101F02DFDFE
:1083200030E72A4B1D6808F051FC0023014641F25A
:108330008832284602F032F800283FF423AF0023A9
:108340003EE7244806F08EFE10B1224806F057FEA4
:1083500008F03CFC1D4B18600D2331E71B4B1D68DA
:1083600008F034FC0023014642F21072284602F065
:1083700015F800287FF458AF04E708F027FC134BEA
:1083800018600E231CE700BFE00300206C030020F0
:108390003C04002048030020D40300205990010031
:1083A000700300206D030020440400206E030020B1
:1083B00063900100BC0300208A9001009A900100A4
:1083C000E4030020D49001007807002090040020EE
:1083D00006900100E8030020E79001003C4B1D6877
:1083E00008F0F4FB002301463A4A284601F0D6FF84
:1083F00000283FF4C7AEF623E2E6FEF7FDFFD0B15A
:1084000001283FF411AF01307FF4BCAE304B1D6842
:1084100008F0DCFB0023014647F23052284601F009
:10842000BDFF00283FF4AEAE2B492C4807F0D2FD2B
:1084300001F0A4FFA6E61323237008F0C7FB244B2A
:1084400018609FE6264806F00DFE10B1244806F09D
:10845000D6FDFDF79BFF08F0B9FB1D4B1860EF231D
:10846000AEE6204D20482B78002B14BF0B210321B2
:1084700001F083FC1D4B1B783BBB12232370C6E627
:1084800000258CE61A49154807F0A4FD134807F0AB
:10849000B1FDF623237094F9000013B030BD1549E7
:1084A000F1E71549154807F095FD01A803F084F997
:1084B00001A801F0B9FE114807F09CFDEBE7104957
:1084C000E1E71049EEE70320E7E76FF01000E4E78B
:1084D00090040020C0D40100049101008C0300200E
:1084E000E80300206C0300203C0400206D03002002
:1084F000279101003091010044910100BC0300204C
:10850000619101007491010008B5184801F037FC31
:1085100008F0B2FB06F01CFCFFF7F6FD022802DDB6
:10852000134806F0C7FE08F0A7FB124B1B7823B1D7
:10853000114B1B680BB101F0FBFB104B1B6843B1E7
:108540000F4B93F90030052B01D0FFF789F908F0A4
:1085500093FBFFF751FA08F08FFB0220FEF794FC23
:1085600008F08AFBBDE80840FEF740BD3C0400204F
:10857000E8030020300400202C040020DC0300204D
:10858000E003002010B54FF4E1311B4808F03AF841
:108590001A48F8F71DF8044630BB1949164807F089
:1085A0002FFD21462046FDF7C7FB1448F8F792FB44
:1085B000144B18701148F8F795FB134B1870FEF721
:1085C000EDFBFEF76FFAFEF7C9FB142008F032FB53
:1085D0000E490F4807F0B5F84FF4FA7008F02AFB7F
:1085E000BDE81040FEF708BF0A490B4807F0F2FC4F
:1085F000094807F0FFFCD8E7E0070020440400200A
:10860000308501000500002006000020415F0000C9
:10861000E8030020458501007003002007B5002312
:1086200000931A461946034807F08CFC03B05DF826
:1086300004FB00BFF00400200320704770470000D7
:1086400073B56E460546304686E80600FCF7DAFB51
:1086500004463046FCF770F910B1002C08BF012425
:108660004FF480416868F9F791FE012C1BD0022C71
:1086700004D0FCB91C491D4807F0ACFC3046FCF79F
:108680006CF970B36868F9F7ADFF18B9012420469A
:1086900002B070BD00206C6802F088F801462046E8
:1086A000F9F7B8FFF2E73046FCF7F6FA01280AD0EE
:1086B000022808D00E490D4807F08CFC0B4807F043
:1086C00099FC0024E3E76868F9F78CFF0028DDD007
:1086D00000206D6802F06AF801462846F9F79AFF13
:1086E000D5E70446D3E700BFDF9301007003002005
:1086F000F793010010B5044608F000FB204610BDBA
:1087000010B504461649174807F084FC002160683C
:10871000F9F780FF236820469B690021984794F968
:10872000080002F05FF840B10F49104807F052FC12
:108730000E4807F05FFC002010BD94F9090002F01C
:1087400051F80028F0D1A17C94F9080008F054FCFD
:1087500094F90900A17C08F04FFC0120ECE700BF70
:1087600020940100700300202F9401008C0300204E
:1087700001292DE9FF41044600F089804FF4804132
:108780004068F9F7EBFD002800F081804FF40041CC
:108790006068F9F7E3FD60B9764D95F90030002B7C
:1087A00075D04FF400416068F9F7F0FD2B78013B7C
:1087B0002B7094F9080002F015F8002867D194F99D
:1087C000090002F00FF80546002860D16068F9F74B
:1087D00009FF2A462946074602A8FBF72FFF4FF458
:1087E0000072616802A8FCF71BFB294602A8FCF78F
:1087F000E7F906466068F9F789FD022801D00528E7
:1088000000D1002694F90A00A0F10E03DBB2072B79
:1088100000F29C804FF0FF0808F0D0FAE289218A2C
:10882000CDF80080002308F05CF8051EC0F28A80B5
:10883000454500F38980002F40F08B80751B15F1B2
:108840000A0F55DA94F90900A17C08F0D5FB60689D
:10885000F9F7C8FE30B9666801F0A8FF0146304656
:10886000F9F7D8FEA37C6842002B3CD00021009190
:10887000FF23192208F035F8FF280146A8BFFF2181
:10888000462994F90800B8BF462108F03BFB0020B8
:1088900004B0BDE8F0813849384807F09BFB374801
:1088A00007F0A8FB3649354807F0B4FBA17C94F9E2
:1088B000080008F0A1FBA17C94F9090008F09CFBDA
:1088C00000216068F9F7A6FE4FF480416068F9F76F
:1088D0009DFD4FF400416068F9F798FD254A137833
:1088E00001331370D3E7FF22009219461922C1E722
:1088F0000A2DD7DD94F90800A17C08F07DFB6068A3
:10890000F9F770FE30B9666801F050FF0146304655
:10891000F9F780FEA37C83B100210091FF2333226D
:10892000284607F0DEFFFF280146A8BFFF214629A1
:10893000B8BF462194F90900A7E7FF220092194623
:108940003322EDE7002576E7454674E77FB14FF027
:10895000FF3508F03BF900230146B4F90C203846F6
:1089600001F01CFD002896D16B1C7FF467AFA6F1C7
:108970007F0564E7040000200394010070030020D9
:1089800012940100002110B5044681744068F9F783
:1089900055FD43B2002BBBBF40422072237201231E
:1089A000B8BFA374237A6068013B182B84BF2023CF
:1089B00023720121F9F742FD43B2002BBBBF4042B5
:1089C000607263720123B8BFA374637A6068013B6D
:1089D000182B84BF212363720221F9F72FFDC3B244
:1089E000192B8ABF0023A072A37203216068F9F7D4
:1089F00025FD80B2431EB3F5806F26BF0023E381BF
:108A0000E08104216068F9F719FD80B2B0F5806F4C
:108A10008ABF4FF480632082238205216068F9F7C2
:108A20000DFD00B20028D6BF42F21073A081A381D1
:108A300010BD000038B50446F7F7D7FC2046FFF715
:108A4000A1FF2549254807F0E5FA94F9080001F04F
:108A5000C9FE40B12249234807F0BCFA214807F07B
:108A6000C9FA002038BD94F9090001F0BBFE0546A3
:108A70000028EFD1012194F9080008F095FA0121AE
:108A800094F9090008F090FAA17C94F9080008F024
:108A9000B3FAA17C94F9090008F0AEFA294694F9DA
:108AA0000A0008F081FA29466068F9F7B3FD4FF42F
:108AB00080416068F9F7AAFC4FF400416068F9F75B
:108AC000A5FC236820469B6902219847064B022299
:108AD0001A700120C6E700BF3C940100700300201B
:108AE0002F9401008C0300200400002007B5002310
:108AF00000931A461946034807F024FA03B05DF8BC
:108B000004FB00BFF80400200020704703207047DA
:108B1000704700002DE9F0410646F7F766FCB4689F
:108B2000002C41D0E468254F254DDFF8A88064B3C0
:108B3000236843B31B7833B33A462146284605F0F1
:108B400040FF30B94FF0FF333A462146284605F042
:108B500080FF42462146284605F033FF30B94FF0EA
:108B6000FF3342462146284605F073FF154A214649
:108B7000284605F026FF30B94FF0FF33114A214651
:108B8000284605F066FF6468D1E70F490F4807F0F3
:108B900021FA0E4807F02EFA336830469B6902210D
:108BA00098470120BDE8F0810949084807F012FA0A
:108BB000064807F01FFA2046F4E700BF449801007A
:108BC000780700200E9401000C950100700300202E
:108BD00017950100FF93010038B5084D0849044678
:108BE000284607F0F7F9284607F004FA23682046DC
:108BF0009B6900219847012038BD00BF7003002009
:108C0000FE9401002DE9F04F93B00AAC8046204657
:108C100084E806000893FCF73FF80B2800F0448234
:108C20002046FCF739F80A2800F03E822046FCF77F
:108C3000E9F882462046FBF77FFE20B1BAF1000F2B
:108C400008BF4FF0010A2046FBF776FE90B12046A0
:108C5000FCF7D8F807280DD12046FCF71DF811289D
:108C600068D0122868D0102804D1FF22214610A80D
:108C7000FCF721F8D8F80830002B00F01582002707
:108C8000CDE90477DC68B946BB46002C00F0DE80F5
:108C9000AF4AB048214605F094FEAF4A214605464A
:108CA000AC4805F08EFEAD4A06462146A94805F0BF
:108CB00088FE0790002D00F08B80002E00F0888049
:108CC0002B7C03F00F03022B40F08280337C03F0F7
:108CD0000F03022B7CD1A24A9E48214605F071FE6B
:108CE00043690693089B002B5FD0194620680BF060
:108CF00058FA002859D10AA8FBF71EFE08BBBAF1A2
:108D0000070F6FD00AAA10460992FBF726FE099AB0
:108D100000283DD0104600210992FBF751FF686101
:108D2000FDF7ECF8099A002832D0236800934FF43D
:108D3000007328E0802299E70A212046FBF702FF12
:108D400098E70AA8FBF7A8FF70610AA8FBF7A4FF41
:108D500001283FD0022843D0FDF7D0F858B17369FD
:108D6000012B08D16B69132B05DC1E226A610AA94D
:108D700010A8FBF7A0FFFDF7C1F848B123680093E6
:108D80000AAA4FF4407306CAD8F80400F9F7ECFEBB
:108D9000079B53B10023CDE9013300930AAB0CCB01
:108DA0004FF0FF31079801F013FB7369022B0DD0D0
:108DB00001330BD06B69069ABB4202FB03F2C2BFC0
:108DC0001F46069B04929344C8BF0593069B994493
:108DD00064685AE76A690AA910A8FBF76CFFBBE749
:108DE0000022F8E70AA8FBF7B8FD00288AD00AA8F5
:108DF000FBF7EEFD7369A8B1022B01D001330CD152
:108E00005849594807F0EFF8574807F0F3F801229E
:108E100072610AA910A8FBF7EEFF0AA8FBF7D8FDBC
:108E20006861A8E7022B0ED001330CD04F494E48A1
:108E300007F0D9F84C4807F0DDF8022272610AA960
:108E400010A8FBF7D8FF00236B6194E7B9F1000F7E
:108E500000F02A81464944489BFBF9F507F0BAF82F
:108E60000A224946404807F01EF942493E4807F0A9
:108E7000B1F8FF260A229BFBF6F13B4807F013F9F5
:108E80003D49394807F0A6F80A222946364807F036
:108E90000AF93A49344807F09DF8049B324893FB9D
:108EA000F6F10A2207F0FFF835492F4807F092F84B
:108EB0000A2205992C4807F0F6F832492A4807F0AB
:108EC00089F8294807F096F810AE0EAF2E4AD8F868
:108ED000081020481DB305F074FD22468146214646
:108EE0003846FBF7ABFB2A46394630460CADFBF75C
:108EF000E2FE012231462846FBF77DFFCDE9014421
:108F0000009495E80C004FF0FF31484601F060FAFC
:108F1000D8F80830D3BB012013B0BDE8F08F05F0BE
:108F200050FD2246054621463046FBF787FB224688
:108F300031463846FBF7BFFECDE90144009497E87F
:108F40000C004FF0FF31284601F042FAE3E700BF82
:108F50004498010078070020FF9301008C940100E1
:108F6000909401009294010070030020A3940100EA
:108F7000B5940100C4940100CF940100D69401007F
:108F8000E0940100E7940100CA9B0100DD68DFF86E
:108F90003881DFF838B1002DBDD0444A294640461B
:108FA00005F00FFD5A4644692946404605F009FD83
:108FB0003F4A81462946404605F003FD3D4A824628
:108FC0002946404605F0FDFCB9F1000F66D0BAF124
:108FD000000F63D0002861D099F8102002F00F0232
:108FE000022A5BD19AF8102002F00F02022A55D112
:108FF000027C02F00F02022A50D1002C4ED04269AE
:10900000022A4DD001324BD0049B002B4AD0DAF813
:1090100014302949294803FB04FA059BCAEB0A22AC
:1090200092FBF4F45C43049B94FBF3F406F0D2FF50
:109030002968224806F0D7FF2149204806F0CAFFD8
:109040000A22FF211D489AFBF1F107F02CF81D4977
:109050001A4806F0BFFF0A222146184807F001F817
:10906000164806F0C7FFD9F81430A34216D00022E4
:1090700011463846FBF7E2FA224639463046FBF7FE
:109080001AFE0023CDE90133009396E80C004FF05F
:10909000FF31284601F09CF9C9F814406D687AE761
:1090A0000024E0E7049CDEE7002035E7909401000F
:1090B00044980100FF930100EB940100700300202D
:1090C000F2940100F8940100780700200E9401004A
:1090D00010B5044607F012FE204610BD0023836041
:1090E00043683BB19B682BB11A7C02F00F02062A41
:1090F00008BF83607047000007B5002300931A463D
:109100001946034806F01EFF03B05DF804FB00BFDC
:109110000005002043687BB1B0F90A20042A05D07D
:10912000052A05D0032A05D1022070470120704787
:1091300011207047187D704718467047704700002F
:1091400038B50446F7F751F92849294806F042FF97
:109150000A22B4F90810264806F0A5FF254924483C
:1091600006F038FF636822485B68196806F03BFF29
:1091700021491F4806F02EFF1D4806F03BFF60689E
:1091800088B3B4F908307BBB236820469B6B9847B3
:109190000128054605D002280AD00121B4F90800AB
:1091A00019E003212046F7F7EDF9294607F0FCFE08
:1091B00000212046F7F7E6F9012107F0F5FE01212D
:1091C0002046F7F7DFF9012107F0EEFE02212046E5
:1091D000F7F7D8F9012107F0E7FE236820469B69DD
:1091E00002219847012038BD0020FCE7709501005E
:1091F00070030020A07E01001195010010B5044607
:109200002449254806F0E6FE0A22B4F9081022484F
:1092100006F049FF2149204806F0DCFE63681E483D
:109220005B68196806F0DFFE1D491B4806F0D2FE98
:10923000194806F0DFFE236820469B6B98470128FB
:1092400005D002280AD00021B4F9080019E0032152
:109250002046F7F797F9002107F0A6FE00212046E7
:10926000F7F790F9002107F09FFE01212046F7F75C
:1092700089F9002107F098FE02212046F7F782F9CC
:10928000002107F091FE236820469B690021984742
:10929000012010BD7095010070030020A07E010028
:1092A000C79101002DE9F041044688B040689DF85F
:1092B00038309DF83C5002AF87E80600002800F0E7
:1092C000A780B4F90820002A00F0A180002B00F04C
:1092D000A2800021F9F7B2F8236880469B6B2046F4
:1092E000984706B2022E19D0032E19D0012E0CBFBA
:1092F00005210121002204A8FBF7A0F94FF0FF335C
:10930000009397E80C0004A906A8FBF7F1FF012ED3
:1093100041D0022E27D1002D52D14CE00421E9E7A3
:109320001DB34FEAD8713846B4F90860FBF748FC22
:1093300001460546304607F0E5FD3849384806F055
:1093400049FE0A22B4F90810354806F0ACFE35494A
:10935000334806F03FFE0A222946314806F0A3FEB4
:109360002F4806F047FE012052E0B4F9080001F052
:1093700039FA0028D5D029492B4806F02BFE0A22BD
:10938000B4F90810284806F08EFE2849264806F051
:1093900021FE2548E5E703212046F7F7F3F80646C6
:1093A0002DB19DF81710304607F0ACFDB3E701F082
:1093B00019FA0028F5D0B4F9080001F013FA28B919
:1093C0009DF81610B4F9080007F09CFD0121204615
:1093D000F7F7D8F8064685B19DF81510304607F026
:1093E00091FD20460221F7F7CDF8044655B19DF8CE
:1093F0001410204607F086FDB5E701F0F3F90028C8
:10940000EAD0EEE701F0EEF90028F0D0ABE7104625
:1094100008B0BDE8F0811846FAE700BFBB81010043
:10942000700300207F7E01008C0300207A950100EC
:1094300010B5044607F062FC204610BD07B50023B6
:1094400000931A461946034806F07CFD03B05DF808
:1094500004FB00BF08050020032070477047000090
:1094600038B50446F6F7C1FF2249234806F0B2FD9D
:109470000A22B4F90810204806F015FE1F491E48BC
:1094800006F0A8FD1C4806F0B5FDB4F9080001F08F
:10949000A9F9054640B11A491A4806F09BFD19483A
:1094A00006F0A8FD002038BD0121B4F9080007F03E
:1094B0007BFDB4F90800A17A07F09EFD606810B149
:1094C0002946F9F7A7F8236820469B6902219847A7
:1094D000606808B90120E6E7FAF7A8FE0028F9DD80
:1094E0000020646801F062F901462046F9F792F81D
:1094F000F0E700BF069601007003002011950100FF
:109500002F9401008C03002038B50F4D0F490446FD
:10951000284606F05FFD0A22B4F90810284606F036
:10952000C2FD0B49284606F055FD284606F062FDAF
:10953000B4F90800002107F037FD236820469B6935
:1095400000219847012038BD7003002006960100D5
:10955000C791010010B5044607F0D0FB204610BDAE
:10956000002110B5044681724068F0B1F8F766FF3B
:1095700003B2002BBBBF4042208123810123B8BF2F
:10958000A37223896068013B182B84BF20232381A9
:109590000121F8F773FF09F045F80022054B09F0A7
:1095A00099F809F06FFB08B1E06010BD41F2883313
:1095B000E360FAE700408F4030B5044687B00023EF
:1095C0002F22CDE90023ADF80830B0F90800A37AC6
:1095D0000D4671B383F0010107F00EFDE368B3F5AA
:1095E0007A7F57D33149324806F0F4FC0A22B4F9A5
:1095F00008102F4806F057FD2E492D4806F0EAFCCA
:109600000A2229462A4806F04EFD294806F0F2FCB7
:10961000294968460AF0A9FD6068F8F777FE002D31
:109620003ED0142807D0152836D00F2836D123492C
:1096300002E01946D0E7224903A80AF0BCFD2149FF
:109640001B4806F0C7FC63685968236809685D6AAF
:1096500003AA6B462046A8470A220146144806F092
:1096600022FD1949124806F0B5FC636810485B6892
:10967000196806F0B8FC69460D4806F0B4FC1349B9
:109680000B4806F0A7FC03A9094806F0ACFC084803
:1096900006F0B0FC07B030BD0D49CDE70D49CBE772
:1096A00002280CBF0C490D49C6E700BF1296010005
:1096B000700300206A820100DD950100D095010051
:1096C000EB9501001796010006800100239601002A
:1096D000E4950100F3950100D4950100D8950100AF
:1096E0000129F7B5044644D04368002B41D000223D
:1096F00011466846FAF7A2FF4FF4007261686846A7
:10970000FBF78EFB00216846FBF75AFA05466846D0
:10971000FBF7C2FA6068F8F765FF064607F056FAED
:10972000E268FF216A430023B2FBF1F201463046B2
:1097300000F034FE0746E6B107F048FA0023014680
:10974000E268304600F02AFE064620B30020666834
:1097500001F02CF801463046F8F75CFF4DB1207A55
:1097600001F02EF8A37A834203D101212046FFF7AE
:1097700023FF002003B0F0BD9FB131462046FFF724
:109780001BFF6068FAF752FD01460028F1D16068BE
:10979000F8F740FFEDE7207A01F012F8A37A834250
:1097A000EAD1002DE5D0207A01F00AF8A37A8342AD
:1097B000DFD1002FDDD1D8E7F7B56E4686E8060089
:1097C0000446454945489DF820501F4606F002FCD6
:1097D0003046FBF713FD37B1414938460AF0E1FC4A
:1097E00008B9002051E06368002BFAD0B4F90800F2
:1097F00000F0F8FF0028F4D13046FBF79DF8002870
:1098000045D13046FBF7FEFA012840D010D302289C
:109810000DD004463349314806F0DCFB0A222146CC
:109820002E4806F040FC2D4806F0E4FBD9E7D5B100
:1098300000213046FBF7C4F9054658B16068F8F7D7
:10984000D1FE08BB646800F0B1FF01462046F8F77E
:10985000E1FE19E001466068F8F7DCFE2946204683
:10986000FFF7AAFE10E06068F8F750FD15280BD846
:10987000012303FA00F01C4B184205D0294630465C
:10988000FBF79EF90028D9D1012003B0F0BD304686
:10989000FBF702FA15280DD80125144F05FA00F040
:1098A0000740CBD1430705D539466068F8F7B2FECB
:1098B0003946D4E70E49094806F08CFB3046FBF7E1
:1098C000EBF90A220146054806F006FC034806F0BB
:1098D00091FB01249EE700BFFB950100700300206F
:1098E000DD9501000A7D01000240380002C0380009
:1098F000FD7C010007B5002300931A461946034872
:1099000006F020FB03B05DF804FB00BF100500204B
:1099100090B1C3687BB11A7C02F00F02042A01D116
:10992000586948B9D86838B1037C03F00F03042B99
:1099300001D14069704700207047000030B52DED1F
:10994000028B054689B008EE101A002852D0324B1F
:109950001B68002B4ED0FFF7DBFF30490446304830
:1099600006F038FB18EE100A08F05CFE02230246EF
:1099700000932B480B4606F06BFC2A49284806F05A
:1099800029FB2968264806F02EFB2749244806F0C3
:1099900021FBDFED267AB4EE678AF1EE10FA2DD0C6
:1099A000DFED237AB4EE678AF1EE10FA26D0B5EE39
:1099B000408AF1EE10FA21D01CB12146184806F079
:1099C00012FB174806F016FB06AC18EE101A04A896
:1099D000FAF741FE032204A92046FBF717FA0023F9
:1099E000CDE90133009394E80C004FF0FF31284695
:1099F00000F0EEFC09B0BDEC028B30BD002CF9D0BC
:109A00000C49074806F0E6FA2146054806F0EBFA4D
:109A1000034806F0EFFAEDE72C0400206C960100F5
:109A2000700300200B980100F99701000000FEC2AE
:109A30000000AA42719601002DE9F043284F3868D2
:109A400089B0002846D0274E3368002B45D001F05E
:109A500073F925492548DFF8A080DFF8A090234C52
:109A600006F0B8FA214806F0C5FA01A9386801F0F5
:109A7000F5FA00282DDD03AA082101A800F078FAE4
:109A8000002303AA31688DF81C30404604F099FF8A
:109A900049460546204606F09DFA03A9204606F0F1
:109AA000A2FA8DB12846FFF733FF05460028DCD027
:109AB0000F49204606F08EFA2946204606F093FA12
:109AC000204606F097FAD0E70A49204606F082FAC7
:109AD000F6E7012009B0BDE8F0831846FAE700BFB9
:109AE000240500202C0400208D970100BC030020D9
:109AF0006A820100A0970100780700206C9601009F
:109B0000FFF79ABF2DE9F3413E4C2368002B77D134
:109B10003D493E4806F05EFA3C4806F06BFA1420D8
:109B200007F0EAF8054601F0C1F83948256000F071
:109B300017FF206801F0D4F800284AD0354936488C
:109B400006F05EFA206801F011FA206801F0D4F8FE
:109B5000206801F04FFA002839D030492B4806F030
:109B60004FFA2F4E3068002847D02E4D2F687FB90E
:109B70001C2007F0C1F82168804601F0F3FA404646
:109B8000C5F8008001F0CEFB3946286801F008FCDA
:109B90003368DFF8A480DC681C4F336883B37CB380
:109BA0006946206800F01CFA50B34146384606F07A
:109BB00011FA2168384606F016FA384606F01AFA05
:109BC0000C226946286801F06AFB6468E5E71649DB
:109BD000C4E700F009FE206801F082F8054638B1BC
:109BE00012490D4806F0F6F90B4806F003FAB8E7FB
:109BF0000F49104806F004FA284602B0BDE8F0818B
:109C00000120FAE724050020CF9601007003002010
:109C10009C050020F5960100BC030020149701006C
:109C20002C0400202C050020289701003D970100FE
:109C30005A9701008C03002076970100034B0146E0
:109C4000186808B101F042B8704700BF2405002031
:109C500037B52D4C206801F03BF8022805D00428C8
:109C600011D0012818D129490EE02949294806F0C8
:109C7000B1F9284806F0BEF9206801F0BBF941F2BD
:109C8000883003B030BD2449224806F0A3F92148AA
:109C900006F0B0F900F0A8FD204D2B6813B1204B61
:109CA0001B683BB91F491B4806F094F9194806F098
:109CB000A1F9E4E71C4C22683AB91A7C02F00F02C1
:109CC000062A02D1DB6803B123601848FFF7B6FF0C
:109CD0002368A3B16946186800F082F978B19DF84D
:109CE0000030282B0BD16946286801F0E9FB0146BA
:109CF0002068FFF723FE6946286801F087FB236888
:109D00005B682360BBE700BF24050020AF9601001D
:109D1000829601008C030020969601002C050020FD
:109D20002C040020C196010020050020B96F00001E
:109D300038B5094C256806F049FF0023014641F279
:109D40008832284600F02AFB20B1FFF781FF06F099
:109D50003DFF206038BD00BF2805002007B5002367
:109D600000931A461946034806F0ECF803B05DF874
:109D700004FB00BF1805002070477047704770470C
:109D800007B5002300931A461946034806F0DAF88F
:109D900003B05DF804FB00BF30050020174B1B78B3
:109DA00070B504460D469BB1154B027A1B789A425A
:109DB0000ED8144A0A291368164616D1124A0021F1
:109DC000D154406910B1217A06F082F80023336043
:109DD000E06840B10D4B227A1B789A4203D80368A1
:109DE00029461B689847012070BD4E2BF0DC0D29D9
:109DF0001FBF591C1160044AD554E9E780040020B4
:109E000006000020900500204005002005000020ED
:109E100030B5002545604361034D9DF80C30056069
:109E2000C1600272037430BDB097010007B5002312
:109E300000931A461946034806F084F803B05DF80B
:109E400004FB00BF38050020D0E90423D05C704734
:109E50000368DB681847704700207047184B70B5DF
:109E60000E461968044679B10B7C03F00F03062BEC
:109E70000AD13246134804F0A4FD037C03F00F031B
:109E8000042B01D1406970BDB4F924506B1E9BB204
:109E90000C2B13D80C4930460AF083F970B90B49E2
:109EA0002F2305EB850584F826300622294404F18A
:109EB00027000AF0D2F904F12600E4E70020E2E7E7
:109EC000A004002078070020D498010087980100A2
:109ED0002DE9F041056A044625B1002303622846B6
:109EE000BDE8F081D0E90432995C242934D1991875
:109EF00049787B2930D1023213442E461A4613F892
:109F0000017B4FB37D2F0FD00136F7E7A2612269A5
:109F10003AB16369D25C12B10133636125E0226119
:109F2000DDE74FF0FF35DAE7B6B14FF0000882F811
:109F3000008061692269236802319B6911442046CF
:109F40009847D4E9043233441344C4E906089F70A7
:109F5000636903331E446661A269002AD7D0E369AE
:109F6000D25C002AD2D00133E3611546B7E7000086
:109F700070B5D0B1CAB14D1E0C4E441E13462844D4
:109F8000844203F102030CD014F8015F2D11755DBA
:109F900003F8025C257805F00F05755D03F8015C98
:109FA000EEE709B2002302F8113070BD6D98010090
:109FB000A0F16103052B02D85738C0B27047A0F159
:109FC0004103052B01D83738F7E73038C0B20928EC
:109FD00005D919B101230B7000207047084670475E
:109FE00037B500238DF80730F9B1E0B1851C4C1E60
:109FF00000F1120215F8020C0DF10701FFF7D8FF6E
:10A00000000104F8010F0DF1070115F8010CFFF72D
:10A01000CFFF23780235184395422070EAD19DF88E
:10A02000070080F0010003B030BD0846FBE738B5FB
:10A030000546D8B10468ACB124789CB1286803788F
:10A040003BB12D2B05D0303B092B02D901302860C4
:10A05000F4E708F0ACFE2C21044628680AF094F8D6
:10A0600010B92860204638BD0130FAE70446F9E708
:10A070002DE9F7430E46002206210746FAF7DEFADD
:10A08000002E55D03368002B52D01B78002B4FD0B8
:10A09000D6F8008098F800404CB32D2C6CD0303CA2
:10A0A000092C03D908F101033360F1E7414600248C
:10A0B00000220FFA82F9013211F80930303B092BE6
:10A0C000F7D92E2140460AF05FF818B3002211B2EA
:10A0D000431801325B78303B092BF8D94378A3F160
:10A0E0003002092A01D82F2B03D8002204E0A14610
:10A0F000E7E7392B88BF09220A2555438278A2F168
:10A100003003092B05D82F2A16D9392A88BF0923ED
:10A110001D4499B9404608F04AFE39460246684651
:10A12000FAF7DDFD2C2130680AF02EF810BB306004
:10A13000384603B0BDE8F0830023E9E70229404632
:10A140000EDCB9F1070F0BDC08F031FE642242434C
:10A1500004B16D422A4439466846FAF7E6FDE1E764
:10A1600008F01EFE08F0AEFD394602466846FAF7D2
:10A17000C2FDD7E70130DAE708F10101012497E7D2
:10A1800008B500200BF048F8ADEB000008BD7047A3
:10A1900030B5441E224612F8013F002BFBD11A466F
:10A1A0000A2514F8010F70B1032A14DC2E2806D1F9
:10A1B000FF2B10DC8818013203710023F1E73038DF
:10A1C00005FB0303EDE7FF2B04DC032A02DC11444B
:10A1D00001200B7130BD0020FCE700002DE9F341A8
:10A1E0000024DFF840800C700D461746061D0A2239
:10A1F00001A916F8010B08F0F3FF3A4601A9284619
:10A200000AF005F8032C04D03A464146284609F0E6
:10A21000FEFF0134A3B2042B1CB2E8D1284602B0E1
:10A22000BDE8F081BB9101002DE9F0410E4D0F4FCB
:10A23000DFF83C8006460024032C0ED033190A2296
:10A240001979284605F00DFF41462846013405F0EE
:10A25000C1FE042CF0D1BDE8F081F1790A22284634
:10A2600005F0FFFE3946F0E7BC030020A07E0100A8
:10A27000BB9101002DE9F047DFF8F0A0DAF80050BB
:10A2800004460E4617469946002D49D02B7C03F014
:10A290000F03062B43D12C4A2C48294604F091FB8E
:10A2A000022F804637D0032F37D1294ADAF8001021
:10A2B000264804F086FB0546B8F1000F30D098F828
:10A2C000103003F00F03042B2AD1D8F814103246B3
:10A2D000204609F0C2FF32461E49204609F097FF8A
:10A2E0000DB32B7C03F00F03042B1CD1696932469C
:10A2F000204609F08CFF32461649204609F087FFB8
:10A30000B9F1000F04D032464946204609F07FFFDC
:10A310002046BDE8F087104AC8E70025CCE70025B5
:10A3200032460E49D4E7022F0AD0032F05D0012F61
:10A33000E1D10B4B32461968DAE732460949D7E7D3
:10A3400032460949D4E700BF63980100780700202E
:10A350000E9401001B8B010068980100CD9801004C
:10A3600088030020819801007E980100A00400204D
:10A370000B460A220146184606F07FBC10B5054C74
:10A380000549204605F02FFE2046BDE8104005F0A7
:10A3900031BE00BF700300202E98010010B54AB1F5
:10A3A00002441BB1B2FBF3F403FB14228A4208D22D
:10A3B00088420AD9012010BD884294BF00200120A4
:10A3C000F9E78242F8D80020F5E78242F5E700007D
:10A3D0002DE9F04FA7B004AE0D4686E80C00DDE98C
:10A3E00030BA0446002800F0F180037C03F00F032C
:10A3F000062B1ED8DFE813F0E3001D001D001D0032
:10A40000DF0007001F00934FC4683B7801333B70A7
:10A4100064B1329BCDF800B0CDE901A3204696E8A7
:10A420000C002946FFF7D4FF6468F1E73B78013B55
:10A430003B7000200FE00146874A884804F0C1FACB
:10A44000814658B10023CDE90133009396E80C0012
:10A450002946FFF7BDFF27B0BDE8F08F804A7F484F
:10A46000214604F0AEFA7F4A214680467B4804F03C
:10A47000A8FA7D4A07462146784804F0A2FA1DB1A1
:10A48000012D7BD04D460EE0784A7448214604F0F9
:10A4900098FA8146764A7148214604F092FA0546B8
:10A4A000B9F1000F00D1A146002D08BF2546B8F133
:10A4B000000F00F08780002F08BF5746B9F1000F4A
:10A4C00000F0828099F8102002F00F02042A7BD15C
:10A4D000D9F81440002D7BD02B7C03F00F03042B04
:10A4E00076D1D5F814904FF0000AB8F1000F00F0C3
:10A4F000D380002C00F08E805E495F4805F06AFD35
:10A50000D8F814105C4805F06EFD5C495A4805F017
:10A5100061FD2146584805F066FD574805F06AFD83
:10A520003046FAF76BFE002F40F0288198F8103083
:10A5300003F00F03042B40F01F81514BD8F8141087
:10A540001A6816A8F8F756F916A8F8F791F888B11E
:10A55000FFF716FEB0F5966F054669DA49494A4895
:10A5600005F038FD0A222946474805F09CFD46487B
:10A5700005F040FD16A8F7F7BFFEFDE0434A374857
:10A58000214604F01EFA424A81462146334804F02F
:10A5900018FA0546B9F1000F40F0F480334A2F480D
:10A5A000214604F00EFA8146002D3FF473AF0028D7
:10A5B00008BFA1467BE700252F46A84673E7002584
:10A5C000A9462F46D84676E7002483E75746D84663
:10A5D0000023009310224FF4407306A93046FAF787
:10A5E000F9FC81463046FAF70DFC0FFA80FABAF111
:10A5F000000F7FF47AAF3046FAF79EF938B930464B
:10A60000FAF7ABF9002818BF4FF0020A6DE74FF0D8
:10A61000010A6AE71F49184805F0DCFCD8F8141055
:10A62000154805F0E0FC1549134805F0D3FC77E721
:10A630002CB10022214616A8F9F7FEFB9AE7012368
:10A6400000930194234696E8060016A8F8F734FD17
:10A6500090E700BF6D030020F07D01007807002027
:10A660004A7E01008C7E01004F7E0100DC970100D4
:10A67000E1970100F097010070030020F7970100B7
:10A68000DC030020159801008C030020E6970100F0
:10A69000EB970100FC970100002F6DD0B9F1000F7E
:10A6A0006AD03B7C03F00F03042B61D17B69ADF8CA
:10A6B0004CA000254FF47A72CDE90B52334A0A922E
:10A6C000CDE90E3516AA402329460AA8CDE9105532
:10A6D00012958DF84E5005F061FF26AB18442C49B9
:10A6E00000F8405C2B4805F075FC7969294805F0B5
:10A6F0007AFC2949274805F076FC16A9254805F07B
:10A7000072FC2649234805F065FC4946214805F0BE
:10A710006AFC204805F06EFC214804F0A3FC38B325
:10A72000204B93F900301BBB2F2116A809F02CFDFC
:10A7300028B97B690322402116A8FFF79BFD1A491F
:10A74000144805F047FC16A9124805F04CFC1349C3
:10A75000104805F03FFC49460E4805F044FC0D4802
:10A7600005F048FC01234A4616A90D4804F0D7FE1F
:10A77000B8F1000F7FF4DAAE01206CE6B9F1000FFA
:10A780008FD1D3E600287FF492AE83E6C097010014
:10A790000698010070030020F9970100F797010067
:10A7A000E8030020B80300200E98010010B504460D
:10A7B00006F00CFAE040431E033388BF012010BDB1
:10A7C000054B1A68054B53F8201001238B401342A8
:10A7D00014BF01200020704708050050049C0100B0
:10A7E000012070470020704738B52149214805F005
:10A7F00007FC0121204800F07CF91F4800F006F911
:10A800000121172006F0D0FB0021162006F0CCFB1A
:10A81000142400252946172006F0EEFB0A2006F036
:10A8200009FA013C85F00105F4D11420134C06F01F
:10A8300001FA114800F094F82068A0B100F050FA35
:10A8400088B1206800F092FB0D490A4805F0D8FB5A
:10A85000206800F051FA206800F0CCFB28B10949CB
:10A86000044805F0CDFB012038BD0749F8E700BFDB
:10A870003E980100700300209C0500202405002064
:10A8800048980100149701002897010007B500239C
:10A8900000931A461946034805F054FB03B05DF8CF
:10A8A00004FB00BF940500202DE9F84380460D46C7
:10A8B000174601EB02090C464C45A4EB05060BD0EC
:10A8C000D8F8003014F8011B1B6840469847002850
:10A8D000F2D13046BDE8F8833E46FAE770472030B3
:10A8E00005F0E1BC203005F0D0BC203005F0E1BC23
:10A8F00038B5437F0D460BB9002038BD00F1680420
:10A90000204605F0DEFC0028F6D12046294605F059
:10A91000ADFC0120F1E700002DE9F0411E460025C5
:10A920004FF47A73C0E901530C4B044640F8203BC6
:10A930008846174605F091FC04F1680005F08DFC8F
:10A940009DF8183063769DF81C302676C4E904879C
:10A95000A37665772046BDE8F08100BFE09801004E
:10A96000817E284A0123C37670B552F82140417E8A
:10A9700052F821104FF0A04504F5E07401F5E071A4
:10A9800040F20C6645F8246045F8216001694FF0FB
:10A99000CC74C1F8244501690624C1F80045847EC1
:10A9A000016952F82440C1F80845447E016952F813
:10A9B0002420C1F80C2590F91820510902F01F023B
:10A9C00093406031104A42F8213090F91830002B42
:10A9D000BDBF03F00F0302F6FC32D2189B18B5BFBF
:10A9E00040234022137683F8002390F91830012287
:10A9F000590903F01F0302FA03F3034A42F8213016
:10AA000070BD00BF049C010000E100E0C37E23B1E3
:10AA100003690022C3F8002570474269C2F8003577
:10AA200070472DE9F041044688461F461546002A26
:10AA300050D000F12006304605F023FC2369C3F80E
:10AA40008885236901221A622369C3F83465236962
:10AA5000C3F8385523691A602269D2F84C311BB902
:10AA6000D2F82431002BF8D00023C2F84C312269EF
:10AA7000D2F85C311BB9D2F82431002BF8D0002376
:10AA8000C2F85C3122696FB9D2F8243153B901237D
:10AA9000D3612369D3F84821002AFBD00022C3F8F0
:10AAA000482109E0012353612369D3F80421002AD6
:10AAB000FBD00022C3F804212369D3F8242112B16A
:10AAC0000022C3F824212369D3F83C052066C0B2D4
:10AAD000BDE8F0811046FBE70123FFF7A2BF10B5E8
:10AAE000044680F8B010683005F0CBFB0123637793
:10AAF00010BDF8B500234377036990F8B020C3F880
:10AB00008825036901261E62036900F16805044671
:10AB1000C3F8445528460F4605F0C5FB2369C3F822
:10AB2000480523699E602369D3F850211AB9D3F8E8
:10AB30002421002AF8D00022C3F85021284605F02D
:10AB4000B2FB236930B1D3F860211AB9D3F82421BC
:10AB5000002AF8D00022C3F8602123696FB9D3F826
:10AB6000242152B90122DA612369D3F84821002A4D
:10AB7000FBD00022C3F8482109E001225A61236971
:10AB8000D3F80421002AFBD00022C3F80421236952
:10AB9000D3F8240168B10022C3F824212369D3F833
:10ABA000C404C3F8C404022803D004280CBF032043
:10ABB0000420F8BD0121FFF79CBF70B54369D3F8AD
:10ABC0006421044692B10022012500F12006C3F859
:10ABD00064210577304605F054FB6369C3F834659A
:10ABE00063694022C3F8382563691D636369D3F83C
:10ABF0006821DAB10025C3F8685104F16806012321
:10AC000063772577304605F03CFBD4F8B43003B1C8
:10AC10009847636965773046C3F8446505F043FBA0
:10AC20006369C3F84805636901225A636369D3F80D
:10AC3000042162B10022C3F80421237F3BB1636980
:10AC4000D3F83C05D4F8B830206603B1984763695F
:10AC5000D3F8242152B10022C3F824216369D3F828
:10AC6000D024C3F8D024636901225A6170BD00006A
:10AC70000148FFF7A2BF00BF9C05002007B51623BF
:10AC80001722CDE900324FF0402204231146034839
:10AC9000FFF742FE03B05DF804FB00BF9C050020F7
:10ACA0000148FFF787BF00BF9C05002010B54FF497
:10ACB000C053038000230446837003610248FFF7FA
:10ACC0004FFE204610BD00BF9C050020016170476B
:10ACD0008078704741780148FFF701BF9C0500204C
:10ACE00008B5FFF7F7FF0348FFF764FFB0FA80F0FD
:10ACF000400908BD9C050020012303707047FF2315
:10AD0000C37200230373C370037143718371C371F2
:10AD1000037243728372704710B5064A01440023E0
:10AD2000884204D010F8014B6340D35CF8E7184622
:10AD300010BD00BFF8980100FFF7E1BF38B5084C1F
:10AD40000D46FFF7C7FFE1212046FFF7D1FD294659
:10AD50002046FFF7CDFDBDE83840FFF7A1BF00BF9B
:10AD60009C05002010B5054C417801222046FFF7D4
:10AD7000B3FE2046FFF7B6FDC0B210BD9C05002013
:10AD800010B5F0210446FFF7D9FF2046BDE810407A
:10AD9000FFF7E8BF70B5044605F018FF002506462A
:10ADA00005F014FF801BB0F57A7F4DD2236903B103
:10ADB00098472046FFF7E4FF10F00103054605D150
:10ADC000A278012A00D1A370284670BD1420013852
:10ADD00000BF00BF00BF00BF00BF00BF00BF00BF7B
:10ADE00000BF00BF00BF00BF00BF00BF00BF00BF6B
:10ADF00000BF00BF00BF00BF00BF00BF00BF00BF5B
:10AE000000BF00BF00BF00BF00BF00BF00BF00BF4A
:10AE100000BF00BF00BF00BF00BF00BF00BF00BF3A
:10AE200000BF00BF00BF00BF00BF00BF00BF00BF2A
:10AE300000BF00BF00BF00BF00BF00BF00BF00BF1A
:10AE400000BF00BFC3D1ABE70123BCE710B5E121D0
:10AE50000446FFF773FF2046BDE81040FFF782BFAE
:10AE600010B50446FFF796FF2046FFF733FF962103
:10AE70000648FFF73DFDFFF713FF2046FFF78AFF67
:10AE80002046BDE81040FFF7E1BF00BF9C05002051
:10AE9000FFF7E6BF10B5C3210446FFF74FFF20467A
:10AEA000BDE81040FFF75EBF38B504460D46FFF71A
:10AEB00071FF2046FFF70EFFD2210C48FFF718FD67
:10AEC000E94345EA0111C9B20848FFF711FDFFF750
:10AED000E7FE2046FFF746FFA84202D00423A370F6
:10AEE00038BDA378042BFBD10023F8E79C05002094
:10AEF00010B50446FFF7CEFF40F00401C9B220466A
:10AF0000BDE81040FFF7D0BF70B5164604460D46A9
:10AF1000FFF740FF16B12046FFF7EAFF2046FFF794
:10AF2000D9FEA5210548FFF7E3FC29460348FFF7B2
:10AF3000DFFCBDE87040FFF7B3BE00BF9C050020FA
:10AF400070B500220C4655210646FFF7DDFF651E51
:10AF5000073415F8011F00223046FFF7D5FFA54240
:10AF6000F7D170BDFFF7ECBFFFF7CEBF10B50446B9
:10AF7000FFF7B0FE20460022F021FFF7C5FFBDE835
:10AF80001040FFF78DBE000070B5164605460C4612
:10AF9000FFF700FF16B12846FFF7AAFF2846FFF784
:10AFA00099FE87210648FFF7A3FC002C0CBF214621
:10AFB00080210348FFF79CFCBDE87040FFF770BE9E
:10AFC0009C05002010B5002204460121FFF7DCFF9C
:10AFD0002046FFF7DFFEC0F3401010BDFFF7F2BFC1
:10AFE00010B50446FFF756FF20460021BDE810408B
:10AFF000FFF75ABF38B50446FFF7CCFEC30729D484
:10B000002046FFF7EDFF2046FFF7C4FE2046FFF77E
:10B0100061FEB4211048FFF76BFCFFF741FE2046AC
:10B02000FFF7B8FE10F00403054602D00223A37018
:10B0300002E0A278022AFAD0237843B12046FFF733
:10B0400029FF40F00101C9B22046FFF72DFFC5F3EB
:10B05000400038BD0020FCE79C0500202DE9F74F9B
:10B06000057B04460F46002D6BD1FFF7C3FF002878
:10B0700069D02046FFF78EFE2A46F0212046FFF7D2
:10B0800043FFDFF8C8804FF0FF394FF0010A94F911
:10B090000B30EEB24FEAD60B9D4206F007060AFAD5
:10B0A00006F623DA04EB0B03DB78334020460193EA
:10B0B000FFF770FE2046FFF70DFE78214046FFF7B0
:10B0C00017FC019B002B0CBF194680214046FFF75F
:10B0D0000FFCFFF7E5FD2046FFF75CFE820600F05F
:10B0E000400307D55BB16FF0010027E00CBF0123DF
:10B0F0000023DBE71BB9030658BF4FFA85F904EBC1
:10B100000B03010693F9032076B205F101054CBF4C
:10B110003243B243402DDA70B9D1B9F1FF3F04BFD9
:10B120000123237384F80B90E31C013F0B3413F8C5
:10B13000012B07F8012FA342F9D1012003B0BDE88C
:10B14000F08F0020FAE74FF0FF30F7E79C05002072
:10B1500008B5FFF783FF20EAE070C0B208BDFFF733
:10B1600049BF7047054A82610022027102700922BC
:10B170004270012281608270C270704763B100002A
:10B1800010B50C4620460721FFF7C6FDE3791B1AD0
:10B190005842584110BD70B5044680680E461546A9
:10B1A000FFF7DDFFB8B13146A068FFF7DBFE0022F4
:10B1B000BE21A068FFF7D8FE6E1E0835A068FFF715
:10B1C00067FE06F8010FAE42F8D1A068FFF7C7FF8F
:10B1D000431E5842584170BD10B51446FFF7DBFFBF
:10B1E00038B108212046FFF797FD237A1B1A5842F1
:10B1F000584110BD70B504460D4680681646FFF7ED
:10B20000AEFF2946A068FFF7ADFE00224E21A068E0
:10B21000FFF7AAFE0022B178A068FFF7A5FE002282
:10B22000F178A068FFF7A0FE2B78102B04D0002245
:10B230003179A068FFF798FEA068FFF790FF2946D4
:10B24000A068FFF78FFE2278A0684821FFF78CFEE8
:10B25000142005F0EFFC237813B10A2005F0EAFC76
:10B26000A068BDE87040FFF77ABF38B504460D46C8
:10B270008068FFF774FF2946A068FFF773FE00227D
:10B28000B421A068FFF770FEA068FFF7A7FE05468F
:10B29000A068FFF764FFB5FA85F0400938BDF0B546
:10B2A00085B0144601AA07460E46FFF795FF0546EE
:10B2B00090B13378102B0FD00B2C10D00C2C03D066
:10B2C0000A2C0ED13F2300E07F2301AA31463846E5
:10B2D0008DF80830FFF78EFF284605B0F0BD5F23DC
:10B2E000F3E71F23F1E71FB50B78102B10D001AA4D
:10B2F000FFF772FF78B19DF808303F2B0ED003D8CE
:10B300001F2B0DD0002006E05F2B03D07F2BF9D13F
:10B310000C2000E00B2005B05DF804FB0A20FAE7E2
:10B320000920F8E7F0B587B0044605F04FFC00F5BA
:10B330001C55A068FFF700FD00231035237101267E
:10B3400001A9A068FFF704FF40B305F03FFCA84245
:10B3500024D201A92046FFF713FF0028F0D023785C
:10B360002BB901A92046FFF780FF00B1267003AA80
:10B3700001A92046FFF70FFF01A920466778FFF7D4
:10B38000B2FF874205D96078237960700133237159
:10B39000D6E701A92046FFF7A6FFF5E707B0F0BD05
:10B3A000817070471FB501AAFFF7F5FE9DF80400F4
:10B3B000003018BF012005B05DF804FB0939C9B29F
:10B3C0000229F8B598BF104B0546164694BF33F9CD
:10B3D000114040F2EE248AB1C3787BB103786BB997
:10B3E00005F0F4FB074631462846FFF7DBFF20B99E
:10B3F00005F0ECFB001BB842F5D3F8BD2046BDE8D4
:10B40000F84005F017BC00BFF8990100F8B50446F4
:10B410000F46FFF768FF064610B900252846F8BD1D
:10B42000A068FFF79CFE0028F7D03946A068FFF718
:10B4300099FD2278A0684421FFF796FDA5782DB1EB
:10B440003A4631462046FFF7B9FFE7E70125E5E731
:10B4500010785378C00040EAC3200B78102B00B25C
:10B460000BD1D1799379C000CB1ADB0120F07F009A
:10B4700093FBF1F3103B184400B2704730B585B030
:10B4800001AA04460D46FFF7A7FE30B101AA2946DE
:10B490002046FFF7DDFF05B030BD0148FBE700BFE8
:10B4A00080E4FFFF10F5DC5FCABF07EE900ADFED16
:10B4B000037AFAEEEC7A17EE900A70470000FEC2AB
:10B4C00008B5FFF7DBFFBDE80840FFF7EBBF01461B
:10B4D0000422012001F0AABA01460422052001F04D
:10B4E000A5BA01460622092001F0A0BA01460422AD
:10B4F0000F2001F09BBA00002DE9F04F3D4E3E4C6D
:10B50000336813F0010387B082468B4615460ED18F
:10B51000E3644FF47A732365384BA36404F15C0051
:10B5200004F008FD082384F8683001233360344EAA
:10B53000346001F04DFC0027002859D04FF000493D
:10B540004FF00208CDF80C9005978DF8108003ACF1
:10B5500094E80E002B4805F0D9FD5046FFF7C1FFD7
:10B560003B463A4639460097204604F0EBFC04A8D7
:10B57000FFF7BCFF234805F0D5FD2B465A46514640
:10B58000306801F08FFF012805462DD1CDF80C90D1
:10B5900005978DF8108094E80E001A4805F0B6FD66
:10B5A0003168204601F0E5FC04A8FFF79FFF3168F1
:10B5B000204601F0ECFC04A8FFF789FF3168204623
:10B5C00001F0DEFC04A8FFF787FF0E4805F0AAFD96
:10B5D0003168204601F0E2FC0B4B049A5A6005F0FA
:10B5E0000FFB80B200F08EFD284607B0BDE8F08F5B
:10B5F0000546F9E75806002070060020649A01000D
:10B600006C0600205808002064060020F0B585B0C4
:10B6100007460E4614461D4601F0DAFB00B34FF014
:10B62000004301930023039302238DF8083004ABF9
:10B6300013E90E000B4805F069FD3846FFF751FF8E
:10B64000301DFFF753FF281DFFF741FF0A98043014
:10B65000FFF742FF034805F065FD034B62685A603F
:10B6600005B0F0BD5808002064060020F0B58DB08C
:10B670001D4600230F460093FF2304461646194635
:10B680001A4602A804F05EFC0B4B7A680493CDE9DD
:10B6900005237268CDE907236A68CDE90923039B76
:10B6A0000B930AAB009306AA08AB04A92046FFF748
:10B6B000ADFF0DB0F0BD00BF749C010000B50B4B99
:10B6C0004968526889B0CDE90231CDE90523049378
:10B6D000012301918DF80730019B079304AA06AB63
:10B6E00002A9FFF7C3FF09B05DF804FB749C0100D9
:10B6F0007FB5094B4A680493CDE9023201230192D8
:10B700008DF80730019B059304AA02A9FFF7D6FF25
:10B7100007B05DF804FB00BF749C010008B501F0A0
:10B72000BDFB012803D002280CBF0220002008BD69
:10B730007FB51E4E3068002836D001F0CBFE0228BF
:10B74000044601D004282CD14FF00043019300237C
:10B750000393022301AD8DF8083095E80E001448DC
:10B7600005F0D4FC3168284601F003FC02A8FFF77D
:10B77000BDFE3168284601F00AFC02A8FFF7A7FECB
:10B780003168284601F0FCFB02A8FFF7A5FE084837
:10B7900005F0C8FC3168284601F000FC054B029A10
:10B7A0005A60204604B070BD0446FAE76C060020DB
:10B7B000580800206406002030B585B0044604F027
:10B7C000B9FB4FF000430193002303930A4D02237A
:10B7D0008DF8083004AB13E90E00284605F096FCFE
:10B7E0000422A1180F2001F0D9F9284605F09AFC8F
:10B7F000204605B030BD00BF5808002030B585B0E8
:10B80000044604F097FB4FF0004301930023039399
:10B810000A4D02238DF8083004AB13E90E002846C8
:10B8200005F074FC0422A118052001F0B7F92846A0
:10B8300005F078FC204605B030BD00BF5808002058
:10B8400030B585B0044604F075FB4FF0004301931A
:10B85000002303930A4D02238DF8083004AB13E94B
:10B860000E00284605F052FC0422A118012001F028
:10B8700095F9284605F056FC204605B030BD00BFBE
:10B880005808002007B5002300931A4619460448BB
:10B8900004F058FB034803B05DF804EB04F04ABB26
:10B8A0005C06002064060020007C07288CBF002076
:10B8B0000120704781F0010070470846704708B5C5
:10B8C0000368DB6B984780F00100C0B208BD41827D
:10B8D000704713B502AB026803F8011D546819469E
:10B8E0000122A04702B010BD037C087C984204D11D
:10B8F00007288CBF002001207047002070470000FF
:10B9000010B50446007C072816D800F0A1FD1828C1
:10B9100006D80A4B23FA00F0C04300F0010010BD26
:10B920001C2807D1236820469B689847003018BF21
:10B930000120F4E70120F2E70020F0E70100100108
:10B94000F0B591B0044604A80F46164604F0F2FA8A
:10B9500000224FF47A73CDE908230CA8184B079303
:10B9600004F0E8FA082368468DF83C3004F0E2FA67
:10B97000207C072807D800F06BFD10B1207C00F078
:10B98000CBFD082323740F4B0F4D5B68039302A973
:10B9900004A8029501F0DDFD41F288336A4639467C
:10B9A00004A801F05FFF40B12368019A9B690392EC
:10B9B0000295324602A92046984711B0F0BD00BF5B
:10B9C000649A010064060020749C010008B5007CA4
:10B9D000072802D800F02EFF08BD0020FCE710B5B4
:10B9E0000446207C07280BD800F032FD172801D030
:10B9F0001C2805D1207C00F01DFFB0F5006FF0D3AE
:10BA000010BD38B50546007C0728144605D892B20B
:10BA100000F092FE10B901236B600024204638BD6F
:10BA200008B5007C072802D800F02EFE08BD0020D3
:10BA3000FCE7007C072802D812B200F08BBD002082
:10BA4000704707B501220DF10701007C00F082FD6F
:10BA50000028CCBF9DF807004FF0FF3003B05DF821
:10BA600004FB10B5037C072B044602D94FF0FF30CE
:10BA700010BD03689B6898470028F7D0207C00F031
:10BA80002FFEF5E738B50446007C07280AD800F0F9
:10BA900043FD05F09BF80546207C00F0D9FC10B969
:10BAA0000823237438BDFBF78BFA012005F0C2F898
:10BAB00005F08CF8638A401B9842EDD3207C00F09F
:10BAC000E5FCEDE77FB50446007C07280D461646E9
:10BAD00007D800F0BDFC10B1207C00F01DFD08234C
:10BAE00023740021684604F039FA6A68019B9A427F
:10BAF00002D1002004B070BD4FF0FF3102A804F065
:10BB00002DFA6A68039B9A42F3D00021212000F0AD
:10BB100003FB07282074ECD8291D324600F0D4FC22
:10BB200005F054F80546207C00F092FC172815D04B
:10BB30001C2813D00028DCD005F048F8638A401B8D
:10BB4000984205D8FBF73CFA012005F073F8EAE7C4
:10BB5000207C00F09BFC08232374CAE70120C9E77E
:10BB600010B41446064A127801EB022101EB0020C2
:10BB70001A46214680B25DF8044B01F00FB800BFB1
:10BB80003C0700207FB5037C072B05464FF00004DF
:10BB90001BD84FF0004302260394019301AC8DF8AB
:10BBA000086094E80E000A4805F0B0FA33462246D1
:10BBB0000421287CFFF7D4FF9DF804309DF8054050
:10BBC000034844EA032405F0ADFA204604B070BDF2
:10BBD000580800207FB50B7C072B05460E4605D97B
:10BBE000002104F0BBF9284604B070BD4FF00043BB
:10BBF000019300230393022301AC8DF8083094E8ED
:10BC00000E00084805F082FA042322460C21307CFD
:10BC1000FFF7A6FF034805F085FA2146284604F001
:10BC2000A3F9E0E7580800207FB5037C072B054601
:10BC30004FF000041BD84FF00043022603940193F9
:10BC400001AC8DF8086094E80E000A4805F05EFA31
:10BC5000334622461021287CFFF782FF9DF80430EE
:10BC60009DF80540034844EA032405F05BFA2046AA
:10BC700004B070BD5808002007B5002300931A4691
:10BC80001946034804F05EF903B05DF804FB00BFF9
:10BC9000DC06002003681B6B18470000024A0260A4
:10BCA0008A694260704700BF749C0100808B7047B6
:10BCB000008A7047408C704713B502AB026803F8E6
:10BCC000011D546819460122A04702B010BD7047FB
:10BCD00010B5044690F82000072804D800F0D6FBE1
:10BCE000082384F8203010BD38B5044690F82000B1
:10BCF00007280D4601D800F0C9FB2946022000F0B4
:10BD00000BFA072884F820004FF000009EBF6084E3
:10BD10002582012038BD0000F0B591B0044604A88A
:10BD20000F46164604F006F900224FF47A73CDE967
:10BD300008230CA8134B079304F0FCF8082368466B
:10BD40008DF83C3004F0F6F80F4B104D5B68039310
:10BD500002A904A8029501F0FCFB41F288336A466F
:10BD6000394604A801F07EFD012808D12368019A14
:10BD70001B6A03920295324602A92046984711B0E9
:10BD8000F0BD00BF649A010064060020749C0100AD
:10BD900008B50023C383043190F8200000F09CFD17
:10BDA00008BD08B590F8200000F0C4FD08BD10B52E
:10BDB00093B204460A46C18B90F8200000F060FD63
:10BDC000E38B0344E38310BD13B5438C04461BB9D6
:10BDD0004FF0FF3002B010BD01220DF1070190F8C5
:10BDE000200000F0B7FB0028F2DD638C9DF807000F
:10BDF000013B6384EEE710B5438C044613B94FF062
:10BE0000FF3010BD934294BF1AB212B290F82000D6
:10BE100000F0A0FB0028F2DD638C1B1A6384F0E7BE
:10BE200008B590F82030072B05D8428C1AB1184677
:10BE300000F056FC08BD4FF0FF30FBE773B5044639
:10BE400090F8200007280E46154601D800F01EFB8A
:10BE5000094B00932A46736801936946822000F0DB
:10BE600017FA072884F820004FF000009EBF608476
:10BE70000120258202B070BD749C010013B50446F8
:10BE8000628C2AB1236800211B6B20469847F7E794
:10BE900094F8200000F0F8FBD8B10822694694F825
:10BEA000200000F057FB002813DD694604F1140060
:10BEB00004F062F89DF804209DF805309DF8070015
:10BEC00003EB0223A3839DF8063000EB032080B22E
:10BED000608402B010BD000007B5002300931A462D
:10BEE0001946034804F02EF803B05DF804FB00BFC8
:10BEF000E406002007B5084B1B7801EB032101EB9A
:10BF0000002001220DF1070180B200F047FE9DF8EC
:10BF1000070003B05DF804FB3C07002007B5084BA1
:10BF20001B7801EB032101EB002002A980B201F88C
:10BF3000012D012200F07AFDC0B203B05DF804FBD0
:10BF40003C07002010B41446064A127801EB022187
:10BF500001EB00201A46214680B25DF8044B00F048
:10BF600065BD00BF3C0700202DE9F7430C4617468E
:10BF70001E4601AA022324210546FFF7F1FD9DF884
:10BF800004209DF8053043EA0223224A1C4413781A
:10BF9000332B0CBF05F1080005F11000A4B2C0025C
:10BFA000C4F30A0980B24844372B904680B22DD0A2
:10BFB00009EB0603B3F5006F28DDC9F500691FFA28
:10BFC00089F94A46394600F031FD98F80030332BA4
:10BFD0000CBF05F1080005F11000C002A6EB090234
:10BFE00080B292B207EB09013444A4B200F01EFD06
:10BFF00023128DF8043001AA0223242128468DF84B
:10C000000540FFF79FFF03B0BDE8F0833246394695
:10C01000EAE700BF3D07002008B50321FFF76AFFEC
:10C0200008BD07B50B128DF804308DF805100223FA
:10C0300001AA0421FFF786FF03B05DF804FB08B5F1
:10C040000A4604230C21FFF77DFF08BD07B50B123C
:10C050008DF804308DF80510022301AA1021FFF796
:10C0600071FF03B05DF804FB07B5022301AA20218C
:10C07000FFF776FD9DF804009DF8053043EA0020A7
:10C0800003B05DF804FB000038B50546FFF7ECFF90
:10C0900004462846FFF7E8FF8442034604D1034BD9
:10C0A00003EBC5039C8038BD1C46F2E7F406002074
:10C0B00007B5022301AA2621FFF752FD9DF80400CF
:10C0C0009DF8053043EA002003B05DF804FB07B596
:10C0D000022301AA2821FFF743FD9DF804009DF8E3
:10C0E000053043EA002003B05DF804FB044B1B78E5
:10C0F000332B0CBF0C301830C00280B2704700BF29
:10C100003D070020034B1A88C0F30D0050401880F3
:10C11000704700BF080000202DE9F043574B1B7803
:10C1200085B081460F468BB3332B4FF0004301930C
:10C130004FF000054FF0020303958DF8083001AE73
:10C1400096E80E004E4814BF4FF008084FF0040860
:10C1500004F0DCFFECB22046FFF75EFF7055D8B16B
:10C160000135EBB29845F5D800234FF03451F25C1D
:10C170001D2ADCB203D821FA02F2D20708D4013317
:10C18000DAB24245F3D33E4804F0CCFF082465E020
:10C190001021204600F0C6FE3A4B002123F814106F
:10C1A000FA20013800BF00BF00BF00BF00BF00BFC2
:10C1B00000BF00BF00BF00BF00BF00BF00BF00BF87
:10C1C00000BF00BF00BF00BF00BF00BF00BF00BF77
:10C1D00000BF00BF00BF00BF00BF00BF00BF00BF67
:10C1E00000BF00BF00BF00BF00BF00BF00BF00BF57
:10C1F00000BF00BF00BF00BF00BF00BF00BF00BF47
:10C2000000BF00BF00BF00BF00BF00BF00BF00BF36
:10C2100000BF00BF00BF00BFC3D14A462046FFF7A2
:10C220007DFEFF2202212046FFF778FED7B1394676
:10C230002046154DFFF7F5FE00260121204600F0AF
:10C2400071FE25F834602046FFF741FF05EBC4037B
:10C2500058809E719E800A4804F064FF204605B015
:10C26000BDE8F083094B1A88013292B2B2F5404F13
:10C2700038BF4FF440421A801988D9E73D070020A3
:10C280005808002058070020F4060020080000206D
:10C290002DE9F047694B1B7886B082460E4617465B
:10C2A000A3B3332B4FF0004303934FF000054FF03F
:10C2B000020305958DF810300DF10C0898E80E007A
:10C2C0005F4814BF4FF008094FF0040904F01EFF47
:10C2D000ECB22046FFF7A0FE08F80500E0B10135FA
:10C2E000EBB29945F4D800234FF0345118F80320ED
:10C2F0001D2ADCB203D821FA02F2D20708D4013396
:10C30000DAB24A45F2D34E4804F00CFF082485E027
:10C310001021204600F006FE4A4B002123F814109D
:10C32000FA20013800BF00BF00BF00BF00BF00BF40
:10C3300000BF00BF00BF00BF00BF00BF00BF00BF05
:10C3400000BF00BF00BF00BF00BF00BF00BF00BFF5
:10C3500000BF00BF00BF00BF00BF00BF00BF00BFE5
:10C3600000BF00BF00BF00BF00BF00BF00BF00BFD5
:10C3700000BF00BF00BF00BF00BF00BF00BF00BFC5
:10C3800000BF00BF00BF00BF00BF00BF00BF00BFB5
:10C3900000BF00BF00BF00BFC3D152462046FFF719
:10C3A000BDFDFF2202212046FFF7B8FD002F39D046
:10C3B00039462046FFF735FE5E238DF80630737947
:10C3C00003F07F038DF80730B3798DF8083001252D
:10C3D000F3798DF80930311D2046ADF80450FFF790
:10C3E0002EFE39462046FFF731FE0623194601AAE4
:10C3F0002046FFF7A7FD2946134D0026204600F0F2
:10C4000091FD25F834602046FFF761FE05EBC4037B
:10C4100058809E719E800A4804F084FE204606B033
:10C42000BDE8F087094B1A88013292B2B2F5404F4D
:10C4300038BF4FF440421A801988BAE73D07002000
:10C440005808002058070020F406002008000020AB
:10C4500030B585B04FF000430193002303930A4C9D
:10C4600002238DF8083004AB13E90E000546204680
:10C4700004F04CFE2846FFF7CFFD0546204604F0A9
:10C4800051FE284605B030BD5808002030B585B0B3
:10C490004FF000430193002303930A4C02238DF8CD
:10C4A000083004AB13E90E000546204604F02EFECA
:10C4B0002846102100F036FD204605B0BDE830408A
:10C4C00004F030BE58080020F0B585B04FF00043AE
:10C4D0000193002303930F4D02238DF8083004AB22
:10C4E00004460F461646284613E90E0004F00EFED9
:10C4F00039462046FFF7A3FD31462046FFF7A6FD4B
:10C500002046042100F00EFD284605B0BDE8F040AD
:10C5100004F008BE5808002030B585B04FF0004345
:10C520000193002303930A4C02238DF8083004ABD7
:10C5300013E90E000546204604F0E8FD28460821D0
:10C5400000F0F0FC204605B0BDE8304004F0EABD44
:10C55000580800202DE9F04F85B04FF000430193BB
:10C56000464E00230393022336F830408DF80830FE
:10C5700001AB17460546894641480ECB04F0C6FD7F
:10C58000A7420EDD2846FFF793FD04462846FFF735
:10C590008FFDA042F9D106EBC5039B79E41A26F87A
:10C5A00035408CB92846FFF737FD142805D020B157
:10C5B000B0F11C0418BF4FF0FF34314804F0B2FD55
:10C5C000204605B0BDE8F08F4FEAC50BBC4206EB34
:10C5D0000B03A8BF3C46B3F80280A7B2B9F1000F25
:10C5E00021D02846FFF782FD264A1278C8F30A0AAE
:10C5F0005044372A80B23DD01AFA84F2B2F5006F67
:10C6000038DDCAF500631FFA83FA5246494600F046
:10C61000C5FA2846FFF76AFDA7EB0A02D14492B299
:10C62000494600F0BBFA06EB0B0236F8353091793B
:10C63000B844DB1B0F44BFB21FFA88F89BB2F92F36
:10C64000A2F8028026F8353000D8ABB95E4400234A
:10C65000B3714FEA28238DF8043001AA0223282160
:10C6600028468DF80580FFF76DFC4021284600F034
:10C6700059FCA2E73A46D3E797719EE7F4060020FB
:10C68000580800203D0700207FB5134D064635F8B9
:10C690003000F8B94FF000430193022303908DF866
:10C6A000083004AB0D4813E90E0004F02FFD3046AE
:10C6B000FFF7FEFC04463046FFF7FAFCA042F9D132
:10C6C000064804F02FFD05EBC6039879201A80B2C6
:10C6D00025F8360004B070BDF4060020580800208C
:10C6E0007FB54FF00043019300230393104D0223C5
:10C6F0008DF8083001AC94E80E000646284604F098
:10C7000005FD3046FFF7F2FC0A4B03EBC60301229E
:10C710005B88C3F30A031844214680B200F03EFA56
:10C72000284604F0FFFC9DF8040004B070BD00BF73
:10C7300058080020F40600202DE9F04FB2F5006FF4
:10C7400087B028BF4FF40062DFF8E49005468A46C0
:10C75000164603AC02234FF000474FF00008039742
:10C76000CDF814808DF8103094E80E00484604F09F
:10C77000CDFC2846FFF788FC83462846FFF74CFC93
:10C780000190484604F0CEFC019B172B01D01C2BD6
:10C7900032D104F071FAB345DCD303974FF00008AF
:10C7A0000227CDF814808DF8107094E80E00204810
:10C7B00004F0ACFC4146334652462846FFF7D4FB12
:10C7C0002021284600F0AEFBDFF864804FF0004BDC
:10C7D00002212846FFF78EFB10F0100A1FD12846D1
:10C7E000FFF71AFC814648B9114804F09BFC4E46FD
:10C7F000304607B0BDE8F08F4646CEE7404604F02D
:10C8000091FC04F039FACDF80CB0CDF814A08DF8F5
:10C81000107094E80E00404604F078FCD8E710222F
:10C8200002212846FFF77AFB014804F07BFCDFE792
:10C830005808002030B585B04FF000430193002325
:10C84000039302238DF8083004AB054613E90E006C
:10C850000A4804F05BFC2846FFF716FC044628460D
:10C86000FFF7DAFB0546054804F05CFC172D02D003
:10C870001C2D18BF0024204605B030BD58080020EC
:10C880002DE9FF411C464FF0004301930023039321
:10C89000104D02238DF8083004AB06460F46904633
:10C8A000284613E90E0004F031FC3046FFF7ECFB9C
:10C8B000844228BF0446A4B2234642463946304645
:10C8C000FFF752FB284604F02DFC204604B0BDE8DB
:10C8D000F08100BF580800207FB50B7806460D4652
:10C8E00014462BB94B781BB98B780BB9C878D0B1EB
:10C8F000DCB14FF0004301930023039302238DF832
:10C90000083004AB13E90E00094804F0FFFB294688
:10C910003046FFF794FB21463046FFF797FB04486B
:10C9200004F000FC012004B070BD2046FBE700BF0E
:10C93000580800202DE9FF4700234FF00048022748
:10C94000CDF8048003938DF8087001AC94E80E00D4
:10C9500005461F48DFF8789004F0D8FB20212846D0
:10C9600000F0E0FA02212846FFF7C4FA10F01006A2
:10C9700023D102212846FFF7BDFA10F0080A0BD098
:10C98000182202212846FFF7C9FA114804F0CAFB11
:10C99000304604B0BDE8F087484604F0C3FB04F01D
:10C9A0006BF9CDF80480CDF80CA08DF8087094E8F0
:10C9B0000E00484604F0AAFBD4E7102202212846C4
:10C9C000FFF7ACFA024804F0ADFB0120E1E700BF3D
:10C9D0005808002007B5002300931A46194603485B
:10C9E00003F0B0FA03B05DF804FB00BFEC060020D2
:10C9F00070B505460C468E18B44206D021782846FC
:10CA000004F091FB04F8010BF6E770BD024B002126
:10CA1000187804F0F1BA00BF0A000020024B01218F
:10CA2000187804F0E9BA00BF0A0000202DE9F341AC
:10CA30004F4B1B78332B04460D4616461FD100EB97
:10CA400002084C4F4D1E1FFA88F8A0457AD0FFF718
:10CA5000DDFFF021384604F066FB210A384604F079
:10CA600062FBE1B2384604F05EFB013415F8011FA9
:10CA70003846A4B204F057FBFFF7D0FFE5E7342BAC
:10CA8000C7B21DD1FFF7C2FF330A241263F07F0340
:10CA90000422694637488DF800408DF801708DF802
:10CAA00002308DF80360FFF7A3FF013D314CAF1951
:10CAB000AF4245D015F8011F204604F034FBF7E7DC
:10CAC000FFF7A4FFFF2C08D800238DF800308DF865
:10CAD000017004238DF802300DE0230419D4E41012
:10CAE00024F01F04002344F00C048DF800308DF86E
:10CAF00001708DF80240052E28D82A46531BDBB260
:10CB0000B34218DA02A8034412F8011B03F8051C0B
:10CB1000F4E744F3871323F01F03B4F5404F4FEAC3
:10CB200014228DF800208DF8017034BF43F01403F7
:10CB300043F01C03CEE7F21C69460E48FFF758FF8E
:10CB4000FFF76CFF304602B0BDE8F0810322694672
:10CB50000848084FFFF74CFF731E6C1E15FA83F54B
:10CB600014F8011F384604F0DEFAA542F8D1E7E7D1
:10CB70003D0700205808002007B502AB012203F84A
:10CB8000011D1946FFF752FFC0B203B05DF804FB68
:10CB900008B501460020FFF7EFFF08BD2DE9F3417E
:10CBA0003E4B1B78332B04460E46154620D100EB36
:10CBB00002083B4F4E1E1FFA88F8A0453AD0FFF7F7
:10CBC00025FF0F21384604F0AEFA210A384604F05A
:10CBD000AAFAE1B2384604F0A6FA0021384604F079
:10CBE000A2FA013406F8010FA4B2FFF717FFE4E739
:10CBF000342BC7B222D1FFF709FF2412C5F3062355
:10CC000004228DF804408DF805708DF806308DF8FB
:10CC100007500DEB02012248FFF7EAFE2A460021E9
:10CC2000304606F046FB2A4631461D48FFF7E0FE37
:10CC3000FFF7F4FE284602B0BDE8F081FFF7E6FEFC
:10CC4000FF2C07D800238DF804308DF805708DF87F
:10CC500006300DE023040ED4E41024F01F0400235A
:10CC600044F008048DF804308DF805708DF8064006
:10CC7000032201A9CFE744F3871323F01F03B4F580
:10CC8000404F4FEA14228DF804208DF8057034BF10
:10CC900043F0100343F01803D9E700BF3D0700201D
:10CCA0005808002007B501220DF10701FFF776FFB4
:10CCB0009DF8070003B05DF804FB08B50020FFF7FE
:10CCC000F1FF08BD10B58020FFF762FF1424FFF7C5
:10CCD000F4FF40B1013C0120A4B203F0ABFF002CF3
:10CCE000F5D1204610BD0120FCE7000008B50F4B30
:10CCF00033221A70FFF7E6FF08B9002008BD1020A4
:10CD0000FFF746FFFFF7D9FF1028F6D11220FFF7F3
:10CD10003FFFFFF7D2FF1228EFD10020FFF738FFC7
:10CD2000FFF7CBFFB0FA80F04009E7E73D070020AE
:10CD300008B5124B34221A70FFF7C4FF08B900205F
:10CD400008BD0820FFF724FFFFF7B7FF0828F6D13A
:10CD50001020FFF71DFFFFF7B0FF1028EFD10020D4
:10CD6000FFF716FFFFF7A9FF0028E8D11F20FFF704
:10CD700099FFC31E58425841E2E700BF3D0700201B
:10CD800008B5124B37221A70FFF79CFF08B9002034
:10CD900008BD0820FFF7FCFEFFF78FFF0828F6D13B
:10CDA0001020FFF7F5FEFFF788FF1028EFD10020D5
:10CDB000FFF7EEFEFFF781FF0028E8D13920FFF7EB
:10CDC00071FF031F58425841E2E700BF3D070020B2
:10CDD0007FB52D4E3478002C53D14FF40C7003F0F6
:10CDE00029FF2A4804F07CF9294B0121187804F026
:10CDF000DBF8FFF713FE4FF00043019302238DF899
:10CE00000830039404AB13E90E00204804F07EF9C7
:10CE1000FFF78EFFB0B11F4B40221A70E5B202221D
:10CE20001E212846FFF77AF8013402221F212846E6
:10CE3000FFF774F8082CF1D11448012404F072F9BA
:10CE400034701BE0FFF79CFF18B1124B10221A70D0
:10CE5000F2E7FFF74BFF044658B10E4B0422552171
:10CE60001B201A70FFF788FE55211A20FFF784FE59
:10CE7000E2E7094B1870054804F054F9204604B065
:10CE800070BD0124FAE700BF3E07002058080020CB
:10CE90000A0000203C0700203D0700201FB5FFF7D7
:10CEA00097FF38B11D4B1B78342B4FF0000003D097
:10CEB000372B1BD004B010BD4FF000430193022369
:10CEC00003908DF8083004AB13E90E00144804F009
:10CED0001DF93520FFF7E6FE0446114804F022F95B
:10CEE00014F0200F14BF01200220E3E74FF00043AD
:10CEF0000193022303908DF8083004AB13E90E0070
:10CF0000074804F003F92E20FFF7CCFE044604483E
:10CF100004F008F914F0010FE4E700BF3D0700201A
:10CF20005808002038B50A4601210446FEF7F6FFEE
:10CF3000054D2402287804EB0020013080B2FFF771
:10CF4000B1FE0028F6D138BD3C07002007B500230C
:10CF500000931A461946034802F0F4FF03B05DF847
:10CF600004FB00BF3407002014220021103006F01B
:10CF7000A0B910B51031044602F0F6FF204610BDEE
:10CF800010B51431044602F0EFFF204610BD10B575
:10CF90001831044602F0E8FF204610BD10B52031DC
:10CFA000044602F0E1FF204610BD30204B1C087003
:10CFB000110902F00F02092A94BF3032373203F808
:10CFC00001290A460029F3D17047000007B5002364
:10CFD00000931A461946034802F0B4FF03B05DF807
:10CFE00004FB00BF400700202DE9F0418EB004464D
:10CFF000884616460021202206A806F05AF9FF238B
:10D000001A461946009302A802F09CFF04F1480555
:10D01000554B04934322039B059304A92846FEF72E
:10D02000B7FE013000F09D80504B069363688DF889
:10D0300021601BBA0793330A8DF820301C2280230D
:10D0400006A926462846ADF82230FEF7B0FE1A2281
:10D0500000210DF11E0006F02CF956F8080F06907D
:10D06000B388ADF81C30102206A92846FEF79FFEB3
:10D070002022002106A806F01CF90627202206A976
:10D080002846FEF794FE013FF8D1394B069340F253
:10D090003513ADF81C303D238DF81F3007238DF874
:10D0A000203001238DF821303368CDF82230B38849
:10D0B000ADF826302F498DF81E8040F60C430DF157
:10D0C0002A00ADF8283007F076F8E27A0CA920465D
:10D0D000FFF76BFF227B0DF132012046FFF765FF62
:10D0E000627B0DA92046FFF760FF1E2206A9284695
:10D0F000FEF75DFEB8F1030F24D140F23243ADF8E4
:10D100001830237C8DF81A30637C8DF81B30A37C9B
:10D110008DF81C30E37C8DF81D3040F23643ADF8BD
:10D120001E30237F8DF82030637F8DF82130A37F60
:10D130008DF822300C22E37F8DF8233006A9284693
:10D14000FEF735FE0C4A0D4B06A9CDE9062328460D
:10D15000FF2309228DF82030FEF729FE2846FEF72E
:10D1600020FE0EB0BDE8F081749C010001010600B4
:10D1700063825363AC9A010037060103060F3A3B02
:10D180002DE9F04391B005468846164603F01EFD92
:10D1900005F1480407462046FEF770FE00280BDC28
:10D1A00003F014FDC01B404500F2D280F9F708FFE0
:10D1B000012003F03FFDEEE7242207A92046FEF7F9
:10D1C0001AFE9DF81C30022B40F0BD80B5F864308B
:10D1D000432B40F0B880089F3FBA3760062205F124
:10D1E00008010EA806F032F8064628B92B689F42BF
:10D1F00002D36B689F4207D92046FEF768FD0026E0
:10D20000304611B0BDE8F0830B9B2B610146CC2268
:10D210002046FEF7F0FD05F124072046FEF74AFD03
:10D22000002840F391802046FEF7CEFD33287DD0C4
:10D2300015DC012844D006DC0028EED02046FEF79D
:10D24000C3FDC2B253E0032844D00628F6D12046DD
:10D25000FEF7BAFD0422804605F1200141E03A289C
:10D260004AD020DC352823D03628E7D12046FEF7E7
:10D27000ABFD05F11C084146814601A802F074FE91
:10D28000002103A802F06AFE029A049B9A4230D061
:10D29000414605A802F068FE2A6E069B9A4228D0F5
:10D2A0005FFA89F223E03B2833D0FF28B5D0C5E7E9
:10D2B0002046FEF789FD2046FEF786FDC6B2ACE7A4
:10D2C0002046FEF781FD042205F114012046FEF7F9
:10D2D00092FDA2E72046FEF777FD0422804605F185
:10D2E00018012046FEF787FD5FFA88F2043A002114
:10D2F000ECE704224146E9E72046FEF765FD0422FB
:10D3000005F128012046FEF776FDAB6A1BBAAB6239
:10D3100083E72046FEF758FD042205F12C01204644
:10D32000FEF769FDEB6A1BBAEB6276E72046FEF773
:10D330004BFD042239462046FEF75DFD6B6A1BBAA1
:10D340006B622B6369E700262046FEF7C0FC57E7B7
:10D35000FF2655E72DE9F34704464FF4FA61012013
:10D3600003F0B5FA2746606047F8480B3846FEF7E9
:10D37000AFFC44213846FEF7B7FC002800F090804F
:10D3800003F024FC4FF00009804600254FF0030A0B
:10D3900094F84430032B1CD043BB636801336360B3
:10D3A00003F014FC4FF47A72A0EB08000121B0FBEB
:10D3B000F2F2204692B2FFF717FE012384F84430C0
:10D3C000002DE5D103F002FCA36BA0EB080098420E
:10D3D000DBD93846FEF77CFC63680133636003F0F9
:10D3E000F5FB2064284602B0BDE8F087042B11D17C
:10D3F00063680133636003F0E9FB4FF47A72A0EBDA
:10D4000008000321B0FBF2F2204692B2FFF7ECFDD8
:10D410000223D3E7012B19D101AAE16B2046FFF7C4
:10D42000AFFE0228064638D1019B636003F0CEFBB5
:10D430004FF47A72A0EB08000321B0FBF2F2204611
:10D4400092B2FFF7D1FD84F84460B9E7022BB7D15F
:10D4500001AAE16B2046FFF793FE0528064617D187
:10D46000636A84F844A013B94FF461736362A36ADA
:10D4700013B9636A5B08A362E36A1BB9636AA3EB2F
:10D48000D303E362A36A2363E36A636301257FE74F
:10D49000062802D184F8449092E7FF2EFAD08FE755
:10D4A00005469FE7F8B500250F460446C0E9095533
:10D4B000C562C0E90E2385608581FFF755FD3B6895
:10D4C000A360BB88A38184F844502046BDE8F8409F
:10D4D000FFF740BF10B5044603F078FB236CC31A76
:10D4E000B3F57A7F14D34FF47A71B3FBF1F201FBF9
:10D4F0001233C01A236B206451008B4234BF0023C7
:10D500009B1A2363636B99428CBF00239B1A63634E
:10D51000206BE0B994F84430032B06D1042384F83F
:10D5200044302046FFF716FF0130636B73B994F85F
:10D530004430032B00D04BB9002384F844302046FC
:10D54000FFF712FD2046FFF705FF033010BD002056
:10D55000EBE74B68436000230381704770B50024FC
:10D560000139234611F8010FB8B1A0F13005EEB230
:10D57000092E08D803EB830305EB43039BB2FF2B73
:10D58000F0D900200DE02E28FBD1032CF9D0601C2F
:10D5900014442371C4B20023E4E7032C01D1D371F6
:10D5A000012070BD07B5002300931A4619460348B1
:10D5B00002F0C8FC03B05DF804FB00BF4807002080
:10D5C0002DE9F74305460E4603F000FB05F10C0478
:10D5D000288105F10801022202AD2046FEF7E7FB93
:10D5E000012325F8023D022229462046FEF7DFFBF3
:10D5F0004FF48073022229462046ADF80630FEF72C
:10D60000D6FB0023022229462046ADF80630FEF75D
:10D61000CEFB022229462046FEF7C9FB02222946FC
:10D620002046FEF7C4FB37463378E3B13E46B046AA
:10D6300018F8013B0BB12E2B13D1A6EB0709B9F15A
:10D64000000F0CDD01220DF1050120468DF805903B
:10D65000FEF7ADFB4A4639462046FEF7A8FB474693
:10D66000E2E74646E3E702A9012201F8033D20462E
:10D67000FEF79DFB4FF48076294602222046ADF846
:10D680000660FEF794FB022229462046ADF80660AC
:10D69000FEF78DFB012003B0BDE8F0832DE9F043D8
:10D6A00087B006460F46904603F090FA06F10C0448
:10D6B00005462046FEF7E2FB002808DC03F086FA68
:10D6C000401BB84200F2C480F9F77AFCF1E7726AB5
:10D6D00073689A4240F0BF80338D352B40F0BB8099
:10D6E0002046FEF7E7FA0B2840F3B8800C220DEB3A
:10D6F00002012046FEF77FFBBDF80E203189130A98
:10D7000043EA0223BDF80C201BB29DB29142ADF852
:10D71000065001D1002B07DB2046FEF7D8FA4FF662
:10D72000FC7007B0BDE8F08340F20F231D4005D028
:10D730002046FEF7CCFA4FF6FB70F2E7BDF8123048
:10D740001F0A47EA0327BFB22FB92046FEF7BFFAE8
:10D750004FF6FA70E5E7BDF810305BBAAAB29BB29B
:10D760009A4216DA01220DF10A012046FEF743FB28
:10D770009DF80A201AB100212046FEF73CFB9DF8D7
:10D780000A100029EED104222046FEF734FB0135B1
:10D79000E1E70026B14601220DF105012046FEF722
:10D7A0002AFB9DF8052012F0C00134D112B12046A9
:10D7B000FEF721FB9DF80550002DECD1022202A9B5
:10D7C0002046FEF718FB02220DF10A012046FEF763
:10D7D00012FB042229462046FEF70DFB02220DF122
:10D7E00006012046FEF707FBBDF80830BDF806200D
:10D7F000B3F5807F52BA92B21CD1BDF80A0040BA8C
:10D8000085B2012D16D1042A0DD02046FEF75FFA0D
:10D810004FF6F77085E7012200212046FEF7EBFA6C
:10D820008DF80590C6E708F104012046FEF7E3FAFB
:10D83000284676E7013600212046B6B2FEF7DBFA2D
:10D84000B742A8D12046FEF742FA4FF6F67068E7D5
:10D850004FF6FF7065E74FF6FE7062E74FF6FD701A
:10D860005FE700002DE9F34705468A469146984652
:10D87000FFF774FE0446B8BB1E4B6A685B689A42A9
:10D8800034D003F0A3F905F10C0600F00F0101F507
:10D8900080613046FEF728FA0128074620D1164B52
:10D8A000009335226B68019369463046FEF770FAA3
:10D8B00098B151462846FFF783FE70B13046FEF717
:10D8C00070FA50B14A4641462846FFF7E7FE044643
:10D8D000F9F776FB384603F0ADF93046FEF7F8F974
:10D8E000204602B0BDE8F0870124F9E76FF001049B
:10D8F000F6E700BF48070020749C010007B500232D
:10D9000000931A461946034802F01CFB03B05DF869
:10D9100004FB00BF50070020006903681B6918471B
:10D92000006903685B69184713B5006949680368B3
:10D93000034C01919B6900946946984702B010BD61
:10D94000749C010000690368DB691847006903687B
:10D950009B6A18470069003018BF01207047006CAF
:10D9600070470164704710B590F83830044633B9F9
:10D9700020690368DB689847002808DA10BD03684F
:10D980009B6898470028F3D14FF0FF30F6E794F8F2
:10D990002220A2F10803022BF0D8A36A002BC2BFF9
:10D9A000E36A0133E3620A2AE8D1E36B013BE363F4
:10D9B000002BE3D1092384F82230DFE710B50446B9
:10D9C000006903681B6A984794F82230083B022BD1
:10D9D00007D8A36A002B04DD0028A2BFE36A1B1846
:10D9E000E36210BD73B590F82230092B04460ED1C6
:10D9F0000026206903689B68984740B12069036846
:10DA0000DB689847C5B20A2D1CD184F8225094F8DF
:10DA100022300A2B04D1E36B13B9092384F8223096
:10DA200094F82230092B22D0206903689B6898471C
:10DA300094F822300A2B03D1E36B9842A8BF184612
:10DA400002B070BD0D2DD4D0284605F0A8FB0028EB
:10DA5000CFD0E06BADF8046010228DF804500021A7
:10DA6000050101A807F036FB2844E063C1E7002068
:10DA7000E6E7000000234FF0FF32C0E90A23084A1E
:10DA800080F8223012680263064A4362126880F806
:10DA90003830C36347F2305342630364704700BFBA
:10DAA000100000201400002038B504461D46002058
:10DAB0004FF47A73C4E901030B4B2360C4E90412E9
:10DAC00004F1180002F036FA0123258484F844306A
:10DAD00084F84530054904F1480002F051FF204622
:10DAE000FFF7C8FF38BD00BF149B0100CA9B0100AF
:10DAF00010B50446006903685B6A98472046BDE894
:10DB00001040FFF7B7BF012380F8223070470000B4
:10DB100038B504460069154602F065FA04492069E3
:10DB200002F061FA29462069BDE8384002F072BA75
:10DB3000717D010038B504460D460069114602F0BA
:10DB400052FA1D49206902F04EFA2946206902F076
:10DB50004AFA1A49206902F05DFA94F84530F3B1A7
:10DB60006369B3B11649206902F03DFAD4E90401B2
:10DB700002F039FA238C502B08D01249206902F0A8
:10DB800032FA0A22218C206902F08DFA206902F013
:10DB900031FA0D4B0D491A682046FFF7B9FF94F88A
:10DBA000443023B10A4A0B492046FFF7B1FF012355
:10DBB00084F82230002038BDA07E0100D99A0100EF
:10DBC000E39A0100068001000C000020EA9A01009F
:10DBD000F59A0100FB9A010038B504460069154624
:10DBE00002F001FA0549206902F0FDF92946206991
:10DBF0000A22BDE8384002F058BA00BF717D01002A
:10DC000010B50446006902F0F5F9022384F82230C9
:10DC100010BD70B590F82230012B04460D46164613
:10DC200001D8FFF7EDFF20690368324629465B689B
:10DC3000BDE87040184770B590F82230012B0446BB
:10DC40000D4601D8FFF7DCFF2069036829461B68F1
:10DC5000BDE87040184710B50446206903689B680A
:10DC6000984720B120690368DB689847F5E710BD45
:10DC70002DE9F347994690F82230083B022B0446E1
:10DC80000E469246DDE90A7804D8FFF7E4FF204605
:10DC9000FFF7F0FE94F82250012D45D894F8443057
:10DCA0005BB1D4E90401228C0368B9B92149009120
:10DCB000E16901919B69694611E0206903689B6AEB
:10DCC00098470028EDD0314652462046FFF732FFF4
:10DCD000064650B1304602B0BDE8F087DB69984790
:10DCE0000028F0DC4FF0FF36F4E7B9F1000F04D064
:10DCF0004A4611492046FFF70BFF002F17DD3A4631
:10DD00000E492046FFF768FFB8F1000F0FD001253C
:10DD10002046FFF775FF002DDCD023683A465B688C
:10DD2000414620469847D5E76FF00106D2E7002D1F
:10DD3000D0D1EDE7749C0100B39A0100C09A0100B4
:10DD400090F82230012B01D8FFF75ABF7047FFF738
:10DD5000F7BF000007B500234FF0FF32CDE90023E5
:10DD6000024AFFF785FF03B05DF804FB069B010044
:10DD70002DE9F04790F82230012B044651D9DFF805
:10DD8000D8800025032700236362022384F8223011
:10DD900002F01CFF464682464FF00A090A2D46D083
:10DDA00002F014FF236CA0EB0A00984245D22368CE
:10DDB00020469B68984748B323682046DB6898470D
:10DDC000431C0546ECD094F82230022B05D0032BDF
:10DDD0000FD002F0FBFE8246E0E733782A2B01D019
:10DDE00083421AD17278731C0AB984F822701E46D5
:10DDF000EFE7A0F13002092A95BF636A042309FB0B
:10DE0000032384F8223098BF6362E2E74FF47A700C
:10DE100002F010FFC2E70A2D06D16FF00300BDE843
:10DE2000F0876FF00100FAE76FF00200F7E7636A2E
:10DE3000C72B02DC652B18BF002594F82230042B79
:10DE4000E9D1606AC72801DC65289CD10A2D18BF7A
:10DE50006FF00200E3E700BFCF9A010038B501F18F
:10DE6000480504463A21284602F06AFE421C034651
:10DE700005D10649204602F083FD204638BD002228
:10DE80002946204602F07AFEF7E700BFCA9B010050
:10DE9000F8B501F1480605460F4630463A2102F032
:10DEA0004FFE441C013005D10C49284602F068FDA4
:10DEB0002846F8BD3B6DA34209DD2146304602F0FD
:10DEC00023FE007805F062F908B10134F2E73B6DFA
:10DED00022463146284602F051FEE9E7CA9B01007E
:10DEE00010B503680446DB68984794F82230A3F124
:10DEF0000802022AC0B232D9052B31D0072B39D003
:10DF0000042B54D1226B137883420BD1531C23630F
:10DF1000537823B9C4E90A33052284F822200A2859
:10DF20001DD136E0636B197881420BD15A1C6263B4
:10DF30005B78002BF3D1012384F83830062384F872
:10DF40002230ECE71B4909688A42F7D11A4A126865
:10DF50009342F3D10D28F1D1072384F8223010BD6C
:10DF6000A0F13002092AE9D8A36A0A2101FB0323A0
:10DF7000A362D4E70A28F2D194F838309BB1092380
:10DF800084F822300023E36394F82230083B022B0C
:10DF9000E5D9042384F82230064B1B682363064B23
:10DFA0001B686363DBE7082384F82230ECE70A2868
:10DFB000D5D1E9E7100000201400002038B5044650
:10DFC00002F004FE054694F82230083B022B13D9D8
:10DFD00002F0FCFD236C401B98420DD223682046C2
:10DFE0009B68984718B12046FFF77AFFE8E74FF49F
:10DFF0007A7002F01FFEE6E794F82230083B022B0D
:10E0000094BF00206FF0020038BD10B590F82230A8
:10E01000083B022B044601D9FFF7D0FFA06A10BDD0
:10E0200038B590F82230083B022B054601D9002074
:10E0300038BDFFF7EAFF0130F9D02846EC6AFFF758
:10E04000E4FF8442B4BF00200120F1E7FFF7E8BFFE
:10E05000FFF7E6BF38B500F1480504460E492846EB
:10E0600002F0EBFC94F82230083B022B09D9204641
:10E07000FFF736FF0D2801D00A2807D1236D002BAA
:10E08000F0D0206D003018BF012038BDC1B2284645
:10E0900002F0F4FCE6E700BFCA9B010007B50023CD
:10E0A00000931A461946034801F04CFF03B05DF88F
:10E0B00004FB00BF6807002080687047C16070479C
:10E0C000036810B59B690C469847036821461B6896
:10E0D000BDE8104018472DE9F84380460D46174625
:10E0E00001EB02090C46A145A4EB050609D0D8F8BE
:10E0F00000304046DB689847431C03D004F8010B0E
:10E10000F1E73E463046BDE8F883C368013310B5F9
:10E11000044612D1236820469B69984703689B6890
:10E12000984758B123682046DB6898472028F1DDDE
:10E130002368C1B25B6920469847012010BD70B5C5
:10E140000446C068431C18D102F040FD00F5FA7582
:10E15000236820469B69984703689B68984718B9CD
:10E1600002F034FD8542F3D8236820469B69984726
:10E170000368BDE87040DB6818474FF0FF33E36089
:10E1800070BD10B5182005F03FF8044618B11822EC
:10E19000002105F08EF8204610BD70B506460C46ED
:10E1A000D4B1237C65681B0704D4E16811B1304603
:10E1B000FFF7F3FF237C03F00F03042B03D1606907
:10E1C00008B100F0F3FC206808B100F0EFFC204635
:10E1D00005F022F82C46E3E770BD00002DE9F04F72
:10E1E000036885B0DB6805460E469847421C044626
:10E1F00004D14FF0FF3005B0BDE8F08F2D282FD1AE
:10E200002B682846DB689847431C0446F1D04FF042
:10E21000FF330093A4F13003092B4FF000070DD812
:10E220004FF00A082B682846DB689847A0F13003B6
:10E23000303C092B08FB07470446F3D92E2C11D09C
:10E2400024F02003452B0DD0009B7B4373610223F8
:10E2500033742B6828465B69E1B298470020CAE70F
:10E260000123D6E7384604F0CBF92E2C80468946A8
:10E2700039D12B68DFF814B1DB68284698470027AE
:10E2800004464FF0000A52465B464046494604F0B9
:10E2900021FA80468946A4F1300004F0B1F94246E3
:10E2A0004B4604F061F82B688046DB6828468946B7
:10E2B0009847A0F13003092B07F1FF370446E2D954
:10E2C00024F02003452B2AD12B682846DB68984789
:10E2D0002B28044609D12B682846DB68984704465A
:10E2E0004FF0010A0AE00027EAE72D28F8D12B6851
:10E2F0002846DB6898474FF0FF0A04464FF0000BB2
:10E300000A22A4F13003092B0DD802FB0B3B2B682A
:10E310000392DB6828469847039A0446F1E74FF0DA
:10E32000010A4FF0000B009804F06AF942464B4690
:10E3300004F0D0F9CDE90001584604F061F98046B7
:10E340005046894604F04CF902460B464046494681
:10E3500004F0C0F980463846894604F051F9024677
:10E360000B464046494603F0FFFF02460B4600209D
:10E37000064902F019FF0B460246DDE9000104F0F0
:10E38000A9F904F09FFC0323706161E700002440B9
:10E3900019B10A22496901F064BE084670470000BD
:10E3A000F8B504462DED028B00295AD091ED058A6F
:10E3B00018EE100A04F036F9B5EEC08AF1EE10FA44
:10E3C00006460F4606D52C49204601F00CFE07F103
:10E3D00000431F463946304604F054FC0A220546E5
:10E3E0000146204601F06BFE2449204601F0FBFD6A
:10E3F000284604F0F5F802460B463046394603F04D
:10E40000B1FF1BA3D3E9002303F0AEFF1C4B002296
:10E4100004F060F90F46064604F034FC0A22014677
:10E420000546204601F05AFE284604F0D9F8024677
:10E430000B463046394603F095FF0022002306467E
:10E440000F4604F0AFFB60B900220D4B3046394651
:10E4500004F040F904F016FC0A220146204601F0BF
:10E460003DFEBDEC028B0020F8BD00BFAFF3008085
:10E470007B14AE47E17A743F0BA10100BB91010010
:10E4800000002440F8B50368DB6806460F4698474D
:10E49000222803D04FF0FF342046F8BD04233B74FC
:10E4A00000F0F4FA05460028F4D033683046DB6803
:10E4B0009847431C044611D0222C36D01F2C34DD43
:10E4C0005C2C04D02946E0B200F0F6FAEDE73368A0
:10E4D0003046DB689847421C044603D1284600F0CA
:10E4E000F7FAD9E7622817D007DC2F2803D05C2879
:10E4F00001D02228D9D12946E6E76E280FD004DCC6
:10E500006628D2D129460C20DEE772280AD074286A
:10E51000CBD129460920D7E729460820D4E7294648
:10E520000A20D1E729460D20CEE7284600F012FB4D
:10E5300000247861B0E7000038B50D461D49044657
:10E5400001F051FD7DB3013D15F8011F59B31F299D
:10E5500007D9222905D05C2903D0204601F047FDC8
:10E56000F2E75C21204601F042FD29780C2914D005
:10E5700007D8092915D00A2911D00829E4D1622128
:10E58000EBE72229E9D003D80D29DDD17221E4E798
:10E590002F29E2D05C29E0D0D6E76621DDE76E21A5
:10E5A000DBE77421D9E72221204601F020FD00207D
:10E5B00038BD00BF747D01004969FFF7BDBF38B5A4
:10E5C0000368DB68044698474FF48075411C0FD000
:10E5D00020280EDC013D6A1C236803D0DB6820463E
:10E5E0009847F3E72368C1B25B692046984700204B
:10E5F00038BD002DF6D14FF0FF30F9E703682DE963
:10E60000F047DB6804468846914698477B2803D04C
:10E610004FF0FF30BDE8F087062388F81030204621
:10E62000FFF7CDFF23682046DB6898477D2843D05D
:10E630002368C1B25B6920469847FF264FF0000A65
:10E64000FFF79FFD05460028E2D096B3C8F80C00FE
:10E650002046FFF7B4FF29462046FFF713FF01309D
:10E66000D6D02046FFF7ABFF6B692B602368C5F857
:10E6700014A0DB68204698473A28C9D12046FFF706
:10E680009EFF4A462946204600F018F80130BFD0C8
:10E690002046FFF794FF23682046DB6898472C2824
:10E6A0002F464FF00006CBD07D3818BF4FF0FF301B
:10E6B000B0E778608760CBE70020ABE7F7B50446AA
:10E6C0000E461746FFF77BFF013002D14FF0FF30B7
:10E6D00011E023682046DB689847431C0546F5D0C7
:10E6E0002368C1B25B6920469847222D05D1314687
:10E6F0002046FFF7C7FE03B0F0BD2D2D03D0A5F1D6
:10E700003003092B04D831462046FFF767FDF2E7B6
:10E710005B2D05D13A463146204600F078F8EAE70D
:10E720007B2D05D13A4631462046FFF767FFE2E7E9
:10E730006E2D15D102AD002345F8083D2368042253
:10E740001B6929462046984704280246BED11D4928
:10E75000284605F070FD0028B8D100233374CAE7BD
:10E76000662D16D1002300938DF80430236805220E
:10E770001B696946204698470528A7D105221249FA
:10E78000684605F058FD0028A0D101233374307588
:10E79000B1E7742D9AD102AD002345F8083D2368F6
:10E7A00004221B69294620469847042802468DD139
:10E7B0000649284605F03FFD002887D10123337420
:10E7C000337598E78E9B0100939B0100999B010094
:10E7D000F8B5064617460D4611B900242046F8BD87
:10E7E000FFF7CFFC04460028F7D02846FFF7E7FEE6
:10E7F0003A4621462846FFF761FF0130EED1214617
:10E800003046FFF7CAFCE8E70022FFF7E1BF2DE939
:10E81000F8430368DB6804468846914698475B28BE
:10E8200003D04FF0FF30BDE8F883052388F810309F
:10E830002046FFF7C4FE23682046DB6898475D2822
:10E840002AD02368C1B25B6920469847FF26FFF7AC
:10E8500098FC05460028E4D0DEB1C8F80C0020463C
:10E86000FFF7ADFE4A4629462046FFF727FF06463A
:10E870000028D6D12046FFF7A2FE23682046DB6899
:10E8800098472C282F46E2D05D3818BF4FF0FF3054
:10E89000C9E778608760E2E70020C4E738B505463D
:10E8A00051B3CC687B2101F0A2FB013002D14FF0C3
:10E8B000FF3038BDB4B121682846FFF73DFE013076
:10E8C000F5D03A21284601F092FB0130EFD02146E5
:10E8D000284600F013F80130E9D0646814B12C2107
:10E8E0002846E0E77D21284601F081FB01304FF00A
:10E8F000FF3018BF0020DCE70846DAE7E9B10B7CFF
:10E9000003F00F03062B18D8DFE803F004070D0F00
:10E91000111315000A4901F066BB0B7D0BB10949C3
:10E92000F9E70949F7E7FFF733BDFFF739BDFFF70F
:10E9300043BE00F00EB8FFF7B1BF0020704700BF24
:10E940008E9B0100999B0100939B01001046FFF7ED
:10E95000D5BF38B50546F1B1CC685B2101F047FB66
:10E96000013002D14FF0FF3038BD54B12146284666
:10E97000FFF7C4FF0130F5D0646814B12C2128469C
:10E98000ECE75D21284601F032FB01304FF0FF300B
:10E9900018BF0020E8E70846E6E731B1CB6800225F
:10E9A000D0B2013213B15B68FAE70846704731B163
:10E9B000C96821B11AB1013AD2B24968F9E70846EB
:10E9C000704738B515460C4641B1CC6834B129467C
:10E9D000206805F0ACFB08B16468F7E7204638BD55
:10E9E00051B14AB1CB6813B9CA6070470B46596838
:10E9F0000029FBD15A6093607047F8B505460E4672
:10EA000017461C4673B1186808B100F0CFF83846B5
:10EA100000F076F82246206031462846BDE8F840EE
:10EA2000FFF7DEBFF8BD08B5FFF7ABFB18B1037CFD
:10EA30006FF303030374037C6FF30713037408BDC0
:10EA400010B50C46FFF79DFB10B10223037444611F
:10EA500010BD70B50D46194604461646FFF7F0FF87
:10EA60003246034629462046BDE87040FFF7C5BF41
:10EA700007B5002300931A461946034801F062FACD
:10EA800003B05DF804FB00BF7007002038B50C2010
:10EA900004F0BAFB044650B1064820604FF480757C
:10EAA0002A46002104F005FC00236560A36020468F
:10EAB00038BD00BF84080020D1E90132013B9A42F1
:10EAC00004D20B6898548B6801338B600020704728
:10EAD00008B104F0A1BB704738B5054658B1074CE2
:10EAE000216819B1284605F05CFB10B1A468002C20
:10EAF000F6D1204638BD0446FBE700BF7C07002066
:10EB0000F8B50746FFF7E8FF20B103790133037139
:10EB10000068F8BD0E4D2B6843B9384605F054FB2C
:10EB2000012328602B71F4E73546F4E7AE68002E28
:10EB3000FAD10C2004F068FB04460028E9D0A86054
:10EB4000384605F041FB012320602371A660E0E711
:10EB50007C070020826838B5044622B1036813445C
:10EB600013F8013C1BB121460020FFF7A5FF054823
:10EB7000FFF7C6FF054610B1204604F04DFB2846BE
:10EB800038BD00BF8408002010B5074CA06800B94C
:10EB900010BD0268836822B9A36004F03DFBA3683E
:10EBA000204604461846F2E77C07002038B5FFF7F8
:10EBB00093FF054660B10479013CE4B204713CB9AD
:10EBC000006804F029FB2C60BDE83840FFF7DCBF8B
:10EBD00038BD000008B5064B1B7843B9054801F065
:10EBE00009FA05490348BDE8084001F0F3B908BD3A
:10EBF000CD070020E0070020C49B0100F0B5047899
:10EC00009FB005464CB31C4B1C4F1B68986804F022
:10EC1000ABF92846194906F07BF91EAD012445F8E9
:10EC2000780D3946002006F073F91E2C264645F86B
:10EC3000240002D001340028F3D1114B009F1C683E
:10EC400084B12168384605F0ACFA48B963682946B2
:10EC5000304698470446FFF7BDFF20461FB0F0BD81
:10EC6000A468EDE7074B1B78002BF6D1064907484F
:10EC700001F0C6F9EFE700BF38000020A07E0100D8
:10EC8000C8070020CD070020CB9B0100E007002033
:10EC9000F8B505460C200F4604F0B6FA0C4B0446B6
:10ECA0001860284605F0ABFA013004F0ADFA2946A9
:10ECB000064605F080FA284605F0A1FA00233354F1
:10ECC000044B1A68A260C4E900671C60F8BD00BF6D
:10ECD000C807002088070020184B1B7870B5FBB9C7
:10ECE0001748184D01F0D4FCC4B20A2C0CD00D2CDE
:10ECF0000AD0082C15D12146114801F078F92B785B
:10ED000073B1013B2B700BE02B780F4E0F490C4871
:10ED10000024F45401F067F93046FFF76FFF2C70C0
:10ED200070BD2146064801F062F92B783A2B9FBF4F
:10ED30005A1C2A70044AD454F2E700BFCD070020C1
:10ED4000E0070020CC0700208C070020C89B0100B2
:10ED5000064B1B7810B53BB9054C204601F092FCE0
:10ED600010B1FFF7B9FFF8E710BD00BFCD070020D5
:10ED7000E0070020054A00231370054A014613608E
:10ED800010B1044801F03EBC704700BFCC07002022
:10ED900088070020E007002070B504460D4601F00A
:10EDA00015FFA061A068036829461B68BDE8704094
:10EDB000184770B504460D46164601F007FFA061DE
:10EDC000A0680368324629465B68BDE87040184772
:10EDD00010B50446C06804F01FFA204610BD2DE9A6
:10EDE000F04105460E4601F0F1FE4FF47A77804679
:10EDF000A86803689B689847044658B901F03CFF2F
:10EE000001F0E4FEAB8AA0EB08007B439842EFD30D
:10EE1000204605E0A8680368DB6898473070012049
:10EE2000BDE8F08138B5148821441546FFF7D7FFB7
:10EE300008B101342C8038BD2DE9F74F02AD002612
:10EE400025F8026D8A462A46C1680446FFF7EAFFA4
:10EE500018B9002003B0BDE8F08FE3680DF1080990
:10EE600093F8008009F8036D0127BDF80630052BE3
:10EE700007D14FF0FF33A068E36303685B6A9847EC
:10EE8000E7E749462046FFF7AAFF0028E1D0BDF892
:10EE90000630E268591CADF806109DF80510D154F3
:10EEA0009DF8053003F07F0207FB02661A064FEA61
:10EEB000C717DAD49DF8063008F0F008013BB8F126
:10EEC000300F8AF800301DD12A46E1682046FFF74E
:10EED000A9FF0028BDD02A46E1682046FFF7A2FF1F
:10EEE0000028B6D0E2689AF80030134459789D782B
:10EEF000137805EB01259B07ADB201D50235ADB204
:10EF0000022701E000273D46BDF806B0A7EB0B073E
:10EF100007EB0B0296422AD949462046FFF75FFFCE
:10EF2000002896D0A06B88B1B8F1300F0ED19AF8B6
:10EF30000020C2F1FF2202F57F02FE325A44AA42AB
:10EF400004D902689DF8051012689047BDF80620A4
:10EF5000218A914208D9E1689DF805008854BDF8DE
:10EF600006200132ADF806200BF1010BD0E7A26BB1
:10EF700022B9218A594538BFADF80620BDF80600F0
:10EF800068E70120704773B50025DC1103F07F06A8
:10EF9000A3B20CB146F080060DF1080C681C654464
:10EFA000C0B205F8046C0546002CEED1C0F1040592
:10EFB000515501ADA04205DD231A1344615D59711D
:10EFC0000134F7E7013002B070BDF8B506461746C8
:10EFD0001C46FFF7D8FFB368C0B21A680444C0F1FA
:10EFE00005015568394422461846A847054601F0F0
:10EFF000EDFDB061A8B2031B58425841F8BD10B5F1
:10F00000C368E0221A70C36800225A700446806800
:10F01000E168036802225B689847A0684FF0FF33FD
:10F02000E36303685B699847A06803685B6A984775
:10F0300001F0CCFDC4E9060010BD023330B598B232
:10F040000C46631A14F8015B9BB21DB1431C1554A6
:10F0500098B2F6E7C11A0A44191202F8021C02F823
:10F06000013C30BD38B50546806808B9002038BD80
:10F0700003689B6A9847EC6B68B9002CF6D1A868C6
:10F080006FF00203EB6303685B699847A868036845
:10F090005B6A9847EAE7B4FA84F04009E7E70000C2
:10F0A0002DE9FF470C9D9DF840A004468946174670
:10F0B0001E46FFF7D7FF8046002840F0DF80A0689B
:10F0C00003689B6A9847002840D00123E3826E4B77
:10F0D000029345F25443ADF80C3004238DF80E3002
:10F0E000052302A91944E26811F8051CD154013323
:10F0F0000C2BF6D1002D3DD09DF838309DF83420F2
:10F100005B0143F0040343EAC203DBB2BAF1000F30
:10F1100001D043F002031FB1002E2DD143F0800334
:10F12000E2681373638AE2681B125373E368628AAE
:10F130009A73218A484605F0A5F8238A113098422F
:10F140001DD9A06803685B6A984797E0A068216BA7
:10F150000368A28E39B1DB6998470128B5D06FF0FA
:10F160000103E3638AE049499B690291E16A0391E3
:10F1700002A9F1E72B46C9E743F0C003D0E74946AF
:10F180000F23E2682046FFF758FF814605B3218A26
:10F19000284605F077F809F102031844238A9842BB
:10F1A000CFD84B462946E2682046FFF746FF218A22
:10F1B00005460F9805F066F8238A023028449842E5
:10F1C000BFD82B46E2680F992046FFF736FF8146ED
:10F1D00017B3218A384605F055F809F1020318449F
:10F1E000238A9842ADD84B46E26839462046FFF75D
:10F1F00024FF814686B1218A304605F043F809F1A3
:10F2000002031844238A98429BD84B46E268314651
:10F210002046FFF712FF8146A9F105039BB2E26881
:10F2200010212046FFF7D1FE01F0D0FCC4E9060012
:10F230004FF47A75A06803689B68984758B901F045
:10F24000C5FCE369C01AA38A6B439842F2D36FF0FE
:10F250000303E36375E70DF107012046FFF7ECFDBB
:10F2600004287FF46EAFE368DD785DB901F0AEFC91
:10F270004FF00108E06184F82050E563404604B097
:10F28000BDE8F087E5635CE700044D51749C010024
:10F2900010B586B0012404940B9C03949DF828407B
:10F2A00002949DF824400194089C0094FFF7F8FE16
:10F2B00006B010BD2DE9F3470446FFF7D3FE8046A4
:10F2C000D0B101F083FC628A4FF47A735343E26950
:10F2D000821A9A42074603D8A269821A93421FD221
:10F2E00094F8203063B16FF00303A068E363036810
:10F2F0005B6A98474FF00008404602B0BDE8F087CF
:10F30000E268C0211170E2685370A068E168036888
:10F3100002225B689847C4E90677012384F820300D
:10F32000A06803689B6898470028E5D00DF10701A5
:10F330002046FFF781FD83B20646002B73D0E368B9
:10F34000E7611A7802F0F002302A57D1626A002A87
:10F35000D2D09DF807209918901C49781D5C05EBC8
:10F360000125ADB2D11C19442A46184403F088FF88
:10F37000E3689DF807202B44134400229A70E1684B
:10F380009DF807C091F8009009F00609B2B20CF19F
:10F390000200B9F1020F0844666A0CF10303A2EB04
:10F3A0000C0225D12B440CF1050C11F803E00B44A1
:10F3B000521B93F801A06544053A29440AEB0E2A32
:10F3C000B047E36840221A70E36883F80190E3686D
:10F3D0001FFA8AFA4FEA2A229A70E36883F803A098
:10F3E000A068E168036804225B689847A76183E727
:10F3F0002B44033A521B1944B0477DE7C02A0BD176
:10F40000D0221A70E36800225A70A068E16803688D
:10F4100002225B6898476FE7D02A7FF46DAF002324
:10F4200084F8203068E72046FFF71CFE002808BF5C
:10F430004FF0000860E770B590B005460E46FFF744
:10F4400011FEE0B1304604F0DAFE3123C4B28DF88B
:10F450000030A31C8DF801303B220023314601A867
:10F460008DF802308DF8034004F0F7FE2B68221D62
:10F470005B68694628469847003018BF012010B0E5
:10F4800070BD2DE9F0470446884617461D469DF895
:10F490002060FFF7E7FD50B3B4F8109040464946AE
:10F4A00004F0F0FEEB1D1844814520D341460523AE
:10F4B000E2682046FFF7C1FD00211FFA81FC4318D6
:10F4C000AC459BB2E26801F1010104D217F80CC00F
:10F4D00002F803C0F1E7002EA3F1050320469BB21A
:10F4E00014BF31213021BDE8F047FFF76EBD002089
:10F4F000BDE8F08773B505460E4614466AB1018A29
:10F50000104604F0BFFE0346002200923146224618
:10F510002846FFF7B6FF02B070BD1346F4E7F7B513
:10F5200005460E461F46144662B1018A104604F095
:10F53000A9FE03460097224631462846FFF7A1FF61
:10F5400003B0F0BD1046F4E72DE9F04704468846C5
:10F5500092461E46FFF786FD002843D0218A40468A
:10F5600004F090FE9DF82030002BE3680CBF3022A1
:10F57000312287B21A70B21C3A44012002F07F0196
:10F58000E568D20918BF41F08001431C29545FFA95
:10F5900080F9D2B941469BB2E2682046FFF74DFDA3
:10F5A000A368E1681A68D2F8048002461846C0478A
:10F5B00055468046B244AA4509D0A06815F8011BFB
:10F5C00003681B6898478044F5E71846D6E701F0C2
:10F5D000FDFAA06109F1030038443044A0EB0803B0
:10F5E00058425841BDE8F087F7B505460E461F461C
:10F5F000144662B1018A104604F044FE03460097A7
:10F60000224631462846FFF79FFF03B0F0BD104663
:10F61000F4E7F8B505460E4614461F46FFF722FDEF
:10F6200028B331460523EA682846FFF706FD631F25
:10F63000002F03440CBF3021312106469BB2EA68FB
:10F640002846FFF7A0FC0146A868EC680368053E61
:10F650000E44C1F105015B682144324698470446D7
:10F6600001F0B4FAA861A0B2831B58425841F8BD1A
:10F6700070B50D460446018A2846164604F002FE7F
:10F6800045B3012E26D8238A0930834222D320464F
:10F69000FFF7E8FCF0B1E38A01339BB2C3B1E38228
:10F6A000E38AE2681B125371E368E28A9A71E268A6
:10F6B000294607232046FFF7C0FCE3681E54031FBA
:10F6C000E26820469BB28221BDE87040FFF77DBC16
:10F6D0000123E4E7002070BD0022FFF7C9BF70B529
:10F6E0000D460446018A284604F0CCFD25B3238A42
:10F6F0000930834220D32046FFF7B4FCE0B1E38A0F
:10F7000001339BB2B3B1E382E38AE2681B12537107
:10F71000E368E28A9A71E268294607232046FFF7E8
:10F720008CFC431FE26820469BB2A221BDE87040DA
:10F73000FFF74BBC0123E6E7002070BD0163828622
:10F74000704741627047C06B704738B504460D463C
:10F7500009B9002038BD038A4BB9084603F054FDAF
:10F76000E060E0682582003018BF0120F2E7C06841
:10F7700004F022FC0028F3D1EBE7000070B50C4B3D
:10F7800000250446456040F8283B0E4600F0D2FBB9
:10F790004FF0FF33E363A660A56325824FF48071C9
:10F7A0002046FFF7D2FF0F236382A382204670BD5D
:10F7B000E49B010007B5002300931A46194603484D
:10F7C00000F0C0FB03B05DF804FB00BFD0070020D1
:10F7D0008271054A417112680449B2FBF1F14FF49C
:10F7E0007A724A43C26070471800002040420F00FE
:10F7F00038B504460D464079022101F0D5FB01F0F1
:10F80000E5F9A0F5FA60A060657438BD70B50546ED
:10F810000E460024687901F001FCB042A3B206D183
:10F82000EA689A4204F10104F4D84FF0FF33184615
:10F8300070BD30B50D46D1B0044601F0C7F93DB9F1
:10F84000A368C31AB3F5FA6F02D2207C51B030BD61
:10F8500000250221A06025606079257101F0A4FBDC
:10F86000012001F0E7F90121607901F09DFB2946B3
:10F87000607901F0C1FBA379153B012B00F28C806C
:10F8800040F24C40013800BF00BF00BF00BF00BFC6
:10F8900000BF00BF00BF00BF00BF00BF00BF00BF70
:10F8A00000BF00BF00BF00BF00BF00BF00BF00BF60
:10F8B00000BF00BF00BF00BF00BF00BF00BF00BF50
:10F8C00000BF00BF00BF00BF00BF00BF00BF00BF40
:10F8D00000BF00BF00BF00BF00BF00BF00BF00BF30
:10F8E00000BF00BF00BF00BF00BF00BF00BF00BF20
:10F8F00000BF00BF00BF00BF00BFC3D160790221BD
:10F9000001F052FB607C00283BD0013800BF00BFF3
:10F9100000BF00BF00BF00BF00BF00BF00BF00BFEF
:10F9200000BF00BF00BF00BF00BF00BF00BF00BFDF
:10F9300000BF00BF00BF00BF00BF00BF00BF00BFCF
:10F9400000BF00BF00BF00BF00BF00BF00BF00BFBF
:10F9500000BF00BF00BF00BF00BF00BF00BF00BFAF
:10F9600000BF00BF00BF00BF00BF00BF00BF00BF9F
:10F9700000BF00BF00BF00BF00BF00BF00BF00BF8F
:10F98000C3D172B600212046FFF740FF013007D1F6
:10F990000020207462B659E7142001F04BF9ADE75E
:10F9A00001212046FFF732FF0130F1D00025002170
:10F9B0002046FFF72BFF01214DF805002046FFF7F9
:10F9C00025FF0DEB05030835B5F5A07F5860EED196
:10F9D00062B600225DF832500DEBC203691C586814
:10F9E00001D0431C02D1002020742FE7D1108542A2
:10F9F000635C4FEA4303DBB202F1010238BF43F01C
:10FA00000103282A6354E5D16178237822790B44D5
:10FA1000A1780B44E1780B44DBB29A42E3D1012098
:10FA2000E2E70000000000002DE9F8430D462DED4F
:10FA3000028B11460446FFF7FCFE00287ED0A37916
:10FA40000B3B0B2B7AD8DFE803F0063F7979797905
:10FA5000797979796565A378E07808EE103A01063E
:10FA6000B8EE488A48BFFFEE007A00F00F0048BFAA
:10FA700037EEC88A02F0C4FD31A3D3E9002302F0B7
:10FA800029FE064618EE100A0F4602F0CBFD0B4683
:10FA900002463946304602F067FC03F013F903468C
:10FAA0006DB102F0BFFD2AA3D3E9002302F012FEDC
:10FAB000254B002202F058FC03F004F90346BDEC8C
:10FAC000028B1846BDE8F883E078A67800F00F00B6
:10FAD00002F096FD1AA3D3E9002302F0FBFD07EE26
:10FAE000906AF8EE677A804617EE900A894602F02F
:10FAF00099FD02460B464046494602F035FC03F0AC
:10FB0000E1F83206034648BF80F00043002DD6D00E
:10FB10001846C6E7A678E378300200F4FE401843A2
:10FB200007EE900AF8EEE77A17EE900A02F07AFDF7
:10FB300003A3D3E9002302F0CDFDE0E7034BBEE7CA
:10FB40009A9999999999B93F000040400000C07F67
:10FB5000CDCCCCCCCCCCFC3FD0B50446FFF769FE75
:10FB600090B3A3790B3B0B2B2ED8DFE803F00606EE
:10FB70002D2D2D2D2D2D2D2D1C1C607802F040FDDE
:10FB800014A3D3E9002302F0A5FD064620780F4612
:10FB900002F036FD02460B463046394602F0E4FBE1
:10FBA00003F090F8D0BD208840BA80B207EE900AEA
:10FBB000F8EEE77A17EE900A02F034FD05A3D3E9D8
:10FBC000002302F087FDEBE70148EBE7AFF300808D
:10FBD0000000C07F9A9999999999B93F00B55DF84D
:10FBE00004FB0020704700B501205DF804FB10B550
:10FBF0000446C06803F010FBB4F90600002802DBDD
:10FC0000002101F0D1F9204610BD70B50546C0684D
:10FC10000E4603F001FBEC7C2A7C94420CBF0324CB
:10FC2000042414FB06F4A4B2AC80204603F0ECFAE2
:10FC3000E86028B12246002103F03BFB6E8070BDD6
:10FC4000A8806880FBE7F0B4FF29C1F38107C1F306
:10FC50008112C1F30115477401F003078CBF002125
:10FC600001210170C168C47C067CC274057487746C
:10FC700061B1A41B6142A2EB050561416A426A4180
:10FC8000914203D04188F0BCFFF7BFBFF0BC704782
:10FC900038B5437804460D4633B1B0F90600002864
:10FCA00002DB002101F080F96378E5804BB1284642
:10FCB000012101F079F928460021BDE8384001F022
:10FCC0009BB938BD70B50E460021044641700172E3
:10FCD000C160416119461546FFF7B5FF3146204620
:10FCE000FFF793FF20462946FFF7D2FF204670BD5D
:10FCF00070B540F2FA5404FB00F303F500431B1403
:10FD0000B3F5FF7F98B222DAFE2BD8B242DDC0F104
:10FD1000FE00C5B20023FF204E1CC943C9B2704388
:10FD2000013201EB2020504300F47F4406FB03F036
:10FD300006FB05F301EB202001EB232150434A434E
:10FD4000120244EA102002F47F02104370BDB3F5A2
:10FD50007F7F0DDAB0F53F7FDBB28BBFC3F1FC03D1
:10FD60000233D8B2DBB294BFFF20FF230025D3E7D4
:10FD7000A04211D040F2FA44A042DBB204D80433CE
:10FD8000DDB20020FF23C7E7C3F1FA03DBB2002096
:10FD9000FF25C1E70023FBE700231846F8E7000032
:10FDA00070B50446083015460E4600F0C3F8FF2330
:10FDB000064A84F822300023266025712361A3823D
:10FDC000C4E906222384204670BD00BF0BA10100B8
:10FDD0000161828270470000024B002908BF19466A
:10FDE000816170470BA10100024B002908BF194631
:10FDF000C16170470BA101000184704773B50D46C6
:10FE000001690446164639B92B4BC2685B689A42B1
:10FE100002D1002002B070BDA28A002AF9D094F865
:10FE2000223005F007000341DB0738D515F47E7F4B
:10FE300008BF238C206804BF03F47E731D4303684E
:10FE400000292ED05B6A98470128E2D13C21206826
:10FE500000F0CDF80A222946206800F024F9237921
:10FE600033BB1649206800F0B5F8A169206800F09E
:10FE7000BAF82021206800F0BAF8E169206800F0A3
:10FE8000B2F82379B3B90E49206800F0A3F83146DF
:10FE9000206800F0A8F8206803689B6A9847012052
:10FEA000B8E708490091E16801911B6A6946CAE711
:10FEB0000549D7E70549E7E7D8070020EC9B010093
:10FEC000F29B0100749C0100FF7D0100FD9B01007D
:10FED00008B5FFF793FF08BD07B5002300931A4646
:10FEE0001946034800F02EF803B05DF804FB00BF8C
:10FEF000D80700202DE9F84306460D46071D00F1FE
:10FF00000709002417F8011B0A22284600F0E4F82C
:10FF10002E218046284600F06AF84F4540440444AC
:10FF2000F0D10A22F179284600F0D6F82044BDE845
:10FF3000F8830000024A026000224260704700BF5E
:10FF4000749C010030B58371034D9DF80C30056041
:10FF500001714271C37130BD749C0100014AC0E956
:10FF600000217047749C0100024A02600A684260E6
:10FF7000704700BF749C01000B684360704741608C
:10FF800070472DE9F04106460D4601EB02080C468C
:10FF90004445A4EB050707D0336814F8011B1B6820
:10FFA000304698470028F3D13846BDE8F08170B557
:10FFB000044608460D4604F022F923680246294605
:10FFC00020465B68BDE87040184709B1FFF7EFBFF6
:10FFD0000846704708B5FFF7F8FF08BD03688A6850
:10FFE0005B680968184708B5FFF7EFFF08BD0368AD
:10FFF0001B6818470149FFF7DABF00BFC89B010023
:020000021000EC
:1000000038B50546FFF7E1FF04462846FFF7F2FF43
:10001000204438BD38B50546FFF7D7FF04462846CB
:10002000FFF7E8FF204438BD70B58AB00D460AA935
:10003000002301F8043D012A98BF0A22B5FBF2F41F
:1000400002FB1456F3B2092E94BF30333733DBB2C0
:10005000254601F8013D002CF0D1FFF7B6FF0AB0AC
:1000600070BD2DE9F04107460E4615462AB90368D2
:10007000C9B21B68BDE8F04118470A2A05D100291A
:1000800005DBBDE8F041FFF7CFBFD2B2F9E72D2184
:10009000FFF7ADFF2A46044671423846FFF7C4FF1A
:1000A0002044BDE8F081FFF7DCBF38B50546FFF717
:1000B000D8FF04462846FFF79DFF204438BD10B402
:1000C0002AB903685DF8044B1B68C9B21847D2B25D
:1000D0005DF8044BFFF7A8BFFFF7F1BFFFF7EFBFD5
:1000E0002DE9F84F19460646104614461D469DF860
:1000F000287002F089FD28B14C493046BDE8F84F20
:10010000FFF755BF25F000494FF0FF32484B20461E
:10011000494602F079FD48B94FF0FF32444B204682
:10012000494602F053FD08B94249E6E74FF0604204
:10013000414B2046294602F05DFD08B13F49DCE70E
:100140004FF060423E4B2046294602F035FD002824
:10015000F4D1002200232046294602F02DFDD0B123
:100160002D213046FFF743FF05F1004382461D462F
:100170003449DFF8D8904FF0000B00204FF0000812
:100180005FFA8BF39F4208D942464B4602F0CCFB04
:100190000BF1010BF4E78246EAE722462B4602F018
:1001A000E3F80D46044602F06DFD0A220146804642
:1001B0003046FFF739FF8244A7B3404602F010FAF9
:1001C00002460B462046294602F0CCF804460D466E
:1001D00030461D49DFF87490FFF7E9FE4FF0000844
:1001E0008244013FFFB2FF2F1CD04B4642462046BF
:1001F000294602F06FFA0D46044602F01BFD0A2262
:10020000014683463046FFF72CFF8244584602F0F1
:10021000F7F902460B462046294602F0A3F80446A9
:100220000D46DEE75046BDE8F88F00BF789C010020
:10023000FFFFEF7F7C9C0100FFFFEF41809C0100EE
:10024000FFFFEFC10000E03FBB9101000000244030
:100250009DF800100091FFF743BF08B54022002130
:1002600003F027F80022C0E9102208BD026C10B587
:10027000531C446C03F03F039C421CBF8154036435
:1002800010BD0023C0E910337047D0E9102393421A
:100290001FBFC25C013303F03F03436414BF104629
:1002A0004FF0FF307047D0E91030181A48BF403087
:1002B0007047D0E91023934214BFC05C4FF0FF3069
:1002C0007047036C406C013303F03F031B1A584224
:1002D000584170470649074A074B9B1A03DD043B08
:1002E000C858D050FBDC00F037F8EFF7A9FF00004A
:1002F0001CA1010000000020A0020020FEE7FEE794
:10030000FEE7FEE7FEE7FEE7FEE7FEE7FEE7FEE7C5
:10031000044B1868421C04BF034B1878831F5842D3
:100320005841704730010010E00F00F0074B1B7878
:10033000062B09D1064B1B68C3F30313033B032BA6
:1003400002D8044AD05C704700207047E00F00F0EC
:10035000E80F00F0889C010008B5FFF7D9FF28B12D
:10036000654B664A1B68C3F304231360FFF7DEFF87
:1003700010B1634B634A1A60FFF7CAFF28B1624BA2
:10038000624A1B68C3F342331360FFF7CFFF20B10B
:100390005F4AD36823F08073D360FFF7B9FF40B1A1
:1003A0004FF080430022C3F80C21C3F81021C3F89A
:1003B0003825FFF7BBFF10B1564B03221A60FFF739
:1003C000B5FF40B1544B05221A6001229A67002202
:1003D0009A603F225A60514B1A68511C0BBF504B18
:1003E000504B1A781B6802BF08331B68C3F3031312
:1003F000062A4DD1033B032B03D84B4AD35C002B79
:1004000046D04FF08052494BD2F80414C3F820155F
:10041000D2F80814C3F82415D2F80C14C3F8281520
:10042000D2F81014C3F82C15D2F81414C3F83015F0
:10043000D2F81814C3F83415D2F81C14C3F84015B8
:10044000D2F82014C3F84415D2F82414C3F8481580
:10045000D2F82814C3F84C15D2F82C14C3F8501550
:10046000D2F83014C3F85415D2F83414C3F8601518
:10047000D2F83814C3F86415D2F83C14C3F86815E0
:10048000D2F84014C3F86C15D2F84424C3F8702590
:10049000FFF73EFF28B1264B264A1B6803F04F03A7
:1004A0001360FFF735FF48B14FF08043D3F80024C5
:1004B000D20744BF6FF00102C3F80024174B1B683A
:1004C000062B09D1174B1B68033B022B81BF1A4A2D
:1004D000136843F480631360184AD2F8883043F4F9
:1004E0007003C2F88830BFF34F8FBFF36F8F144B88
:1004F000144A1A6008BD00BF2403001040350140B3
:1005000074C007400DF0ADBA440200103C05004035
:10051000F0ED00E0A0050040105600403001001052
:10052000E00F00F034010010849C010000C0004086
:1005300058020010E40E00403C17004000ED00E0BF
:10054000180000200090D00310B5044600F03EFBD8
:10055000E06023682046DB689847002808DA00F04E
:1005600035FBE368C01AA3689842F2D34FF0FF301E
:1005700010BD2DE9F04180460D468F180C46BC4257
:10058000A4EB050607D04046FFF7DEFF002802DB9C
:1005900004F8010BF3E73046BDE8F0812DE9F8439C
:1005A0008046894616461C467BB1D7181546BD4283
:1005B000A5EB060409D04046FFF7C6FF002804DB80
:1005C000814502D005F8010BF1E72046BDE8F8832C
:1005D00070B50D4609490446164600F0D1F9284683
:1005E000FFF7B2FF002806DB864204D0C1B22046E6
:1005F00000F044FAF3E7204670BD00BFCA9B01003B
:100600000120704703681322DB69184770470369AC
:10061000C3F81C150369D3F81C21002AFBD0002263
:10062000C3F81C210120704710B490F95C30144CC1
:1006300059090122203103F01F0302FA03F344F8A1
:10064000213003695DF8044B0421C3F808130369E2
:100650005A600369DA6003690022C3F80025026961
:100660004FF0FF33C2F80C350269C2F81435026945
:10067000C2F8083502691430C2F81035FFF701BE20
:1006800000E100E01430FFF70EBE1430FFF711BE9A
:100690001430FFF7FABD0000036990F85E2010B532
:1006A000C3F80C25036990F85D20C3F8142590F871
:1006B00061200369012A01BF90F85F40C3F810452B
:1006C000036990F8604006BFC3F80845036900223B
:1006D000B1F5966FC3F86C2569D9B1F5166F69D974
:1006E000B1F5965F69D9B1F5165F68D9B1F5615F6B
:1006F00067D9B1F5964F66D9B1F5E14F65D9B1F536
:10070000164F64D9B1F5614F64D9B1F5963F64D9FC
:10071000B1F5E13F63D9B1F5613F63D9364B9942F9
:1007200063D9B1F5E12F63D9B1F5612F94BF4FF0D3
:1007300070634FF080530269C2F8243503690422C4
:10074000C3F8002501690023C1F808310169C1F827
:100750001C31016901230B6001698B600169C1F8DB
:10076000042390F95C20510902F01F02934060318C
:10077000224A42F8213090F95C30002BBDBF03F0D3
:100780000F0302F6FC32D2189B18B5BF602360221B
:10079000137683F8002390F95C300122590903F0A5
:1007A0001F0302FA03F3154A42F8213010BD4FF43B
:1007B0009E23C0E74FF41D23BDE7114BBBE7114B50
:1007C000B9E7114BB7E7114BB5E7114BB3E74FF45E
:1007D0001D03B0E74FF46B03ADE70E4BABE74FF0F3
:1007E000EB73A8E74FF06C73A5E74FF08063A2E7C7
:1007F0004FF0E8639FE700BF90D0030000E100E006
:1008000000B013000050270000F03A0000A04E0096
:1008100000C0750000903A012DE9F0411E46002508
:100820004FF47A73C0E901530D4B044640F8143B72
:1008300017468846FFF711FD0A4AC4F8108084F86D
:100840005C7052F8263084F85D309DF8183052F80C
:10085000233084F85E3084F861502046BDE8F08192
:10086000949C0100049C010010B50369D3F8082191
:1008700004464AB1D3F818151430C9B2FFF7F6FC94
:1008800023690022C3F8082110BD00000148FFF7CA
:10089000EBBF00BFE007002007B519230093022239
:1008A000182303490348FFF7B7FF03B05DF804FBC3
:1008B00000200040E007002010B5044628B103F0F6
:1008C00047FB90FBF4F303FB1404204610BD884261
:1008D00010B5044603DA081AFFF7EEFF0444204679
:1008E00010BD10B5029C401AE41A6043521A90FBE6
:1008F000F2F0184410BD10B50446006802F08CFCFC
:10090000204610BD10B50446006808B102F084FC12
:1009100000232360C4E9013310BD38B504460D46F9
:100920000068013103F048FB10B1C4E90005012063
:1009300038BD036810B5044623B143688B4201D328
:10094000012010BD2046FFF7E8FF0028F9D0A3687A
:10095000002BF5D122681370F2E770B50E461146F0
:1009600004461546FFF7E5FF20B92046FFF7CAFF0A
:10097000204670BDA5603146206803F01CFCF7E7F7
:1009800038B500230446C0E9003383600D4639B111
:10099000084603F034FC294602462046FFF7DDFFF7
:1009A000204638BD38B5054608460C4603F027FCFE
:1009B000214602462846BDE83840FFF7CEBF38B58D
:1009C000054600680C4668B16A688B689A4207D38E
:1009D000096803F0F0FBA368AB600023A36038BD97
:1009E00002F01AFC23682B6063686B60A368AB603D
:1009F0000023C4E90033F1E7884210B50B460446F2
:100A000004D0096821B19A68FFF7A7FF204610BDFE
:100A1000FFF778FFFAE710B500230446C0E900337A
:100A20008360FFF7E9FF204610BD884210B50446F9
:100A300001D0FFF7C4FF204610BD10B5044619B120
:100A4000FFF7B0FF204610BDFFF75CFFFAE770B577
:100A500005460E4609B9002070BD6AB18468144489
:100A60002146FFF766FF0028F5D02868AB683146BD
:100A7000184403F0A0FBAC600120EDE707B50023AC
:100A80008DF80410012201A98DF80530FFF7DFFF72
:100A900003B05DF804FB10B58A6809680446FFF7E7
:100AA000D6FF10B92046FFF72DFF204610BD826803
:100AB00008B53AB921B10878B0FA80F0400900E0F1
:100AC000012008BD006809B90078F5E703F069FB6B
:100AD000F2E7884270B515D083688A6893420FD1D7
:100AE00083B104680D68013C14F8010F50B104F0A3
:100AF0009BFB064615F8010B04F096FB8642F3D0EB
:100B0000002070BD0120FCE783688B4201D900689A
:100B100018B903480023037070470844704700BFAA
:100B2000440800208368934210B506D90468A018D1
:100B300003F02AFB08B1001B10BD4FF0FF30FBE7AC
:100B40000022FFF7EFBFF8B583689342054602D84D
:100B50004FF0FF30F8BD0368541C00221F5D1A558A
:100B60000668304603F09AFB37550028F0D02B6812
:100B7000C01AEFE78268013AFFF7E5BF2DE9F041BF
:100B80009A420E461F460F4988BF134615468046B7
:100B900084BF3D461F46FFF7F3FEB468AC420DD953
:100BA000BC4228BF3C46336800221F5D1A5531689D
:100BB00040462944FFF741FF33681F554046BDE8D2
:100BC000F08100BFCA9B0100FEE700000A4B1968D4
:100BD0000A4B30B5D3F804050C060D0A44EA0002AE
:100BE0004FF47A712B46A2FB014501FB0355E00B44
:100BF00040EA454030BD00BF4808002000100140D9
:100C0000094B1968094B30B5D3F804050D0A0C06D9
:100C1000074944EA00022B46A2FB014501FB0355AC
:100C2000E00B40EA454030BD48080020001001407C
:100C300040420F0038B5044648B1FFF7C7FF0546EC
:100C400000F01AF8FFF7C2FF401BA042F8D338BDEE
:100C5000074B0022C3F8042182B0D3F80431054ABF
:100C60000193019B13680133DBB2136002B070473C
:100C70000010014048080020704770B58AB061B18B
:100C8000931E222B20D801AB1D4648B9AB4207D09A
:100C90000A46AB4213D80023137008460AB070BD51
:100CA000B0FBF2F402FB1406092E204603F1010307
:100CB000F4B294BF3034573403F8014CE5E713F82D
:100CC000010D02F8010BE4E70021E6E770470000A0
:100CD00008B500F015F8FFF7F9FF0120FFF7AAFFAC
:100CE000F4F746FE034CF4F745FE002CFBD0AFF3BF
:100CF0000080F8E70000000002F086BA02F08CBA2B
:100D00002A4BE02283F811234FF40032C3F88021EC
:100D10001A604FF080430122C3F818259A6003F54A
:100D200088330021C3F808150221C3F80413C3F85F
:100D300044131A604FF01023D3F80022002A03DB7B
:100D4000D3F80432002B2FDA194B0122C3F8042503
:100D5000D3F80024002AFBD04FF010221521C2F84E
:100D60000012D3F80024002AFBD04FF010231522E4
:100D7000C3F804220E4B1A46D3F800140029FBD006
:100D80000021C3F80415D2F80034002BFBD0BFF3C8
:100D90004F8F0849084BCA6802F4E0621343CB60E6
:100DA000BFF34F8F00BFFDE7704700BF00E100E0D9
:100DB00000E0014000ED00E00400FA05192837B515
:100DC0000CD84B4B53F82030052B00F0828007D80D
:100DD000032B12D07BD8022B00F08180002074E01E
:100DE0001D2B78D003D81C2BF8D1052206E01E2B32
:100DF00073D01F2BF2D1082200E002223D4B19686C
:100E000008296EDD0A296FDD0D29B5BF0C240E24DB
:100E1000022303233848C0F8F0350123C0F8003519
:100E200000200546030103F1804303F5E043013050
:100E30000828C3F81455C3F81055F3D12F4B186880
:100E40002F4B1B6800021B0303F4805300F4E06087
:100E50001843294BC3F81805C3F81425C3F8102507
:100E60000DF10602C3F82C260122C3F830261A60C1
:100E7000D3F80021002AFBD00022C3F80021012270
:100E80005A601D4B1A46D3F804010028FBD00020FD
:100E9000C3F8040101209860D2F81431002BFBD074
:100EA0000023C2F81431BDF906209A42124AB8BF95
:100EB000ADF80630A142C2F80035BDF9060004D0F5
:100EC00035BF611A091BC840884003B030BD0322FA
:100ED00094E7042292E7062290E707228EE7012298
:100EE0008CE70824002395E70A24012392E700BF3A
:100EF000049C010028000020007000402C0000200D
:100F000054080020192830B53CD8224B53F8200053
:100F1000214B00221D4653F82240B4F1FF3F32D14D
:100F20001E4C45F822006FEA41411D4D1D4B2468BF
:100F300053F822306FEA514125F81210012101FACD
:100F400004F4C3F86005013CC3F8640505EB4202F4
:100F5000C3F86805C3F86C050020C3F80015C3F892
:100F60000C05C3F80405C3F80845C3F81405C3F815
:100F70001005C3F82025C3F82415C3F82815C3F8B5
:100F80002C05996030BD8442CAD00132032AC2D1F7
:100F9000F8E700BF049C01001C0000203000002086
:100FA0004C080020BC9C010019280FD8114B53F8A5
:100FB000203003290AD8DFE801F002160A1003F5F1
:100FC000E0734FF0A042002142F82310704703F570
:100FD000E0734FF0A0420C21F6E703F5E0734FF009
:100FE000A0420421F0E703F5E0734FF0A042032193
:100FF000EAE700BF049C010019280CD8064B53F8FF
:101000002020012393404FF0A04211B9C2F80C35C3
:101010007047C2F808357047049C010019289FBF2B
:101020004FF0A043054AD3F8103552F820009ABF7C
:1010300023FA00F000F0010000207047049C01003A
:1010400038B50025057329B90B4B0C4A0C482521EE
:1010500001F088FE01600B4951F82220027151F81D
:10106000233083719DF8103051F8233043710223EF
:10107000C371856038BD00BFC89C01002B9D010075
:10108000D69C0100049C0100037B23B94373837346
:10109000036101230373704784B00DF1100C0CE958
:1010A0000E009DF80810026800230129C2F80035DF
:1010B000039B12D00BD303290CD0C2F85435019BEB
:1010C000C2F824350123C2F8003504B0704743F05C
:1010D0000203F2E743F00403EFE743F00603ECE713
:1010E00010B5FFF7D1FF03688279C3F8082542796C
:1010F000C3F80C250279C3F81025034BBDE8104056
:101100000ECBFFF7C9BF00BF6C08002010B485B03C
:1011100001AC84E80E0094E80E0005B05DF8044BC5
:10112000FFF7BABF70470368C3F81C15D3F808214E
:10113000002AFBD0D3F818050022C3F80821C0B25A
:101140007047000007B5094B09490A484FF0804233
:101150001A6000229A6002221A710B2300930C225B
:101160000D23FFF76DFF03B05DF804FB6C08002052
:1011700000300240580800200B460146184601F096
:101180001BBE0000C0F3C7537F3B162B024605DC95
:10119000002B04DB0348184122EA0000704700F0EE
:1011A00000407047FFFF7F002DE9F04FDFF82C93E0
:1011B0008DB006460F4614461D4600F095F999F984
:1011C0000080B8F1FF3FCDE9000136D022462B4622
:1011D0002046294601F018FD834670BB32463B4647
:1011E0003046394601F010FD8246002840F0A280CA
:1011F000304639460022002301F0D4FC10B300220F
:1012000000232046294601F0CDFC8346002867D004
:101210009FEDA77B0122AC4BCDF828A00292CDE92F
:101220000467CDE906458DED087B0393B8F1000F07
:1012300041D09FEDA17B8DED007BDDE900010DB07C
:10124000BDE8F08FDDE9000100F066FF8046002870
:1012500000F08D804FF0000A4FF0000BDDE9000137
:1012600052465B4601F09EFC0028E6D030463946E7
:1012700000F052FF0028E0D02046294600F04CFF45
:101280000028DAD099F900308F4A03920421002215
:10129000022BCDE90467CDE90645CDE908AB029103
:1012A0000A9203D002A800F03DFF50B901F092FD70
:1012B0002223036005E002A800F034FF002800F0BC
:1012C0009B800A9B1BB101F085FD0A9B03609DED8D
:1012D000087B8DED007BDDE900010DB0BDE8F08FEE
:1012E0002046294600F018FF0028A6D0002200233F
:1012F0002046294601F060FC00289ED0724A99F9E8
:101300000030CDF828B00121CDE90467CDE90645CC
:10131000CDE90212002B74D06C490020022BCDE9DC
:10132000080172D101F056FD212303600A9B002BB6
:10133000CDD0C8E7002200232046294601F032FC28
:1013400000283FF47AAF624B5F49CDF828B0002205
:101350000120B8F1020FCDE904670290CDE90645FE
:10136000CDE908230391A6D1CDE9002365E73046F6
:10137000394600F0D1FE00283FF46CAF20462946E4
:1013800000F0CAFE00283FF465AFDDE900231046F7
:10139000194601F039FC99F900A000286BD103230C
:1013A000DFF824C10A902946204602930022494BC7
:1013B000CDF80CC0CDE90645CDE9046701F08AF906
:1013C00004460D46BAF1000F25D1DFF814B14FF0F5
:1013D000604A0022002330463946CDE908AB01F0CF
:1013E000EBFB38BB02A800F09DFE00289ED101F067
:1013F000F1FC2223036099E701F0ECFC2123036058
:101400005FE79FED2B7B8DED087B02A800F08AFE45
:1014100000288BD186E79FED2A7B002200233046EF
:1014200039468DED087B01F0C7FBA0B9BAF1020F78
:10143000DDD0D7E72046294600F07CFE22462B4629
:1014400001F0B0FBA0B9244B99F900A04FF0604225
:10145000CDE90823EAE72046294600F06BFE224644
:101460002B4601F09FFB18B9184B0022CDE9082349
:1014700099F900A0DAE70122134BCDF828800292F7
:10148000CDE90467CDE906450393BAF1000FB8D062
:10149000002200231046194601F046FABAF1020F65
:1014A000CDE908013FF43EAFAFE700BFAFF30080E6
:1014B0000000000000000000000000000000F03FFD
:1014C000000000000000F07F689D01000000F0FFB8
:1014D0000000F03F0000E03FFFFFEFC734000020B6
:1014E000FFFFEF47000000002DE9F04F23F000451B
:1014F00055EA020493B00DD06B4E21F00044B44283
:101500000F4682460BDD04F1404404F5801454EA92
:101510000A0350D16549002013B0BDE8F08F9B4607
:10152000944647D0B542EEDC5F4EB5425DD0002F09
:1015300080468946CDE900235BDB0026BCF1000F25
:101540000ED1594B9D423FD0584B9D4200F08880B0
:10155000BBF1804F00F09C80554B9B4500F0B88359
:101560004046494600F0D4FDBAF1000F06D1002CE8
:1015700059D04E4B27F040429A4254D0FF0F013FC2
:1015800056EA070373D04B4B9D4240F39B8003F117
:1015900004739D4240F33E84474B9C4272DDBBF195
:1015A000000F72DD3EA3D3E900231046194601F077
:1015B00091F8B1E728B1414813B0BDE8F04F00F011
:1015C000B3BDA542F7DCAFE704F1404303F5801358
:1015D00053EA0A039ED0384B9C4240F38383BBF10D
:1015E000000F52DBDDE9000196E7BCF1000F9ED051
:1015F00089E7334B9D4231DCA3F154739D429CDD5E
:101600002B15A3F2FF33142B40F3A583C3F134034E
:101610002CFA03F202FA03F363458ED102F00102C1
:10162000C2F102068AE7BBF1000F05DA02460B465B
:1016300000201E4901F078F9002FBFF66DAF04F1CC
:10164000404404F5801454EA060300F03F84012E60
:101650007FF462AF01F1004319465DE702266DE7B2
:10166000BBF1000FC0F248834046494654E742466A
:101670004B461046194600F075FE02460B4601F037
:1016800053F949E7BBF1000F8CDB0020002143E751
:1016900042464B464046494601F01CF83CE700BF35
:1016A0009C7500883CE4377E0000F07F0000F03F2E
:1016B0000000E03F0000E041FFFFEF3F6C9D0100B4
:1016C000FFFF3F43B4F5801F80F261830022D24BBD
:1016D00001F000F86FF0340C0C462315CF4DC4F325
:1016E0001302A3F2FF3342F07F546344AA420B93E8
:1016F00044F4401440F33F83C94B9A4240F30484BE
:101700009FEDAF7B8DED087B8DED107B9FEDAE7B6C
:101710000B9B8DED067B01330B93A4F58014002504
:10172000DDE906232146824600F01CFEA346DDE9E2
:1017300006238046894650462146CDE90CAB00F091
:1017400013FE02460B460020B64901F0EDF80A46AA
:101750000146CDE90E12134649460246404600F0C6
:10176000B9FF631043F0005382468B4603F5002314
:101770008C46CDE904AB5919D3460023CDE902BC10
:101780000293DDE902AB002004460D4602460B46FB
:101790005046594600F09EFF02460B4640464946D9
:1017A00000F0E0FDDDE90623804689462046294613
:1017B00000F0D8FD02460B46DDE90C0100F0D2FD39
:1017C00052465B4600F086FF02460B4640464946BD
:1017D00000F0C8FDDDE90E2300F07CFFDDE90445E3
:1017E000CDE9060122462B462046294600F072FF2D
:1017F00077A3D3E9002304460D4600F06BFF76A3E0
:10180000D3E9002300F0B0FD22462B4600F062FF32
:1018100073A3D3E9002300F0A7FD22462B4600F076
:1018200059FF71A3D3E9002300F09EFD22462B4609
:1018300000F050FF6EA3D3E9002300F095FD22468F
:101840002B4600F047FF6CA3D3E9002300F08CFD8A
:101850002246804689462B462046294600F03AFF1C
:1018600002460B464046494600F034FF52460446C5
:101870000D465B46DDE9040100F076FDDDE9062357
:1018800000F028FF22462B4600F06EFD52468046AF
:1018900089465B465046594600F01CFF0022624BC9
:1018A000CDE90C0100F060FD42464B4600F05CFDC6
:1018B00002980D46044622462B465046594600F0F3
:1018C00009FF002282468B46574B2046294600F0EE
:1018D00049FDDDE90C2300F045FD02460B4640467C
:1018E000494600F03FFDDDE9042300F0F3FE224607
:1018F000804689462B46DDE9060100F0EBFE0246F4
:101900000B464046494600F02FFD80468946024678
:101910000B465046594600F027FD029838A3D3E9FC
:10192000002304460D4600F0D5FE5246CDE90401E1
:101930005B462046294600F015FD02460B46404610
:10194000494600F00FFD30A3D3E9002300F0C2FEAA
:101950002FA3D3E90023804689462046294600F07C
:10196000B9FE02460B464046494600F0FDFCDDE963
:10197000102300F0F9FC80460B98894600F040FEE9
:10198000424682468B464B46DDE9040100F0ECFC02
:10199000DDE9082300F0E8FC52465B4600F0E4FC79
:1019A000029852465B4604460D4600F0DBFCDDE93A
:1019B000082300F0D7FCDDE9042337E0AFF3008013
:1019C0000000000000000000000000000000F03FE8
:1019D000EF4E454A287ECA3F65DBC9934A86CD3F14
:1019E00001411DA96074D13F4D268F515555D53FFA
:1019F000FFAB6FDBB66DDB3F033333333333E33F92
:101A0000000000E009C7EE3FFD033ADC09C7EE3FE6
:101A1000F5015B14E02F3EBE000040438E980300AA
:101A200079B60B000000F03F0000084000F09AFC7F
:101A30000B4602464946404600F094FC013E56EAF9
:101A4000070382468B4600F05E819FEDD37B8DEDD0
:101A5000047BDDE9001200230E461746CDE902673C
:101A60000293DDE9026708463B461146324600F024
:101A700079FC22462B4600F02DFEDDE9002380464E
:101A800089465046594600F025FE02460B46404620
:101A9000494600F069FC3246804689463B4620466E
:101AA0002946CDE9008900F015FE0B4602460646A0
:101AB0000F464046494600F057FCD14B9942044638
:101AC0000D468A4640F3248101F13F4303F5E003CC
:101AD000034340F0FF81B2A3D3E90023DDE9000115
:101AE00000F042FC3246804689463B462046294665
:101AF00000F038FC02460B464046494601F07AF8B1
:101B0000002840F0E781A8464FEA2853A3F2FE32AE
:101B10004FF4801313415344C3F30A52B94DA2F258
:101B2000FF321541C3F3130423EA05010020C2F17B
:101B3000140B44F48014BAF1000F02460B4644FA29
:101B40000BFB30463946B8BFCBF1000B00F00AFC66
:101B500006460F463246DDE900013B4600F004FC34
:101B60004FEA0B5A0D4600248FA3D3E900232046E9
:101B7000294600F0AFFD3246804689463B46204666
:101B8000294600F0EFFB02460B46DDE9000100F0BC
:101B9000E9FB87A3D3E9002300F09CFD86A3D3E9EA
:101BA000002306460F462046294600F093FD0246D4
:101BB0000B463046394600F0D7FB06460F46024634
:101BC0000B464046494600F0CFFB42464B46044692
:101BD0000D4600F0C7FB02460B463046394600F082
:101BE000C1FB2246804689462B462046294600F006
:101BF00071FD73A3D3E9002306460F4600F06AFD8A
:101C000071A3D3E9002300F0ADFB32463B4600F060
